:020000040000FA
:040000006FD00400B9
:101000006F1000140000000000000000902000207D
:10101000B2270020A9BDF9F56828002000000000D3
:101020000000000068280020902000200000000040
:101030000000000090200020000000009020002010
:101040000000000090200020902000209020002030
:101050009020002090200020B4300020902000201C
:10106000000000009020002090200020F4280020A4
:1010700090200020CE2800209020002090200020EA
:101080009020002090200020902000209020002020
:101090009020002001A04111B7170040985F3AC688
:1010A000945F3247E39CE6FE324541018280411164
:1010B000814601468145114506C6EF009014B727C9
:1010C000004011472383E780B7F700E003A707D16B
:1010D0006D9B23A8E7D003A707D15D9B23A8E7D08A
:1010E0007300501001000100B240410182800111E3
:1010F000814601468145114506CEEF009010B72785
:10110000004011472383E780B717004083C6E702FA
:1011100003C5E7041307800893F6C60F136535006F
:1011200093E61600733607801376860832C00100F6
:101130000100930570052380B704130680FA23800D
:10114000C70401000100238207022380070402482C
:10115000732808800100010073380780137888081D
:1011600042C2010001002380B7042380C7040100AC
:1011700001002387D7022387A70423800704924610
:10118000F3A6068001000100F336078093F6860877
:1011900036C4010001002380B7042380C704010086
:1011A000010083C6B70493E60602A385D704238013
:1011B0000704A246F3A6068001000100B7F600E08E
:1011C00003A506D11365450023A8A6D003A506D123
:1011D0005D9923A8A6D07300501001000100733759
:1011E0000780137787083AC6010001002380B704FF
:1011F0002380C7040100010003C7B7041377F70D6C
:10120000A385E70423800704B247F3A70780010002
:101210000100F240056182803971B7F5070022DCD8
:1012200081462A843010E105194506DE02D42316D2
:101230000102EF00007DB717004083C6E7041307E3
:10124000800893E63600733607801376860832C42A
:1012500001000100930570052380B704130680FA8E
:101260002380C704010001002382070223800704B2
:101270002245732505800100010073350780137531
:1012800085082AC6010001002380B7042380C70413
:10129000010001002387D70423800704B246F3A688
:1012A000068001000100F336078093F6860836C8F1
:1012B000010001002380B7042380C704010001005E
:1012C00003D50702F176FD16E98E2390D70223801D
:1012D0000704C246F3A606800100010037F500E0CE
:1012E000832605D193E646002328D5D083D607026E
:1012F0006575110593F60660C18EC98EC206C1825E
:1013000073350780137585082ACA01000100238000
:10131000B7042380C7040100010003C5F70013656B
:101320000504A387A7002390D70223800704D24691
:10133000F3A60680010001001165618D1DE9733778
:101340000780137787083ACC010001002380B70497
:101350002380C7040100010003C7B7041367070215
:10136000A385E70423800704E247F3A70780010071
:10137000010037F700E0832707D1DD9B2328F7D052
:10138000730050100100010013078008F337078035
:1013900093F787083ECE01000100B7170040930580
:1013A00070052380B704130680FA2380C704010068
:1013B000010083D60702C606C5822390D702238088
:1013C0000704F246F3A6068001000100F336078009
:1013D00093F6860836D0010001002380B7042380ED
:1013E000C7040100010003D80702F176FD16B3F629
:1013F00006012390D702238007048256F3A60680B5
:10140000010001000DED73370780137787083AD28A
:10141000010001002380B7042380C70401000100FC
:1014200003C7B7041377F70DA385E70423800704E8
:101430009257F3A70780010001005145ED2EF250AD
:10144000625421618280397152D481462A8A0146D0
:101450008145114522DC26DA06DE4AD84ED63714FD
:10146000004045238347E4020347E40493048008D3
:1014700093F7C70F1367370093E71700F3B604809D
:1014800093F6860836C60100010093097005230013
:101490003405130980FA230024050100010023020A
:1014A000040223000404B246F3A6068001000100F2
:1014B000F3B6048093F6860836C8010001002300C5
:1014C000340523002405010001002307F40223074B
:1014D000E40423000404C247F3A7078001000100CD
:1014E00013055002E128B7F700E003A707D11367FF
:1014F000470023A8E7D073B70480137787083ACA58
:10150000010001002300340523002405010001002F
:101510000347F40013670704A307E400230004044F
:101520005247732707800100010073B704801377C7
:1015300087083ACC0100010023003405230024056C
:10154000010001002167336AEA00231044032300ED
:1015500004046247732707800100010003A707D135
:101560005D9B23A8E7D07300501001000100814665
:101570000146814511457121F3B4048093F4840838
:1015800026CE0100010023003405230024050100BC
:1015900001008347640493E717002303F404230046
:1015A0000404F247F3A7078001000100F2506254DF
:1015B000D2544259B259225A216182800111130733
:1015C0008008F337078093F787083EC201000100C7
:1015D000B7170040930570052380B704130680FAFF
:1015E0002380C7040100010083C6B70493F6F60DFB
:1015F000A385D704238007049246F3A60680010042
:10160000010093760502D5CEF336078093F686085F
:1016100036C4010001002380B7042380C704010001
:101620000100B70614007D89558D88C701000100AF
:101630000100010023800704A246F3A606800100F2
:10164000010073370780137787083AC6010001004D
:101650002380B7042380C7040100010001000100BA
:101660003727004093061005A303D7802380070483
:10167000B247F3A707800100010093078008F3B782
:10168000078093F787083ECE01000100B71700409E
:10169000130770052380E704130780FA2380E7040B
:1016A0000100010003C7B70413670708A385E70417
:1016B00023800704F247F3A70780010001000561BA
:1016C000828093760504BDC6F336078093F68608BC
:1016D00036C8010001002380B7042380C70401003D
:1016E0000100B7061400938606047D89558D88C7CE
:1016F000010001000100010023800704C246F3A697
:1017000006800100010073370780137787083ACA03
:10171000010001002380B7042380C70401000100F9
:101720003727004093062005A303D78023800704B2
:10173000D24781B773370780137787083ACC010007
:1017400001002380B7042380C704010001009847EB
:101750001367070C98C723800704E24719BF0111DC
:10176000814601468145114506CE612C93078008CC
:10177000F3B7078093F787083EC601000100B7174B
:101780000040130770052380E704130780FA2380C5
:10179000E7040100010003C76704136717002383F0
:1017A000E70423800704B247F3A707800100010084
:1017B000F240056182804111814601468145114513
:1017C000892413078008F337078093F787083EC4FE
:1017D00001000100B7170040130670052380C704FD
:1017E000930680FA2380D70401000100FD5523965B
:1017F000B70223800704A245F3A50580010001007C
:1018000073370780137787083AC6010001002380E9
:10181000C7042380D7040100010003C767041367CE
:1018200017002383E70423800704B247F3A7078048
:101830000100010001A0BD473305F50201007D153F
:1018400075FD8280411122C426C206C6AA840144C5
:1018500063179400B24022449244410182800504FF
:101860001305803E4204C13F4180DDB7930500026D
:1018700073A0458082457390153492402242B24253
:101880004243D2436244F244025592552256B25624
:101890004257D2576258F25806499649264AB64AE4
:1018A000464BD64B664CF64C065D965D265EB65EA4
:1018B000465FD65F0961730020304111B7170040C1
:1018C000985F3AC6945F3247E39CE6FE3245410199
:1018D0008280B7170040130700032388E70285477B
:1018E00023A2F18673002030411122C406C63704BA
:1018F00000201C408297F5BF3737004083474700E0
:101900009146BD8B6389D70099466394D70083477E
:1019100057407300203083C6118993871600A3882F
:10192000F18803478700973700009387E73BB69716
:101930002380E700B7E70400BC4F0946894503C58B
:1019400061828297F9B72303048015472303E4805B
:1019500001002302A480828083076480E3CE07FE17
:1019600023030480828083076480E3CE07FE03455F
:101970004480828083076480E3CE07FE2302A48034
:101980008280411126C44AC24EC006C61377F50BA9
:10199000AD47AA892E8995446306F7001945653736
:1019A000653F8D444E854537FD59FD1463983401DC
:1019B000B240A24412498249410182801355090173
:1019C0001375F50F453F2209CDB7011126CC06CE80
:1019D000B704080051371545BD37713769372AC636
:1019E000A53F32459377150089EB136515001375F4
:1019F000F50FF240E24405618280FD14E9FC0145E7
:101A0000CDBF397126DC4ADA4ED852D656D45AD2D6
:101A10005ED006DE62CE66CCB7E700E07D5783AAD3
:101A2000070022C603AA470023A0E71823A2E7184D
:101A3000B7170040130770052380E704130780FAE7
:101A40002380E70483C74704930B75FFB684E2073E
:101A500093FBFB0F8546AA892E8B328937240040E1
:101A6000E187015763FA76016308D50089461307B9
:101A700000026313D5000157D98F93F7F70FB71CF6
:101A800000402382FC0411472303E4801305F00F78
:101A90005D3D094CD135636D7C11B7050700DA95C2
:101AA00037870700795563F2E504B3879500636EC5
:101AB000F702370B0800A94733EB65016399F90674
:101AC00089E48144513D26850DA0DA850945553DBF
:101AD00005090345F9FFFD14050B693D81C49377A2
:101AE000FB0FFDF7DD3569FD7D55B7170040130786
:101AF00070052380E704130780FA2380E70403C7F7
:101B00004704418B2382E704F250B7E700E023A0AB
:101B1000571123A24711E25432445259C259325A42
:101B2000A25A125B825B724CE24C21618280A54713
:101B30006395F90685691309F00FB3069900B3742C
:101B40002B01B6941349F9FFB3749900856B33796F
:101B50006901416B9387F9FFB3F7270199E363FCB0
:101B6000340193D94900C147E3E637FF99BF0569BE
:101B7000C1697D19D9B71305800D63886901130503
:101B800000026384790113051008CA85DD3B353DE9
:101B900021DD4E99B3843441D9B7DA852D45D5334B
:101BA000CA94E30099F205097D3BA30FA9FED5BFB6
:101BB0009387F9FF93F7F70F6361FC0C83C71C044D
:101BC00013073008631FF70437070800636BEB0443
:101BD000B3079B00B706100063F5D704334BEB0047
:101BE00089476393F9068980D549E38C04ECDA854B
:101BF0000945413B11090327C9FF91472320E48090
:101C000003076480E34E07FE23033481FD17EDFBD9
:101C1000FD14110B81C49377FB0FE9FF7D3371F540
:101C2000E1B5B717004003C75704B707080013779B
:101C3000070219E3B78707007955E378FBEA330712
:101C40009B00E3FFE7F855B58547E382F9F2DA85B3
:101C50002D45053B9389F4FFE38504E6293393F78B
:101C6000390091EB8326048003270900930749007C
:101C7000E39AE6E43E89CE84F1BFB5476396F90066
:101C80001305900BC93135BDB1471305B00AE38B7D
:101C9000F9FE99476391F904B7050800B365BB00E5
:101CA0002D45C53181448D4BA14975396396740129
:101CB000832704802320F9008504E39834FF8327D9
:101CC000048013172B01635507002312F900D5BBBD
:101CD0002322F900FDB39D476399F902814513055D
:101CE000B0044531BD442320090023220900FD59D9
:101CF0009D3993F77400CA9703C70700FD14398D07
:101D00002380A700E39634FF6DBBA1476392F904DB
:101D10006D398144630D0B008D479304C003630844
:101D2000FB009304000563048B01930440041375C6
:101D3000C507E30895D819453931393905452131A9
:101D400026850D3909453D314931E31C05D669BB6E
:101D500091476399F90013056006F536F53E1305C2
:101D600090090DB7E38F09D4F154A9BBBD660147B3
:101D70001736000013060624938606A6854583477A
:101D8000060093F7F70F91C382800507E3F9E6FE9B
:101D9000973700002380B722DDB77D166206618683
:101DA00093178601E18763D407000145828093176A
:101DB00026003307F500AE9718439C4363E7E7001E
:101DC0007D16E37FF7FC7D55828005458280FD15F9
:101DD000E205E18513978501618793F7F50F634865
:101DE0000700FD15139725002A97584365D71385DB
:101DF00017006205618582803308B5021C4283A802
:101E00000600B335B502C29733B50701AE984695C3
:101E100085486367B5006394A50063E307018148C3
:101E20000C43C6950CC388C21CC28280814713979D
:101E3000870161876343B7008280139727002A9741
:101E4000232007008507E5B781470147939687015F
:101E5000E18663C5B600133517008280939627008C
:101E6000AA9694428507558FD5B793D755408A07D0
:101E7000AA979C4305453315B5007D8D828017F3E5
:101E8000FFDFE702033B2A84993705C59317250036
:101E90003E940327C4FF814711EB7D1516053E953F
:101EA0004205418517F3FFDF6700E33A05838507A5
:101EB000E5B70145C5BF8147139787016187634334
:101EC000C700828013972700B386E50094422A97C3
:101ED000850714C3D5B77D1662066186014793173F
:101EE0008601E18763D507001335170082809317B9
:101EF0002600B306F500AE9794429C437D16B58F3D
:101F00005D8FF1BF8A05AA9501476363B5008280A2
:101F100083A6C5FFF11593D71600D98F9CC11397DF
:101F2000F601E5B72A830148014701456343D7001D
:101F30008280B387050183A80700B30706019C438D
:101F4000C697AA976384F80033B517010507B3084D
:101F50000301620723A0F80061871108C1BF2A832B
:101F600001478147014563C3D70082803388E5007C
:101F700083280800330EE600032E0E003388A840A5
:101F80003308C8416384080133B508018507B308E5
:101F9000E300E20723A00801E1871107E9B717F37F
:101FA000FFDFE70203290111B286B2842E86AA85DB
:101FB0000A8575372A84A6850A85793533348000E9
:101FC000060413351500018D056117F3FFDF670067
:101FD000832817F3FFDFE70243234111AA89AE8A62
:101FE000328BB68402C202C402C60144131C8401AF
:101FF000135C8C4163499C02939B1400FD1B0549B3
:10200000138CF4FFF15C3304890162046184634D35
:10201000740592478E04CE9423AEF4FE410117F36B
:10202000FFDF6700032213192400B30B2B01014AC1
:1020300093172A00D69783A50B00884378003400B5
:1020400050005D3B050A93178A01E187F11BE351BC
:10205000FCFE92474E9905042320F900A2473EC298
:10206000B24702C63EC459B7131A8901135A8A41AE
:10207000131D240093178A01E18763CF97009247CD
:102080000A044E941CC0A24705091379F90F3EC2F9
:10209000B24702C63EC485BFB3079A0313152A0090
:1020A00056950841780034005000050AEA97DA97FF
:1020B0008C439933C1B70000197106C212C416C609
:1020C0001AC81ECA22CC26CE2AD02ED232D436D658
:1020D0003AD83EDA42DC46DECAC0CEC2D2C4D6C648
:1020E000DAC8DECAE2CCE6CEEAD0EED2F2D4F6D638
:1020F000FAD8FEDA9385C1858841E7000500924051
:102100002242B2424243D2436244F24402559255C3
:102110002256B2564257D2576258F258064996494B
:10212000264AB64A464BD64B664CF64C065D965D43
:10213000265EB65E465FD65F096173002030000000
:1021400097210020938181E6174100201301816BC4
:1021500017F5FFFF130545EB97050020938585EAEA
:10216000171600201306C6FD63FAC500832205007A
:1021700023A0550011059105E3EAC5FE17A501004E
:1021800013054545971500209385C5FB13860184EB
:1021900063FAC5008322050023A0550011059105AF
:1021A000E3EAC5FE13850184974500209385852CBD
:1021B0006377B500232005001105E36DB5FEFD42F0
:1021C000739002BC8D4273904280B72200009382CC
:1021D000828873900230970200209382A2E293E2F9
:1021E000320073905230974200009382C2EA73909B
:1021F00012346FB0F46073002030397101436EC641
:1022000019A0397141536AC866CA62CC5ECE19A062
:10221000397101535AD056D252D44ED64AD826DA02
:1022200022DC06DE33016140828241114AC026C2AF
:1022300022C406C68282B24D4101024D924C224C0C
:10224000B24B4101024B924A224AB2494101024932
:1022500092442244B240410182803D432A87637305
:10226000C3029377F700BDEFADE5937606FF3D8A95
:10227000BA960CC34CC30CC74CC74107E36BD7FEDF
:1022800011E28280B306C3408A0697020000969648
:102290006780A6002307B700A306B7002306B70090
:1022A000A305B7002305B700A304B7002304B700B4
:1022B000A303B7002303B700A302B7002302B700AC
:1022C000A301B7002301B700A300B7002300B700A4
:1022D000828093F5F50F93968500D58D9396050131
:1022E000D58D61B793962700970200009696868257
:1022F000E78086FA9680C1171D8F3E96E374C3F877
:10230000A5B73367B500FD530D8B79E7B7877F7F9E
:102310009387F7F710419441B372F6003363F600E8
:10232000BE92B3E262006397720C6318D606504106
:10233000D441B372F6003363F600BE92B3E262009A
:102340006398720A631BD60410459445B372F60075
:102350003363F600BE92B3E262006391720A631EB9
:10236000D6025045D445B372F6003363F600BE92F0
:10237000B3E26200639A72086311D602104994496D
:10238000B372F6003363F600BE92B3E26200639369
:1023900072085105D105E30FD6F61317060193977E
:1023A0000601631CF7001357060193D70601330596
:1023B000F7409375F50F91E982804183C18333051E
:1023C000F7409375F50F91E182801377F70F93F73C
:1023D000F70F3305F74082800346050083C60500EA
:1023E000050585056313D60065FA3305D64082805E
:1023F00011059105E312D6FE014582802105A10554
:10240000E31CD6FC014582803105B105E316D6FCFC
:10241000014582804105C105E310D6FC014582805B
:10242000B717004003C777051377E70FA38BE704BF
:10243000130700F8A38DE7043D47238CE704130737
:102440005003A38CE70403C7A7051377D70F238D89
:10245000E7048280B717004003C7E7040D894111E4
:102460001377C70F498F93068008F3B6068093F65B
:10247000860836C601000100930670052380D70444
:10248000930680FA2380D704010001002387E70424
:1024900023800704B247F3A7078001000100410130
:1024A0008280B717004003C7E7020D8941111377F7
:1024B000C70F498F93068008F3B6068093F6860807
:1024C00036C601000100930670052380D7049306E9
:1024D00080FA2380D704010001002387E7022380CC
:1024E0000704B247F3A70780010001004101828081
:1024F00041112A83014E930E407E130F0019930F52
:10250000400663E56E129308001913034006B37882
:102510001503854E0D4FA14F337365020D89133599
:10252000150063EFBE121308F6FF79467298420851
:10253000135808013307C70213D61700BE07329796
:102540006146B3F6C60213068070B386C60236979C
:10255000A166F58F42075D8FB716004083C7F6026C
:1025600093F70708A303F1000346710083C7F6023F
:1025700093F70708E394C7FE83477100B71600403E
:1025800093F7F70F6388071293078008F3B7078064
:1025900093F787083EC401000100B7170040930677
:1025A00070052380D704930680FA2380D7040100A6
:1025B000010023AA070383C6170393E60608A3882E
:1025C000D70223800704A247F3A707800100010078
:1025D0001166B71700407D16D45BC85F938547032B
:1025E000A98EF18EF5FA93068008F3B6068093F66D
:1025F000860836C601000100930670052380D704C3
:10260000930680FA2380D7040100010098C103C714
:10261000170313670704A388E70223800704B24760
:10262000F3A7078001000100410182807D13336818
:10263000E3039308E016630E08003368F30393087E
:10264000D016630808009378330093B81800938875
:10265000D81633081E01131E0801135E0E0155B56E
:102660006393E5030548638608000148630303009C
:102670002A8871087298FD15131E0801C205135EA1
:102680000E01C18179BD13F8150063F4BF0079080C
:10269000D5B713381800E5BF83C7F60293F70708CC
:1026A000A303F1000346710083C7F60293F70708FE
:1026B000E394C7FE8347710093F7F70FF1DFE9B5A5
:1026C00031714AD966CB06DF22DD26DB4ED752D5E3
:1026D00056D35AD15ECF62CD6AC96EC7AA8C02D8D2
:1026E000EF00901C2A8993078008F3B7078093F7BF
:1026F00087083EDA01000100B71700401307700594
:102700002380E704130780FA2380E7040100010017
:1027100003C7F7021377770FA387E70203C7F70210
:1027200013678700A387E70223800704D257F3A724
:102730000780010001000545AD33130780C1334711
:10274000E902116A93070AE893065002BD69930BE8
:10275000A004814A014B13048008930470057D1A7C
:10276000B347F9023307D7023EC0FD873ECC9387BB
:1027700009A69309803E3347F7023AC27D873AC4DF
:10278000334739038549B399990193D93940B30641
:10279000D702B30B7703B3C6F602B3CBFB0236C640
:1027A000FD8636C893D6FB4136CEB7460F009386DA
:1027B00006243349D9028566938606FAB3969601B4
:1027C000B389E902130760553309D9029306001053
:1027D000B389E9023349D902B3C9F9029316390022
:1027E00036CA37190040FD8636D0930D090493D7B9
:1027F000F9413ED2F336048093F6860836DC0100B8
:102800000100930770052380FD00930680FA238062
:10281000DD00010001008346390593F6860FA30908
:10282000D9048346390593E61600A309D904238009
:102830000D00E256F3A6068001000100130C80FA99
:10284000116DF336048093F6860836DE0100010030
:10285000930770052380FD0023808D010100010096
:1028600083463905216693E60602A309D9048356F7
:102870000905B3E6A6012318D90483560905D18EAC
:102880002318D90423800D00F256F3A60680010018
:1028900001008346390593F60602638A061803464B
:1028A0003905218A6DDE0818EF00100473360480A4
:1028B00013768608B2C20100010023809D002380A8
:1028C0008D0101000100B717004003C637051376DC
:1028D000F60DA389C70403C6370513660602A3894C
:1028E000C704835609052166B3E6A6012318D90457
:1028F00083560905D18E2318D90423800D009646EE
:10290000F3A60680010001008346390593F606020E
:102910006386061483463905A18AEDFE97F0FF1FF2
:10292000E7806077AA8636D497F0FF1FE780A0760D
:10293000A256E30AD5FE835609054255B3E6A60121
:102940002318D904C12783463905A18AEDDE035631
:1029500009058346290582473376CA00B306DA02A1
:1029600093D5F641B296B388F640E24733B8C60035
:102970002E983308F840A247B3B616013308D84062
:1029800063C70701631DF800924763FA1701C24746
:10299000634DF80E63950701B24763E8F80E894668
:1029A00063E7660FF2469315180013D3F8015E86AD
:1029B00013951800B365B30042D646D4EF604128A2
:1029C0003258050B137BFB0F634700016312083875
:1029D000A258638F083613081500B336A800B695C1
:1029E00013D6F5013298B336C800AE9613581800C6
:1029F000FE06B3E606017336048013768608B2C677
:102A00000100010023809D0023808D010100010051
:102A10000356C902B296C206C1822316D902238088
:102A20000D00B646F3A606800100010019BDF3367D
:102A3000048093F68608B6C00100010023809D0043
:102A400023808D01010001008346390593E60602CB
:102A5000A309D90423800D00864605BDF336048002
:102A600093F68608B6C40100010023809D002380F0
:102A70008D01010001008346390593E60602A30992
:102A8000D90423800D00A646A5BDE30D0BF0F33657
:102A9000048093F68608B6C801000100930680FA08
:102AA00023809D002380DD0001000100834639055D
:102AB00093F5FC0F93F6860FA309D90483463905D5
:102AC000CD8EA309D90423800D00C646F3A6068047
:102AD00001000100130580FA034639059306390504
:102AE0001D8A631496297336048013768608B2CC47
:102AF00001000100130680FA23809D002380CD0091
:102B00000100010003C606001376F60D2380C600FF
:102B100003C60600136606022380C6008356090515
:102B20001166D18E2318D904835609052166D18EEA
:102B30002318D90423800D00E646F3A60680010081
:102B40000100130680FA8346390593F6060263886E
:102B5000062483463905130C3905A18AFDDA0818C5
:102B60006123F336048093F68608B6D00100010095
:102B7000930680FA23809D002380DD000100010080
:102B800083460C00116693F6F60D2300DC008346A5
:102B90000C0093E606022300DC0083560905D18E63
:102BA0002318D904835609052166D18E2318D90428
:102BB00023800D008656F3A606800100010013064F
:102BC00080FA8346390593F606026385062083461C
:102BD0003905A18AEDFE97F0FF1FE780C04B2A8CD4
:102BE00097F0FF1FE780204BE30C85FF8356090514
:102BF00011664255D18E2318D904292383463905FD
:102C000013063905A18AFDDAF336048093F68608A7
:102C1000B6D401000100930680FA23809D00238032
:102C2000DD00010001008346060093F6F60D230047
:102C3000D60023800D00A656F3A6068001000100F1
:102C40008356090503462905D247B376DA003306D1
:102C5000CA021305800C9355F6413696330DF640A3
:102C60008257333CD6002E9C3336A601330CFC40F1
:102C7000330CCC403308850392564E86B335A503FA
:102C80003305A503C295EF50B17B63468001631EF7
:102C90000C16630C0D16130615003335A6002E9581
:102CA0009356F5013696B335D600AA959396F5015D
:102CB00005828585D18E6346B000639D051A638BBE
:102CC000061A0356C90215823305D6003336C500ED
:102CD000B2956348B000639105241306F00F637D3D
:102CE000A622894663F3561593078008F3B7078039
:102CF00093F78708BED601000100371700409307FD
:102D000070052300F704930780FA2300F7040100FD
:102D100001008356C70289678117D58FC207C18317
:102D20002316F70223000704B657F3A70780010014
:102D30000100FA506A54DA544A59BA592A5A9A5A2E
:102D40000A5BFA4B6A4CDA4C4A4DBA4D29618280D3
:102D50001308F5FF3335A800FD152E951356F50120
:102D60003298B336C800AA9651B1F336048093F670
:102D70008608B6CA0100010023809D002380AD00B3
:102D80000100010083463905CD8EA309D9042380B3
:102D90000D00D646F3A606800100010035BBF336D0
:102DA000048093F68608B6CE0100010023809D00C2
:102DB0002380CD00010001008346390593E6060219
:102DC000A309D90423800D00F646F3A6068001006E
:102DD000010095BBF336048093F68608B6D2010055
:102DE000010023809D002380CD0001000100834667
:102DF000390593E60602A309D90423800D009656EF
:102E0000F3A60680010001006DBB9306F5FF33B504
:102E1000A600FD152E959355F501AE96B3B5B600F7
:102E2000AA951396F501858269B5F336048093F669
:102E30008608B6D801000100930680FA23809D0021
:102E40002380DD00010001008356C90205660116DA
:102E500093F6F60FD18EC206C1822316D9022380C3
:102E60000D00C656F3A6068001000100850A93FAFC
:102E7000FA0F49B233E6B60045C20356C90233051C
:102E8000D0403338A000B305B040B385054115826A
:102E90006345B000D1E16371A608894663F0560529
:102EA00093078008F3B7078093F78708BEDA01001D
:102EB0000100B7170040130770052380E7041307CC
:102EC00080FA2380E7040100010003D7C7027D8B4D
:102ED0002396E70223800704D65781BDF33604808A
:102EE00093F68608B6DC01000100930680FA238081
:102EF0009D002380DD00010001008356C9020566A4
:102F0000011693F6F60FD18EC206C1822316D9029E
:102F100023800D00E656B9B793078008F3B7078002
:102F200093F78708BEDE01000100371700409307C2
:102F300070052300F704930780FA2300F7040100CB
:102F400001000356C70293975600B297C207C18388
:102F50002316F70223000704F657C1BB914763EE1F
:102F6000B702178701001307679B8A05BA959C4132
:102F7000BA978287B717004003A7470B1345F5FFA1
:102F8000698F23AAE70A03A7070B698F23A8E70A1B
:102F900003A7070A798D23A0A70A8280B7170040EC
:102FA00083A6470B1347F5FFF98E23AAD70A83A6FA
:102FB000070B558D23A8A70A83A6070A758F23A0A0
:102FC000E70A8280B717004003A7470B498F23AA5F
:102FD000E70A03A7070B1345F5FF45BFB7170040E6
:102FE00083A6470B1347F5FF758F23AAE70A03A7AC
:102FF000070A598D4DB7B717004003A7470B498FF4
:10300000EDB7914763EEB7021787010013074792A8
:103010008A05BA959C41BA978287B717004003A7E3
:10302000470D1345F5FF698F23AAE70C03A7070D8A
:10303000698F23A8E70C03A7070C798D23A0A70CA1
:103040008280B717004083A6470D1347F5FFF98E1E
:1030500023AAD70C83A6070D558D23A8A70C83A6FA
:10306000070C758F23A0E70C8280B717004003A7D9
:10307000470D498F23AAE70C03A7070D1345F5FF5A
:1030800045BFB717004083A6470D1347F5FF758F5F
:1030900023AAE70C03A7070C598D4DB7B7170040BB
:1030A00003A7470D498FEDB7B71700408847420582
:1030B00041819377050491EB9377F5013755E8014A
:1030C000130505803345F50282809377050C1307BD
:1030D00000046397E7009377F50137459C1CCDB753
:1030E0002165130505D0828037E700E01C43544377
:1030F000A183E206D58F1CC1FD572320F718232298
:10310000F718828013178500B7E700E023A0E710C7
:10311000618123A2A7108280B7F700E08847CC47DF
:103120008280814737370040A14663C4C70032859B
:1031300082800345B740E38EA6FE3385F500034544
:10314000050085072304A740CDB797070020938784
:10315000E7659C43173700201307C7313E95636E20
:10316000E500173700201307E7496368A700170732
:103170000020232DA7623E858280FD57EDBF4111BF
:1031800022C406C62A840D372947B307E502B24098
:103190008D83B3D7870222449507B3D7E702373729
:1031A0000040C207C1832316F70041018280716588
:1031B00041111305052006C6D937B737004013075C
:1031C00070F82381E7000D47A381E700130700048F
:1031D000A380E70005472387E700B24041018280D2
:1031E00037370040834727001A0593F7F703C98F45
:1031F00093F7F70F2301F7008280B737004003C72A
:10320000170019C9D98DA380B70003C7070013673A
:1032100087002380E700828093C5F5FFF98DA380A6
:10322000B7008280B73700402147B736004091E1B0
:10323000828003C6B700E30CC7FE05050346F5FF11
:10324000FD15C2052384C600C181D5B7411122C432
:1032500006C62A84913D2947B307E502B2408D8313
:10326000B3D7870222449507B3D7E7023737004028
:10327000C207C1832316F740410182807165411165
:103280001305052006C6D937B7370040130770F875
:103290002381E7400D47A381E74013070004A38083
:1032A000E74005472387E740B24041018280CC4197
:1032B000411106C6328503C6150083C505002206E6
:1032C0004D8E42068D654186138875A263080611EE
:1032D000634BC804138845A2630C060B634AC800FD
:1032E000938535A2630FB60623900600294669A888
:1032F000138855A26301060D938565A2E316B6FEF9
:103300008D451D4663E2E5081146198E63F3C7003B
:103310003E86B7E704002390C600FC47979501005E
:1033200093854525B9A8138895A2630F060F634AB4
:10333000060D1388A5A2630C0611938505A5E31558
:10334000B6FA99451D4663E1E504198E63F3C7009B
:103350003E86B7E704002390C600FC479385818032
:103360000DA09D451D4663E1E5022146198E63F3DC
:10337000C7003E86B7E70400FC472390C60093854C
:103380000184BA9582970146B2403285410182801C
:10339000AD451D46E3EAE5FE3146198E63F3C700ED
:1033A0003E86B7E704002390C600FC4797750100EE
:1033B0009385055BF9B7B1451D46E3E7E5FC354666
:1033C000198E63F3C7003E86B7E704002390C6005A
:1033D000FC47977501009385A55965B78D451D4636
:1033E000E3E4E5FA1146198E63F3C7003E86B7E7BA
:1033F00004002390C600FC4797950100938545186B
:1034000049B78D451D46E3E1E5F81146198E63F392
:10341000C7003E86B7E704002390C600FC47979597
:1034200001009385A517B1BFA5451D46E3EEE5F460
:103430002946198E63F3C7003E86B7E70400239040
:10344000C600FC47977501009385C5501DBFB54563
:103450001D46E3EBE5F23946198E63F3C7003E865D
:10346000B7E704002390C600FC47977501009385D9
:10347000654D01BFB7E7040003A3071397060020BB
:10348000938646D54146A54517050020130585CBF3
:1034900002832D4559EF03C5050009476317E50869
:1034A00003A84500411106C60347180032850346AC
:1034B000080022074168518F930828FE630817030C
:1034C00063E9E80005186303070523900600294512
:1034D0001DA8130648FE630BC7021518E31707FF64
:1034E00015463E87637BF602154705A83E8691C3C5
:1034F0000546B7E70400FC472390C6004206CC45CA
:10350000418282970145B240410182801306700FCB
:103510003E876374F6001307700FB7E7040023902B
:10352000E600FC4713160701D9BF239006000545A6
:1035300082808280416779176302E504411122C4C9
:1035400006C685472A84639DF500B7E704002285F7
:103550002244B24003A387139385C18441010283AF
:1035600089476399F500B7E7040083A7070B8545F2
:10357000829761DDB240224441018280828079716C
:1035800022D452CC2E842A8A9775010093858540D7
:10359000177501001305C54106D63AC626D24AD092
:1035A000B68432894ECEEF50F134A68517750100EE
:1035B00013050541EF5011342945EF50B1378347CA
:1035C000840093F70702F1E3834904008947054526
:1035D00032476394F908544083C7160083C6060037
:1035E000A207D58FC166138616FE638CC7028D169F
:1035F000638DD7068D66938626902945639FD704F1
:10360000B7E70400A285225403A34714B250F2493D
:10361000A6864A86925402595285624A8547456178
:1036200002832D451DEB9307700F354563E7970225
:10363000B7E70400FC4748441306700FCA85829719
:103640008149938781859C43014581CB9C4391C7E8
:103650004E852686CA8582970145B25022549254DF
:103660000259F249624A456182802D457DF79307F0
:10367000700F3545E3E397FEB7E70400FC47484485
:103680001306700FCA8582976DBF2145F9B74111A6
:1036900022C437E404008327841326C2AA84416528
:1036A00006C69385C1847D1582978327C40A1705B2
:1036B0000000130565E88588829795C003230413ED
:1036C0002244B240924497060020938666C2414647
:1036D000C545170500201305A5B041010283B2407E
:1036E0002244924401454101828009C523ACA18452
:1036F000014582804545828011476360A70A97761D
:1037000001009386E6270A0536951841411106C641
:103710003697AE87B28502871307700F6145639BAA
:10372000E700B7E70400FC471306700F1385C18B51
:1037300082970145B2404101828005476145E39B84
:10374000E7FEB7E70400FC47054613858184CDB743
:103750001307700F6145E39FE7FCB7E70400FC47E0
:103760001306700F1385419BE1B71307700F614576
:10377000E392E7FCB7E70400FC471306700F1385DC
:10378000C1AA7DB715476145E396E7FAB7E704009C
:10379000FC4715461385018561BF094582804111AB
:1037A00026C2B7E4040083A7C41322C44AC006C6D5
:1037B0002E849385C1842A898297058905C5970738
:1037C00000209387E7A183D7A70BA28503A3440D0D
:1037D0002310F4002244B24092444A850249014633
:1037E00041010283B24022449244024949454101C9
:1037F000828011456FE0DFEC411193962500AA8588
:103800002D4506C697F0FF1FE780A01FB240014577
:1038100041018280011122CC06CE3714004026CA15
:103820004AC84EC652C483447405034AB40583494A
:10383000840503499405EFE0BFBE8347A40593F4D4
:10384000F40F137AFA0F93E71700230DF40493F99A
:10385000F90F1379F90FB717004003C7A705058BB8
:103860006DFF03D5C705A38D4705238C3705A38CB2
:103870002705A38B9704F2406244D2444249B249DF
:10388000224A0561828041119397050122C406C630
:1038900026C2C1872E8463D00702B7E40400FC541B
:1038A000829719C1BC5482972165218DB240224470
:1038B00092444101828093F7150013C51500FDF76E
:1038C0009397250163D30702B7E4040083A7C41EBE
:1038D00082970537BC4C37F60200130606E089656F
:1038E00003C5018682970965C9B7939715010145FC
:1038F000E3DE07FA1775010013054513EF50D113E6
:10390000B7E70400BC4F13060064916503C5018648
:103910008297116559BF2D71232A9110FD74E98C8E
:10392000232C811023282111232631112A84AE89CA
:103930003289930600100A86A6852D45232E111084
:1039400097F0FF1FE780E00B13154401B7E7040071
:10395000FC4751810A0513962900CA850A9582976A
:10396000A68585660146254597F0FF1FE78060091B
:103970000A86A68593060010294597F0FF1FE78069
:1039800040088320C111032481118324411103299C
:1039900001118329C11015618280B7F7070003C7A1
:1039A0000701411106C622C426C24AC0A547631AB0
:1039B000F7009537B2402244924402490145410143
:1039C000828013942500AA843289A286AA850146A2
:1039D000254597F0FF1FE780C002A2864A86A6858C
:1039E000294597F0FF1FE780C001E9B71D71A2CC00
:1039F00037E404005C5C485886CE49469775010060
:103A0000938545FE829701E9177501001305C5FEF0
:103A1000EF50910201A0B7F600E0795798CAFD5720
:103A2000DCCA0567B7E700E023A0E7101306F00241
:103A300090C223A0E71801000100370700201847B3
:103A400013060004814523AEE1844157A38AE74071
:103A50003C4408088297971700209387A7E83EC840
:103A6000856713870740231AE1001D673ACC3707A3
:103A70000105130707109387B7D33ACE2312F1023B
:103A80001307B00F97F7FFFF938747692310E102F1
:103A90003ED8094797070000938707D82301E10222
:103AA0003EDC17070000130767D5970700009387D0
:103AB00087D4B7F50700BAC23EDE17070000130728
:103AC00007EE970700009387C71B81463000E1058A
:103AD0001945BAC43EDA97F0FF1FE78080F2180854
:103AE0008147994630003E96034606008507050744
:103AF000A30BC700E398D7FEC24791C70357410104
:103B000085676373F70001A0B7E7040083A7470A3E
:103B100008088297AA8501C917750100130505EFEA
:103B2000EF50415D01A0F64066442561828041115D
:103B300026C2B7E4040083A7040806C622C41705FA
:103B40000000130585D48297138401862300A40006
:103B50008520E12A03450400224403A38405B240E2
:103B60009244130600328965410102834111930793
:103B70008008F3B7078093F787083EC6010001006D
:103B8000B7170040130770052380E704130780FA76
:103B90002380E70401000100C8DB23800704B2474B
:103BA000F3A707800100010023A201864101828062
:103BB000797106D622D413078008F337078093F76C
:103BC00087083EC201000100B71700409305700549
:103BD0002380B704130680FA2380C7040100010084
:103BE00083C6F70293F6A60FA387D70223800704A4
:103BF0009246F3A606800100010073370780137711
:103C000087083AC4010001002380B7042380C70459
:103C10000100010003C7F70213672700A387E7022B
:103C200023800704A247F3A7078001000100054590
:103C3000EFE03F877D3E0147814681470546854548
:103C40001305407EEFE0DF8A37E404003C4468005F
:103C5000514681458297B707C0A83EC8B787E80399
:103C6000938707D03ECA97F7FF1F938707C53EC6C5
:103C70007C5868008297B2502254456182800111BD
:103C800022CC06CE930730031304D5FC63E7A700CC
:103C90003704C0A81304D4FC2A946800EFF0CFC402
:103CA00097E0FF1FE780203FB307A4406376A4009E
:103CB000B707C0A8A297898F3747F6A681171307C1
:103CC00007C6637AF7003245EFF0CFC30945F240EB
:103CD0006244056182802285513D3245EFF08FC2FA
:103CE000373700408347574093F707048DCF9387BA
:103CF00041869C430D45E1FF1165690597E0FF1F73
:103D0000E78080510545EFE0EFF497E0FF1FE78083
:103D100080382AC497E0FF1FE780E037A247E30B13
:103D2000F5FE01456DB7010075BF4111130780080D
:103D3000F337078093F787083EC401000100B717E7
:103D40000040930570052380B704130680FA238092
:103D5000C7040100010083C6E70093E686002387BD
:103D6000D70023800704A246F3A6068001000100C5
:103D700073370780137787083AC601000100238054
:103D8000B7042380C7040100010003C717031367AA
:103D90000702A388E70223800704B247F3A707803E
:103DA00001000100B7E700E03707001023A0E7108B
:103DB000410182804111977501009385E5361775A1
:103DC00001001305E5BE06C6EF50C13217750100AC
:103DD00013050550EF500132B240294541016F50A3
:103DE00061354111977501009385453517750100BF
:103DF000130505BC06C6EF50E12F1775010013052A
:103E0000E54BEF50212FB240294541016F508132DF
:103E1000411122C406C6834705002A849DC39775B5
:103E200001009385653717750100130565B8EF50DC
:103E3000612C4C40177501001305C55DEF50812BB7
:103E40001DA058411DE7977501009385E53417754E
:103E500001001305E5B5EF50E129177501001305C1
:103E6000E55CEF5021292244B240294541016F50C1
:103E7000612CA1679386D7036311D7029775010060
:103E80009385853117750100130585B2EF508126A2
:103E9000177501001305855AE9B7ED0797750100FD
:103EA0009385852F17750100130585B06319F700F9
:103EB000EF50412417750100130585595DB7EF5088
:103EC00061234C40177501001305855A85BF4111C8
:103ED000977501009385C52717750100130545AD3A
:103EE00006C6EF502121B240294541016F5081247F
:103EF000797122D426D24AD02E842A898145B2846F
:103F00004800714606D6EFE04FB597F7FF1F93873D
:103F1000A75DDC4783D70700231421012313F10099
:103F2000EF20206C9547A305F1009307401F3EC684
:103F3000FD572305A100230AF100EF20007C26860F
:103F4000A2854800EF20406CB2502254925402598E
:103F5000456182802399018823880188B7E704009E
:103F6000BC47411106C6414681451715002013057F
:103F7000A5958297EF109055EF1050340145EF2032
:103F8000107E03C7417A9307F00A631BF70093077B
:103F9000F00889451385417A2392F17AEF300027A2
:103FA000EF30003981453705040023A401882392AE
:103FB000018823830188239F0186239E0186239104
:103FC000018823960188EF2000250145EF30E02C81
:103FD000977501009385451A177501001305459DD6
:103FE000EF504111177501001305C54EEF508110B8
:103FF000B240294541016F50E113411122C406C668
:1040000026C293F715002E846389070C814617F6A4
:10401000FF1F1306E64A854503D58187EF8040756B
:1040200005C5977501009385E51517750100130502
:104030002598EF50210C17750100130565B7EF5057
:10404000610B2945EF50010F97750100938585138A
:10405000177501001305C595EF50C10917750100CB
:10406000130545B6EF5001092945EF50A10C17F58E
:10407000FF1F130565475C4505472390E700EFF0F8
:104080008005977501009385E50F177501001305ED
:104090002592EF502106177501001305E5B3EF5087
:1040A00061052945EF500109930710F82382F17A41
:1040B00083D74187A382F17A1385417AA183914501
:1040C0002383F17AA383017AEF304014134514005F
:1040D000B240224492444101828093F72500D1C32B
:1040E00003D7418825CF9386818894429777010032
:1040F0009387474003C66188814517050020130553
:10410000A57CEF402074AA8431C99775010093857E
:10411000250E177501001305A589EF40B17DA68511
:10412000177501001305C5ACEF40D17C2945EF5050
:10413000610023920188930710F82382F17A83D7D4
:104140004187A382F17AA1832383F17A91458D4738
:104150001385417AA383F17AEF30400B1345240095
:1041600085BF93F74500A1CF97750100938545085A
:10417000177501001305C583EF40D177177501004E
:104180001305C5A8EF4011772945EF40B17A930791
:1041900020F82382F17A83D7E187A382F17AA18381
:1041A0002383F17A8547A383F17AEF2000551385A5
:1041B000417A9145EF3080051345440011BF93F7D4
:1041C00085009DCB977501009385850217650100D9
:1041D0001305057EEF40117217750100130545A404
:1041E000EF4051712945EF40F17423920188EF406F
:1041F000407213458400E9BD93F70501A1CF8545C1
:1042000003D5E187EF00513C97750100938545FE8A
:10421000176501001305C579EF40D16D17750100D1
:10422000130545A1EF40116D2945EF40B17093078B
:1042300030F82382F17A83D7E187A382F17A13855C
:10424000417AA1838D452383F17AEF20307C134599
:104250000401BDBD93F70502B1CF977501009385A9
:1042600025F9176501001305A574EF40B1681775AE
:1042700001001305659EEF40F1672945EF40916B02
:10428000930740F82382F17A83D7C187A382F17A1A
:10429000A1832383F17A8547A383F17A239E018644
:1042A000EF20A0451385417A9145EF2030761345E4
:1042B000040239BD93F70504D9CF977501009385A2
:1042C00025F3176501001305A56EEF40B162177560
:1042D00001001305E599EF40F1612945EF40916533
:1042E00083C7417A1307700A6384E7041307800ABF
:1042F0006380E7061307600A6395E702930760F897
:104300002382F17A83D72188A382F17AA183238340
:10431000F17A8547A387F17AB1451385417AEF2079
:10432000F06EEF20803D13450404239101884DB3C6
:10433000930770F82382F17A83D72188A382F17AD8
:10434000A1832383F17A8547A384F17A9945F1B754
:10435000930780F8C5B793F705080145E38A07D6A8
:10436000977501009385C5E817650100130545643D
:10437000EF4051581775010013050591EF40915713
:104380002945EF40315B9307A0F82382F17A83D768
:10439000C188A382F17AA1832383F17A8547A3831D
:1043A000F17A23960188EF2040351385417A9145B3
:1043B000EF20D0651345040821BB411122C4977535
:1043C00001009385A5DE2A84176501001305455E6B
:1043D00006C6EF4031524C40177501001305050128
:1043E000EF4051512945EF40F15403470400930732
:1043F000F00F6319F70297750100938525DB1765A8
:1044000001001305E55AEF40F14E4C4017750100CD
:104410001305C5FEEF40114E2244B240294541012B
:104420006F405151B24022444101828085CD4111FB
:1044300022C4176501001305A5572E849775010046
:104440009385C5D106C6EF40F14AA28517750100D4
:1044500013050506EF40114A2244B24029454101A7
:104460006F40514D8280411122C426C22E84AA84FD
:1044700097750100938545CF1765010013054553D6
:1044800006C6EF4031471775010013052503EF40BD
:1044900071462945EF40114A977501009385C5CCB7
:1044A000239C918617650100130585508544239A46
:1044B0008186239B918623998188EF40B14383D5E0
:1044C0002189177501001305E5FFEF40B142294529
:1044D000EF40514623889188EF10405E2285EF20FF
:1044E00010280545EF20705B97F7FF1F9387C7FFE4
:1044F000DC4703D70700C167FD176310F7022244AA
:10450000B7E70400B240924403A3870503C5818640
:104510001306000A854541010283B24022449244B9
:1045200041018280011122CC37E404005C5C06CE9C
:1045300026CA3546977501009385C5DA17750100BF
:1045400013054569829701E9176501001305C54AFE
:10455000EF40914E01A097F7FF1F9387675F3EC41E
:10456000B7F507008567938707C081461386C18624
:10457000E10519453EC697E0FF1FE78080487C446F
:1045800019469385C186170500201305252D8297AE
:1045900034001386C186977501009385251F177512
:1045A000010013052520EF406002AA8415C9977504
:1045B00001009385E5C2176501001305653FEF40D3
:1045C0007133A685177501001305C5D2EF409132EE
:1045D0002945EF403136F2406244D2440561828081
:1045E000EFA04019177501001305C5C7EF30A01DD6
:1045F000EF708007EF00112617F5FF1F130585EBFD
:10460000EF00F112177501001305C5C6EF00512622
:10461000AA84EF304078EFC0604BEF20B145EF4007
:104620007014EF309057EFE0502897750100938594
:1046300025BB176501001305A53789C8EF40912BED
:10464000A68517750100130525CD49B7EF40912ABE
:1046500017750100130585CEEF40D1292945EF409C
:10466000712DEFE0F00AEFB02035630D050C8545A4
:1046700037050400EF10303A97750100938545B671
:10468000176501001305C532EF40D12617750100EB
:10469000130545CCEF4011262945EF40B12997F786
:1046A000FF1F9387A7D483D707002399F1888547F5
:1046B0002388F188EF10405CEF10404003D521893A
:1046C000EF20F00983C7F188B9EFA3030100832726
:1046D000441713067100854513055030829797756E
:1046E00001009385E5AF176501001305652CEF40C8
:1046F000712017750100130525C8EF40B11F29452A
:10470000EF40512397750100938585AD1765010032
:104710001305052AEF40111E177501001305C5CBBF
:10472000EF40511D75B597750100938565AB176511
:1047300001001305E527EF40F11B17750100130574
:1047400025C765BF97750100938585A91765010089
:1047500013050526EF40111A17750100130585D7BB
:10476000EF4051192945EF40F11C0145EF20F0328F
:1047700051BF411122C437E404008327041A06C63E
:104780008297EF2090068327040817050000130581
:10479000058782972384A18617F5FF1F1305C5D4CB
:1047A000EF2000212244B2404101ADBB411122C49F
:1047B00091462A84170600201306C6079D652D45DD
:1047C00006C697E0FF1FE780C023B7F7070003C7BF
:1047D0000701A5476313F70001A0930600100146E7
:1047E0009D65254597E0FF1FE780A02197070020E2
:1047F000238287042244B240914617060020130604
:1048000066039D652945410117E3FF1F6700631F8C
:10481000B7E704001171FC47CED79389417AA2DD36
:10482000CAD986DFA6DB2E8432892E86AA854E85DC
:10483000829783C70900130780029387E70793F7DE
:10484000F70F636CF772176701001307671E8A077B
:10485000BA979C43BA9782878D47977501009385D5
:10486000659A176501001305A514630BF400EF406A
:104870007108176501001305A557EF40B107CDA2D8
:10488000EF4051071765010013050558EF409106E9
:104890002945EF40310A930720F811469385417A64
:1048A0004A852382F17AA383017AEFF06FE42A84A8
:1048B0000DC5977501009385E594176501001305F3
:1048C000250FEF403103A2851765010013058557B9
:1048D000EF4051022945EF40F1059775010093859E
:1048E0006592176501001305A50CEF40B10017652F
:1048F000010013056556EF40E17F2945EF40910324
:104900004165930730FA05469385417A7D152382E8
:10491000F17AEFF0EFDD2A840DC5977501009385DC
:10492000658E176501001305A508EF40A17CA285DF
:104930001765010013050551EF40C17B2945EF4084
:10494000617FB7E70400BC4F0566130606C8A145A2
:1049500003C581868297FE506E54DE544E59BE596F
:104960001161828091476301F4029775010093857C
:104970006589176501001305A503EF40A177176549
:1049800001001305A550D5BDB7E70400FC4F9145C4
:1049900003C581868297977501009385A586176563
:1049A00001001305E500EF40E174176501001305F0
:1049B000A54FEF4021742945EF40C177EF10F05328
:1049C0009145C1A285476301F40297750100938563
:1049D0006583176501001305A5FDEF40A1711765FB
:1049E00001001305E54D51BD239F2187B7E7040062
:1049F0000566BC4F130606C8C14599BF8D476301C4
:104A0000F402976501009385E57F176501001305A2
:104A100025FAEF40216E176501001305254CB1BD45
:104A2000930740F811469385417A4A852382F17AAB
:104A3000A383017AEFF0CFCB2A84E30E05F09765CC
:104A400001009385257C17650100130565F6EF408D
:104A5000616AA285176501001305C53EEF408169B3
:104A60002945EF40216DC5BD9147E31CF4F8B7E738
:104A70000400FC4F9305000203C581868297976569
:104A800001009385257817650100130565F2EF4055
:104A90006166176501001305E54521BF894763E19C
:104AA0008702976501009385E57517650100130579
:104AB00025F0EF402164176501001305E54475BB3F
:104AC00083C4617A83C7517A9765010093858573A2
:104AD000A204176501001305A5EDDD8CEF4081618F
:104AE000A2851765010013056543EF40A160C2046C
:104AF0002945EF402164C1849305D4FF93960401B6
:104B0000C1824A8693F5F50F1385717AEF102074F0
:104B1000E35390E4930750F82382F17A83C7390076
:104B200022869385417A85074A85A383F17AEFF03F
:104B30002FBC2A84E30105E2976501009385856C0B
:104B4000176501001305C5E6EF40C15AA285177528
:104B500001001305E59419B7894763E1870297655A
:104B600001009385256A17650100130565E4EF4090
:104B70006158176501001305253C01B3EF10F037AC
:104B8000A2851385417AEF206068F1B38D476301F8
:104B9000F402976501009385E5661765010013052A
:104BA00025E1EF402155176501001305A53AF1B144
:104BB000B76602000146B7750200054597E0FF1F82
:104BC000E78020E4930760F82382F17AA383017AD7
:104BD0009307002623A4F17AE5779387072123968C
:104BE000F17A3146A387A17A9385417A4A85238752
:104BF000017AEFF0EFAF2A84E30F05D49765010047
:104C00009385456017650100130585DAEF40814EF5
:104C1000A285176501001305653589B5B1476301A4
:104C2000F402976501009385E55D176501001305A2
:104C300025D8EF40214C176501001305E53435B93F
:104C4000B7E70400FC4F9305000403C581868297F3
:104C5000EF10B02AB14535B7914763E187029765F8
:104C600001009385255A17650100130565D4EF40AF
:104C70006148176501001305E53201B183C4817AEB
:104C800083C7717AA204DD8C8E04B77702006D149D
:104C9000BE942286A685176501001305E531EF4015
:104CA0006145B7E70400FC4722869385917A280086
:104CB000829793160401C1823000A685094597E0CA
:104CC000FF1FE78000D42A8419C51765010013056A
:104CD0006530EF406156930770F819469385417A25
:104CE0004A852382F17AA384817AEFF06FA02A8427
:104CF000E30305C6976501009385C550176501005C
:104D0000130505CBEF40013FA28517650100130590
:104D1000652DA9B399476301F41097650100938548
:104D2000654E176501001305A5C8EF40A13C176546
:104D300001001305A52C91B6914763E187029765A1
:104D400001009385254C17650100130565C6EF40EA
:104D5000613A176501001305E52B05B683C4817A16
:104D600083C7717AA204DD8C8E04B77702006D14BC
:104D7000BE942286A685176501001305E52AEF403B
:104D80006137B7E70400FC4722869385917A2800B3
:104D9000829793160401C1823000A6850D4597E0E5
:104DA000FF1FE78000C62A8419C517650100130597
:104DB0006529EF406148930780F819469385417A49
:104DC0004A852382F17AA384817AEFF06F922A8454
:104DD000E30305B8976501009385C5421765010097
:104DE000130505BDEF400131A285176501001305CC
:104DF000A526ADB199476301F4029765010093853B
:104E00006540176501001305A5BAEF40A12E17658F
:104E100001001305E52595B4B7E70400FC4F9305A1
:104E2000000403C581868297EF10300D994591BB30
:104E30008D476301F402976501009385A53C1765D2
:104E400001001305E5B6EF40E12A176501001305DF
:104E5000A52325B41765010013050524EF40C13DC6
:104E60001305C01297E0FF1FE780C09D0145EFE0EA
:104E7000AFA70D45EFF09F93294597E0FF1FE7800F
:104E8000609C97E0FF1FE780808DF1B49947630134
:104E9000F402976501009385E53617650100130557
:104EA00025B1EF402125176501001305A51FF1B2BB
:104EB00003C7917A83C7817A22075D8F9166BA967C
:104EC000C2061166C1821306F6EF8D476363D602F0
:104ED00097E7FF1F938747619C4B03C6717A9386C0
:104EE000C70039C603D607004DCA8907E39CD7FE21
:104EF00089471307A0F811469385417A4A85238292
:104F0000E17AA383F17AEFE0BFFE2A84E30505A4EA
:104F1000976501009385052F17650100130545A9C5
:104F2000EF40411DA285176501001305E5183DB648
:104F300003D607006300E60A8907E39BF6FE8D4768
:104F40004DBF91476302F402976501009385852B5D
:104F5000176501001305C5A5EF40C11917650100CC
:104F6000130505176FF07F91B7E70400FC4F930519
:104F7000000803C58186829791B4976501009385E7
:104F80006528176501001305A5A2EF40A116176556
:104F90000100130565156FF05F8E2390E70017E59C
:104FA000FF1F13056554EFE0A0149765010093857A
:104FB0006525176501001305A59FEF40A11317652F
:104FC000010013056513EF40E1122945EF408116FA
:104FD000814705B72390070017E5FF1F1305C5504C
:104FE000EFE00011976501009385C5211765010069
:104FF0001305059CEF4001101765010013054511CD
:10500000D9B7411122C406C6834705002A849DC32F
:10501000976501009385C51A176501001305459929
:10502000EF40410D4C40176501001305A54DEF40C1
:10503000610C65A05841B707CF009387777D631156
:10504000F706976501009385A517176501001305FD
:105050002596EF40210A1C448356E4008355C40082
:1050600003C60700176501001305454BEF40810893
:105070002945EF40210C0357E40083D721896307BA
:10508000F7008355C4000844EFE0CF990356E400CD
:105090008355C40008442244B24041016FF04FF7E9
:1050A000B707CC009387777D631FF70297650100F0
:1050B00093850511176501001305858FEF40810366
:1050C0001C448356E4008355C40003C607001765DB
:1050D00001001305A544EF40E1012244B2402945F7
:1050E00041016F402105B707CE009387777D6302AA
:1050F000F702976501009385A50C1765010013055C
:10510000258BEF30317F4C40176501001305453684
:1051100039BFB2402244410182805171CAD137E97E
:1051200004008327C904A2D52E8686D7A6D32E8451
:10513000AA851385417A829783C7417A1307700A3B
:10514000638BE70C636CF7001307600A6382E70464
:10515000BE502E549E540E596D6182801307800AF2
:105160006380E7121307900AE394E7FE8D47630913
:10517000F416976501009385A50A176501001305CC
:105180002583EF303177176501001305A59F15A022
:105190008D476306F40297650100938565081765DE
:1051A00001001305E580EF30F17417650100130568
:1051B000A596EF3031742945EF30D17751BF85473F
:1051C00017650100130505972380F188EF40C1069C
:1051D000B7750200B76602000146054597E0FF1F5C
:1051E000E7802082930760F82382F17AA383017A13
:1051F0009307002623A4F17AE57793870721239666
:10520000F17AB1452387017AA387A17A1385417A80
:10521000EF10D07F35BF914763E1870297650100AA
:10522000938505001755010013058578EF30916CC3
:105230001765010013050592ADBF83C4817A83C74A
:10524000717AA204DD8C8327C9046D1422869385AC
:10525000917A280082978E0493160401B775020094
:10526000C1823000A695094597D0FF1FE78060797D
:10527000930770F82382F17A9945A384A17A79B7CC
:10528000914763E1870297650100938565F917559A
:1052900001001305E571EF30F16517650100130595
:1052A000E58C01BF83C4817A83C7717AA204DD8C47
:1052B0008327C9046D1422869385917A28008297EA
:1052C0008E0493160401B7750200C1823000A695C2
:1052D0000D4597D0FF1FE780C072930780F859BF34
:1052E000176501001305458BEF3011751305C012CA
:1052F00097D0FF1FE78000550145EFD0FFDE0D4539
:10530000EFF0CFCA294597D0FF1FE780A05397D071
:10531000FF1FE780C0442DBDB7E704004111FC47E3
:1053200026C29384417A2E8606C622C44AC02E84A1
:105330002A89AA852685829797650100938505F0BD
:10534000175501001305C566EF30D15A83C5417A60
:10535000176501001305C594EF30D1592945EF3089
:10536000715D83C7040041479387070693F7F70FE2
:105370006363F746175701001307C7758A07BA9783
:105380009C43BA9782879D476303F40297650100A7
:105390009385C5EA1755010013058561EF309155D6
:1053A0001765010013054590EF30D15455AA83C706
:1053B000517AADC783D7817A03D7617AC207D98F73
:1053C00023A4F18883C7640097650100938505E7EE
:1053D000175501001305C55D2383F188EF30915106
:1053E000938781888C4303C6618817650100130584
:1053F000658DEF3031502945EF30D153A382017ACA
:105400002244B24092440249930700F82382F17A81
:105410009D451385417A41016F10505FEF30005B6D
:105420002393A17A935705012A842384F17A935711
:1054300085010145A384F17AEF30005A2385A17AD2
:1054400097650100938585DF1755010013054556C3
:10545000EF30514A03C6A17AA285176501001305F2
:10546000E58741BFCD476301F4029765010093854D
:10547000E5DC175501001305A553EF30B14717655B
:105480000100130525870DB737E404007C4441462D
:105490009385517A17F5FF1F13050543829717F57A
:1054A000FF1F13056542EF008076092D83C7617BDE
:1054B00003C7517BA20703238405D98F2392F18868
:1054C0001306000A89452244B2409244024903C5AA
:1054D0008186410102838D476301F40297650100D3
:1054E0009385C5D5175501001305854CEF309140C4
:1054F000176501001305C58F45BD03C4617A83C7D5
:10550000517A97650100938565D3220417550100F0
:105510001305054A5D8CEF30F13DA285175501005A
:105520001305C57EEF30113D2945EF30B1400D46E2
:105530009385417A2285EFE0BF9BAA8415C99765C0
:1055400001009385A5CF1755010013056546EF307F
:10555000713AA685175501001305857CEF30913906
:105560002244B24092440249294541016F30913CA6
:10557000239F8186B7E70400116603A387051306FE
:1055800006E8914589B78D476301F40297650100EC
:105590009385C5CA1755010013058541EF30913534
:1055A000176501001305859301B503C4617A83C7AC
:1055B000517A97650100938565C82204175501004B
:1055C0001305053F5D8CEF30F132A28517550100C0
:1055D00013054576EF3011322945EF30B1350D46D0
:1055E0009385417A2285EFE0BF90AA840DC197652B
:1055F00001009385A5C4175501001305653BEF30E5
:10560000712FA685175501001305057481BF239ED0
:105610008186B7E70400116603A38705130606E831
:10562000930500024DB5894763E187029765010044
:105630009385C5C01755010013058537EF30912BB1
:10564000176501001305458C85B383C4617A83C750
:10565000517A97650100938565BEA2041755010034
:1056600013050535DD8CEF30F128A68517550100AF
:105670001305056FEF3011282945EF30B12B228635
:105680009385417A2685EFE0BF862A846304051658
:1056900097650100938585BA1755010013054531BB
:1056A000EF305125A285175501001305A56C7DB576
:1056B000854763F18714834519002244B240924420
:1056C0000249B335B0002380B18817550100130596
:1056D000A56B41016F301122A2852244B240924451
:1056E0004A85024941016FF05FA399476301F402C3
:1056F00097650100938585B4175501001305452B67
:10570000EF30511F176501001305C59971B903C426
:10571000617A83C7517A97650100938525B2220487
:10572000175501001305C5285D8CEF30B11CA2850B
:10573000175501001305C566EF30D11B2945EF3021
:10574000711F19469385417A2285EFE06FFAAA848A
:105750000DC197650100938565AE175501001305CE
:105760002525EF303119A68517550100130545642D
:10577000F5B323968188B7E70400116603A3870574
:10578000130606E8930500083DBB854797650100B1
:105790009385C5AA17550100130585216309F400F7
:1057A000EF305115175501001305C561F5BEEF30F7
:1057B00071141755010013056562EF30B1132945C7
:1057C000EF3051172244B24092440249239201889B
:1057D00041016F30001497650100938525A6175588
:1057E00001001305E51CEF30F110176501001305EA
:1057F000A58F5DBEB240224492440249410182809D
:10580000411106C622C4EFE0AFEE9377F50F95CBBA
:105810002A84976501009385E5A3175501001305B8
:105820002519EF30310D9375F40F1765010013053D
:1058300025C7EF30310C2244B240294541016F3079
:10584000710FB24022444101828001114EC683D6BD
:105850002189B28903D6818226CA4AC806CE22CCC3
:10586000AA842E89CD2183C70189A9C703C4440016
:1058700083C7340017650100130585CE22045D8CB3
:10588000EF3051074A86A68522859D3F638B09022A
:1058900083C7E1889DC76306090283C7018895E332
:1058A0006244F240B249CA8526854249D244056124
:1058B0006F10D01517650100130505CBEF30D11718
:1058C000F1B7F2406244D2444249B2490561828054
:1058D000834755008345450017650100130505C73B
:1058E000A207DD8D6F30110117650100130505C595
:1058F0006F3091148D4763FAB708011126CA06CE9E
:1059000022CC0344350083C4F18897650100938558
:1059100065C6B3378000A387F18809C49765010085
:10592000938505C617650100130505C6EF30817C18
:1059300083C7F18863839700212C83C7F1889DC3B7
:1059400085472306F100B7E7040083A747177000D7
:105950008545130550308297176501001305C5C3AF
:10596000EF30910D9967938757EE2316F100680089
:1059700085479145A30781002307F100EF10100927
:10598000F2406244D244056182808280894763FE8E
:10599000B706011122CC06CE26CA834425008547CE
:1059A0002A846396F404914763FEB70203454500D9
:1059B0008347340022055D8D2394A18209299967CC
:1059C000938767EE2314F100834734002305910089
:1059D000A305F10083474400954528002306F10004
:1059E000EF10D002F2406244D24405618280FDF89B
:1059F0009967938767EE2314F10083D78182A3050B
:105A0000F10023050100A183C1BF828001119967C4
:105A100022CCD517138401892314F1008347040095
:105A200026CA938421892305F10083D70400280026
:105A30009545A305F100A18306CE2306F100EF10E2
:105A4000E07C03D6040083450400176501001305BC
:105A500025B6EF30216AF2406244D244056182806B
:105A60009D677971D9172316F10083C7018906D67E
:105A70002307F1009DCBB7E70400FC47414697F5AB
:105A8000FF1F938565E41305F10082976800CD45FB
:105A9000EF10C07783C5018917650100130545B470
:105AA000EF304165B25045618280B7E70400BC47E2
:105AB000414681451305F1008297C9BFB7670203CC
:105AC0006971938757AA3EC48967938717902316F5
:105AD000F1009387018983C7070023248112A3075C
:105AE00001002307F1009387218983D7070037E45A
:105AF0000400232611122318F1009387818283D793
:105B00000700414648082319F1007C4497F5FF1F20
:105B1000938585DB8297F1452800F5222312A102A7
:105B20007C442C002810794682973C44130561047C
:105B30001306900D8145829730109305700F014533
:105B4000EFD09FBB8320C112032481125561828054
:105B5000B7C7A55A01119387C7333EC483C7F188DD
:105B60003EC6B7F7070003C7070106CE22CCA547FC
:105B70006313F70001A01164930504F0930600106D
:105B80000146254597D0FF1FE780A0E73000930529
:105B900004F0A146294597D0FF1FE78080E683C522
:105BA000F18817650100130565B4EF30A154F24088
:105BB00062440561828001119165A14630009385A0
:105BC00005F02D4506CE97D0FF1FE78080E32247E2
:105BD000B7C7A55A9387C7336310F702B245176555
:105BE00001001305E5A3B335B000A387B188EF30FA
:105BF0006150F240056182808145176501001305FF
:105C000065A4A3870188EF30E14E9937DDB7B7C7A8
:105C1000A55A79719387F7353EC6B7E70400FC476C
:105C2000AA8506D622D4414608088297B7F707000E
:105C300003C70701A5476313F70001A0116493058B
:105C400004E8930600100146254597D0FF1FE78022
:105C500040DB7000930504E8D146294597D0FF1F2B
:105C6000E78020DA17650100130505ACEF30C15C51
:105C7000B25022544561828079719165D14670009D
:105C8000938505E82D4506D697D0FF1FE78060D79E
:105C90003247B7C7A55A9387F73517650100130533
:105CA00065A26310F702B7E70400FC4717F5FF1F72
:105CB000130585C141460C0882971765010013053D
:105CC000659EEF306157B25045618280B7F707009B
:105CD00003C70701A5476313F70001A091654111B0
:105CE000930600100146938505E8254506C697D022
:105CF000FF1FE78000D1B2401765010013058590B2
:105D000041016F306153C16769768146FD17050611
:105D10001397060141836364B7003E858280330791
:105D2000D50003470700B98F214713F81700858373
:105D300063050800B18FC207C1837D171377F70F82
:105D40006DF78506F1B749C1A547054763FFB7065B
:105D500083471500034705003168A207D98F1397C1
:105D60008700A183D98FC207C1831308C85505478F
:105D7000639D0705411106C622C426C203442500BF
:105D8000914763FD8702930754006399F502A301CD
:105D9000C50021822302C5009304340091C6A302EA
:105DA000D500A1822303D5002A84A685A93F269485
:105DB0002300A4002181A300A4000147B240224493
:105DC00092443A854101828005473A858280B7C76F
:105DD000A55A01119387E7343EC42AC6B7F70700D6
:105DE00003C7070106CE22CC26CAA5476313F700D6
:105DF00001A091642A84938504EE93060010014665
:105E0000254597D0FF1FE780C0BF3000A14693858E
:105E100004EE294597D0FF1FE780A0BEA285176535
:105E200001001305A58EEF30E12CEFF03FC9F240E1
:105E30006244D2440561828001119165A14630001F
:105E4000938505EE2D4506CE97D0FF1FE78060BBFA
:105E50002247B7C7A55A9387E7346312F702B245C2
:105E600017650100130505802394B182C205C18125
:105E7000EF304128EFF09FC4F24005618280D147A6
:105E8000D145175501001305E57F2394F182EF30CA
:105E9000612603D58182253FC5B7011126CA06CEEA
:105EA00022CC93F71500AE849DC7AD67371700402D
:105EB0009387A7AA1CC3B7E70400BC4F13060019B9
:105EC000854503C56182829713C51400F240624480
:105ED000D2440561828093F72500638B0710976594
:105EE0000100938565882D464800EF30411583C534
:105EF0001189854793C4240063EDB70299C983C70C
:105F0000E18891CF8545170500201305A5DDEF1029
:105F1000E02F13950401A3880188418145BF4165A5
:105F20000546970500209385E5DB7D15EFF05F8D35
:105F3000CDB7170400200344E4DA9707002083C795
:105F400077DA22045D8CAD67C2059387B755C181AE
:105F50006302F40863E48702A9679387A755630285
:105F6000F40883C7E1888DE741652E867D15970586
:105F70000020938525D7EFF0BF88A9A0B16793874C
:105F8000C755630EF400B5679387D755E31BF4FC40
:105F900017050020130505D5EF10402725A005465D
:105FA00017050020130505D4EFF03F8A83C7018948
:105FB00091EB4800EF30013093150501C181480095
:105FC000EFD04FA6A285175501001305E577EF30F6
:105FD000611281B7170500201305C5D0EFF05F8F60
:105FE000D5B7170500201305E5CFEFF0FF8FD9BF18
:105FF00093F745000145E38B07EC175501001305A6
:10600000E575EF306123EF10203413C544007DBDEA
:10601000411122C437E404005C5C06C6354697553E
:1060200001009385252C176501001305A5BA8297F9
:1060300001E9175501001305E573EF30E11F01A0D9
:106040008327041C82972A840545EF800072EF1095
:10605000A165EF10E143EF7090262285B240224403
:10606000410182801567B71700401307575598C341
:10607000D8439D66558FD8C3D843FD76758FD8C356
:10608000D8431367F70FD8C335671307C7CC98C336
:10609000828041111305800406C622C426C24AC06C
:1060A00097C0FF1FE780805185457D55EFC01FEBEE
:1060B00085457D55EFC0FFF4371400408327840ADF
:1060C0008D451305002093E707202324F40AEFC031
:1060D000FFE8B7E40400EFD06F9AC8581309840CA6
:1060E0001304C40CEF30411517650100130585AE8C
:1060F000EF3081148327C4FF8545414593E70708A6
:10610000232EF4FEEFC0FFEF8D4513050008EFC00E
:106110005FEFEFD0CF890145EFD08F8C85450545E6
:106120008947238AF188EFD04F8D37070004B7E7FE
:1061300000E023A0E710EFD07F8BEFD05F9FC93D39
:10614000EFF07FA7EFF05FCFEFE0AFE28D450D6599
:10615000EFC03FEB170500201305C5C885671CC5B8
:1061600089672320250140C12326250100C95CC978
:1061700083A7841E829783A70408170500001305D0
:1061800005D282972383A182BC4C13060064854507
:106190008297C93D97C0FF1FE78000750145828047
:1061A000B7F7070003C70701A547AE866316F700D8
:1061B0009397450191C301A0AA850146254517D3B0
:1061C000FF1F670003844111B2862E86AA852D45E4
:1061D00006C697D0FF1FE780C082B240014541014B
:1061E00082809307000463E6C7021D71A2CC2A8453
:1061F000080886CE32C6EF209164B2461008A28508
:10620000294597C0FF1FE780C07FF640664425619F
:10621000828039558280411126C2AE848D4522C4C8
:1062200006C62A84EFC0FFDDB717004099C803A552
:10623000C70C418D23A6A70CB240224492444101D1
:10624000828003A5870C418D23A4A70CF5B7834753
:10625000050003471500A207D98FC2076177C187E0
:10626000130727206397E7008345250037050400BF
:106270005DB782809387818918429C4383D645000D
:106280000345070083C5C700035646006396A50073
:1062900083D5E700638DD502011106CE2386A700C2
:1062A0002397D700B705CF00DC4B9385757D050795
:1062B0007D162EC2230001003AC42316C100231705
:1062C000D10099C30A858297F2400561828082805D
:1062D000DC4DDC4B91CBB7E70400904503A3870569
:1062E000914503C5C189028382806D713C083EC619
:1062F000B707E500232291103EC8AA843C083285E6
:10630000232611103ECA23248110232021112E8917
:10631000EF2070652A84975501009385E54D174558
:1063200001001305E568EF20F15CA2851755010017
:106330001305855CEF20115C2945EF20B15FB7059F
:10634000CB009385757D6800EF108041A2856800C1
:10635000EF201057014781467000CA852685EF104F
:10636000A06015C52A84975501009385E548174517
:1063700001001305E563EF20F157A28517550100D1
:1063800013054558EF2011572945EF20B15A8320B6
:10639000C11003248110832441100329011051618D
:1063A00082809387818918429C43797122D406D6D2
:1063B0000348070083C807012A8483D64500035594
:1063C00046006396080183D82701638DD80223888D
:1063D000070105072399D7003708CC00DC4B1308C9
:1063E000787D3ACC1307F5FF42CA23080100231E2B
:1063F000E100231FD10099C7080832C62EC4829736
:106400003246A2452285D535B2502254456182805C
:106410006D713C083EC0B707E5003EC23C083EC473
:106420002326111023248110232291102317010009
:106430002318010023190100231A0100231B010066
:1064400097D7FF1F83D7470E99E3C167FD17231620
:10645000F10097D7FF1F83D7470D81EB9387818981
:106460009C439C43DC4783D7070017D4FF1F1304CA
:10647000A40B584C2317F10083574400484B2318B2
:10648000F10005ED975501009385053E1745010084
:1064900013050552EF201146175501001305053E5F
:1064A000EF2051452945EF20F1488320C1100324F6
:1064B0008110832441105161828097D7FF1F83C7C9
:1064C000170789EBB7E70400BC5782975C4C23AAF7
:1064D0000700E1BFFD1797D6FF1FA38AF6040356F6
:1064E0000701834704014C470A85230BF100EF2085
:1064F000503B938781899C430147814688430A86A4
:106500006C00EF106046AA841DC997550100938561
:10651000A535174501001305A549EF20B13DA68516
:106520001755010013054536EF20D13C2945EF20D2
:106530007140584CB7E70400BC57484B79B797D720
:10654000FF1F83C7D7FEF5D7B7E70400BC4F104441
:10655000854503C5C189829789BF5C4EDC4BB9C7AD
:10656000B1C5411122C417450100130565442E84AD
:10657000975501009385852D06C6EF20B137A2857A
:106580001755010013058532EF20D1362945EF203C
:10659000713AB7E704002244B24003A3870503C55C
:1065A000C189130640069145410102838280411151
:1065B00022C417D4FF1F130424F51C4C06C689C738
:1065C000DC4399C34C488297584CB7E70400BC574A
:1065D000484B82975C4CB240224423AA07004101F9
:1065E00082801387A182834707009306F00B8507FB
:1065F00093F7F70F63E7F6002385F1820345070061
:106600008280930700F8CDBF835745006384070E4F
:1066100001114AC817D9FF1F130909F152C4032AEF
:10662000C90106CE22CC03274A0126CA4EC656C24D
:10663000F15721EF1307D00DFD576368C704B7E981
:10664000040083A709072A841305860042054181B7
:10665000B284AE8A8297232AAA000325C9015C4925
:106660009DEF975501009385651C174501001305A3
:106670002534EF203128175501001305652BEF2035
:1066800071272945EF20112BDD57F2406244D24497
:106690004249B249224A924A3E85056182809387E7
:1066A0004400B705CF002319F5009385757D3105AA
:1066B000EF10000B0325C901834564003105EF206D
:1066C00030200325C9012686D6853105EF20701DAF
:1066D0007146A2854A85EF209116504409CA83A7C6
:1066E0008905854503C5C1898297814779BFEFF048
:1066F0003FD2E5BFFD573E858280411126C297D427
:10670000FF1F938464E2D84C22C437E404003C5455
:10671000484B06C68297DC4C0323C4052244B24092
:10672000924423AA070003C5C1898545410102831C
:10673000411126C2938481899C4006C622C44AC066
:10674000C9C7DC43D9C35CC12300B5002A8497556F
:1067500001009385E5081745010013056525EF2025
:1067600071192945EF20111D9C4023A4070023A285
:10677000070097D7FF1F938727D9DC4FDC4B81C7D2
:106780002955EFF0DFE297D7FF1F9387E7D9DC4F5A
:10679000DC4B91C39D3737E904008327C905894540
:1067A00003C5C18982978327C905914503C5C1895E
:1067B00082979C4003A3470163090300228522447A
:1067C000B2409244024941010283B24022449244C1
:1067D0000249410182800111328506CE22CC26CAAF
:1067E0002E84EF205018AA849755010093858502C6
:1067F000174501001305C51BEF20D10F03078400C7
:106800000356640083554400A686175501001305FE
:10681000E50BEF20310E2945EF20D11197D7FF1F4F
:1068200083C7E7CE639897000145EFF05FD88145B5
:106830000A85FD3DF2406244D244056182806D715B
:1068400023248110232611102322911093F7450051
:106850002E84638107123C083EC0B707E5003EC2A4
:106860003C083EC42317010023180100231901002E
:10687000231A0100231B010097D7FF1F83D7C7C826
:1068800099E3C167FD172316F10097D7FF1F83D740
:10689000C7C781EB938781899C439C43DC4783D79F
:1068A000070017D7FF1F130727C62317F100544F00
:1068B000835747002318F100DC4A95EF97550100F4
:1068C000938585F9174501001305850EEF20910288
:1068D00017550100130585FAEF20D1012945EF2056
:1068E0007105134544008320C110032481108324C3
:1068F00041105161828097D7FF1F83C757C125552B
:10690000BDC7FD1717D6FF1FA303F6C003D60601A8
:1069100083470701CC460A85230BF100EF206078FE
:10692000938781899C4317D7FF1F1307E7BD97669D
:106930000100938666C988430A866C00EF10C00286
:10694000AA8445D197550100938505F117450100AB
:1069500013050506EF20017AA685175501001305DA
:10696000A5F2EF2021792945EF20C17C2685EFF0A3
:106970001FC485BF93F725009DC3B7E70400BC473C
:1069800041468145280882972555EFF05FC22808C7
:106990009305F00FEFF0DFD913452400A9B793F763
:1069A00015000145A9D3EFF0BFA61345140025BF7C
:1069B0005C4D411106C688C323ACF188B7E70400DB
:1069C00083A70708170500001305A5E78297B240C3
:1069D000238EA18801454101828082800111939715
:1069E000050122CC06CE26CAC1872E8463D40706B1
:1069F000B7E70400FC5703C501838297AA8429C125
:106A0000034705009307F0076303F7049306000BA1
:106A10006313D70203474500631FF70083558500C2
:106A20002399B18285471755010013056504A38496
:106A3000F18AEF20216CB7E70400BC5726858297C6
:106A40002165218DF2406244D244056182808355E4
:106A50002500F9B793F715009DC3B7E7040083A796
:106A6000471A17D6FF1F130626AE97F5FF1F93850B
:106A7000653C03C50183829713451400E1B793F782
:106A8000250089CFB7E70400BC4F13060064894591
:106A900003C501838297134524006DB793F78500E2
:106AA0009DC3B7E7040003A8871A1307401F83C7D5
:106AB0000183814613064006994503D5C18A029891
:106AC0001345840041B793F7450095C3B7E404002C
:106AD00083A7041803D5C18A8297BC4C13060064AF
:106AE000914503C50183829713454400A1BF93F7E5
:106AF00005010145A1DB83C7918A99E7C16703D5E9
:106B0000C18AF9176315F5001345040125BF9307E2
:106B1000700F2316F100B7E7040083A7870D03C6A3
:106B200001836C0082976DF18547A384F18AE9BFE8
:106B300083D7C18A6390A7022397B18A2398C18A19
:106B40002399D18A2E8617550100130565F6BE8557
:106B50006F20415A17550100130505F76F20C16DCD
:106B6000C1670111F91723A6F18A22CC23A8018A53
:106B700037E404007C4C06CE894503C50183829727
:106B80007C4C914503C5018382977C4CC14503C56C
:106B900001838297DD472399F182A384018A83C709
:106BA000F18895C78547A307F1008327441713068B
:106BB000F1008545130550308297175501001305E4
:106BC000E5E3EF206167F24062440561828083C79C
:106BD000018917550100130525E7E5F78547A30748
:106BE000F100832744171306F10085451305503043
:106BF0008297175501001305A5E2E1B76D712324B3
:106C000081102326111023229110328401CD89474F
:106C10006306F5028320C1100324811083244110F0
:106C20005161828017550100130505F6AE84EF20EF
:106C3000A160A2852685EFE02FEEE9BFB7E704004B
:106C4000FC4728008297175501001305A5F4EF2093
:106C5000A15E8347810029C01307000B638EE70004
:106C60001387A7051377F70F8D4663E7E602A28522
:106C70002800EFE08FCA79BF8547E3FD87F8834599
:106C800091001745010013052510B335B00023808E
:106C9000B188EF202146BDBF03479100A207D98FDD
:106CA00035671307D755638DE7066366F7022D67CF
:106CB0001307B7556381E70631671307C755638626
:106CC000E70429671307A7556392E702A285280006
:106CD000EFE09FC181B739679306E7656383D70605
:106CE00063E9F6001307E7556388E704A2852800E7
:106CF00099B73D679306F755638AD7041307F7667C
:106D0000E396E7FEEFE0DFD531B70146A285280024
:106D1000EFE0BFB301B7A2852800EFE07FBBDDBD88
:106D20008947E3F987EE9305E4FFC205C1811305A6
:106D3000A100EFC02FCFF9BDA2852800EFE09FBBD7
:106D4000D1BDA2852800EFE07FC4E9B5EFE01FCCFC
:106D5000D1B57D15954763E3A71C175701001307AD
:106D6000A7C60A053A951C41011122CC06CE26CAB7
:106D7000BA972E84828717550100130565D5EF2039
:106D8000A14B05AA03C7250099476312F70203D751
:106D9000450083D7C18A6313F702EFF07FDC834598
:106DA0006400175501001305A5D3EF20A1342387F4
:106DB000018817550100130565D4D1B71755010097
:106DC000130585D0EF204147D9BF03C7250095475C
:106DD0006315F702C16703D7C18AF91703D5A50068
:106DE0006305F702B7E7040083A7C7178297175513
:106DF00001001305A5D1EF20214485472387F188A1
:106E000017550100130505D39DBF2396A18A83D78B
:106E1000E500B7E4040009662397F18A83D70501EA
:106E20001306069003C501832398F18A83D72501B1
:106E3000A1452399F18ABC4C8297BC4C130600648F
:106E4000914503C501838297DD472399F182A3848D
:106E5000018ABC4C0566130606FAC14503C50183C9
:106E600082970356E4008355A400175501001305CB
:106E700025CBEF20212851B717550100130545CC2C
:106E8000FDBD83C525009147639AF50285471755D7
:106E90000100130565CCA307F100EF20E139B7E746
:106EA000040083A747171306F100854513055030EA
:106EB0008297F2406244D244056182809947639A86
:106EC000F5020357440083D7C18A631DF700EFF032
:106ED0003FC98345640017550100130565C0EF20C5
:106EE0006121C1BF17550100130505BEEF20C13454
:106EF000CDB79547639FF5008347140017550100F0
:106F0000130585C5E39D07E617550100130585C6E2
:106F1000BDB517550100130565C6D1B78280411173
:106F200022C417C4FF1F1304E463AA861756010086
:106F3000130606AB2285C14506C6EF20A1300357D4
:106F4000440097C7FF1F9387E7622393E700035727
:106F500064002394E700B240224441018280011181
:106F600006CE22CC6D3F37E404008327841417C675
:106F7000FF1F1306265FD545014582978327841797
:106F80009305F1001305503082978347F100A1C7A4
:106F9000A3070100832744171306F1008545130555
:106FA000503082978327441717C6FF1F1306865C4D
:106FB000CD451305703082978547A307F1008327DD
:106FC00044171306F1008545130550308297F240AF
:106FD0006244056182808327441717C6FF1F13068A
:106FE0006659CD4513057030D5B7130101DE232C4A
:106FF000812037E4040083270408232E1120232A4C
:107000009120232821212326312117050000130573
:10701000259D829713890183994785442300A90000
:107020002318F10097550100938585A59307400625
:10703000174501001305C5972314F110230491008F
:1070400093892189EF20010B83D509001755010091
:107050001305C599EF20010A2945EF20A10D03D59D
:107060000900EFF0DFEB8327441730008545130557
:10707000503082978327441717C6FF1F1306864F89
:10708000CD451305703082978327441717C6FF1F1D
:107090001306464CB5451305603082978327441785
:1070A0001008894513051031829783274417300251
:1070B00089451305203182978327441593050005E0
:1070C0000D45829783274415930500051145829746
:1070D000A3019100230291002304910023240110B5
:1070E0002308010083278416300291451305704060
:1070F00082978327841613063100854513050040C7
:107100008297832784165000854513051040829787
:10711000832784161008854513052040829783270E
:107120008416300085451305504082978327041547
:107130007D558297832744137D5582977D55EFC0F7
:107140000FD58327440C8297EFC0CFB283278414D6
:1071500017C6FF1F13060641D5450145829789478B
:107160001306700F814508082302F100EFB0EF8E7F
:107170008D471306700F814528022308F100EFB0F8
:10718000CF8D91472304F11093878183984383C760
:1071900047003AC42306F100EFE05F9250008545B6
:1071A0000545EFC06FD510089305700F0945EFC076
:1071B000AFD430029305700F0D45EFC0EFD3300010
:1071C00095451145EFC04FD3C1671387C18AF917A1
:1071D0001CC3232207001385C182EFC00FD1832770
:1071E000C41D1385018A82973C48034509008545E3
:1071F00082978320C12103248121832441210329F3
:1072000001218329C1201301012282800111C1675C
:1072100026CA06CEAA8422CC03D5C18AF9176302F6
:10722000F504A1C183D721838D46514763F6F6004B
:10723000F5171397070141836365B70237E404002C
:10724000832784122E862315B10001478146ED4520
:1072500082972AC601ED1755010013056583EF10CB
:10726000B17DF2406244D244056182807C44035681
:10727000A100A68582972C0003D5C18AEFC02FD22A
:107280006DD1175501001305E581EF10F17A8327C1
:10729000C412ED4528008297E9B7011106CE22CC31
:1072A0002DC9854717C7FF1FA30BF72A97C7FF1FD5
:1072B0002388072A37E40400832784179305F10005
:1072C0001305503082978347F100A9CBA307010033
:1072D000832744171306F100854513055030829724
:1072E0008327441717C6FF1F1306C626B545130587
:1072F000603082978547A307F10083274417130660
:10730000F1008545130550308297F24062440561D3
:10731000828097C7FF1FA384072449BF8327441790
:1073200017C6FF1F13060623B54513056030E9BFD6
:10733000C16703D5C18AF9176307F500B7E70400F1
:1073400003A3C7170283828001118547A3070100A9
:107350002384F18AB7E7040083A7471706CE1306F4
:10736000F1008545130550308297F2400561828017
:10737000EFA21FEA2A8408452E89B28909C900C1F3
:10738000970500009385C5746105EF008101814474
:107390007D5AEF10C00963C3A4048144EF10200A92
:1073A00063C6A40497F7FF1F938787A99C43DC4714
:1073B000B307F94091872302F4006381090483270E
:1073C000C900B307F4409587A302F4001C4C89C799
:1073D0009C4799C3228582976FA0DFE65C44139790
:1073E00014008504BA972390470165B71C4813978A
:1073F00014008504BA97239007004DB783278900AE
:107400000547B307F4409587A302F40083570400AF
:10741000638EE7028DC309476384E7040D47E39752
:10742000E7FA975701009387A7C91CCC975701002B
:10743000938707CA11A8975701009387E78F1CCC41
:1074400097570100938747905CC849B79747010059
:107450009387877B1CCC974701009387E77BEDB729
:1074600097570100938787CA1CCC975701009387D1
:10747000E7CAD9BF85E1EFA25FDB00461844834726
:10748000940075839D8B6315F700EF00501C48C472
:107490006FA0FFDB8280EFA2BFD713893500C164E4
:1074A00042094111AA890144F11413590901054AFD
:1074B0002EC6EF00D077B2456346A40001454101D6
:1074C0006FA05FD883A7090013171400BA9783D75A
:1074D00007006388B7006394970063742A0105046A
:1074E000C1BF0545E9BFEFA2DFD1AA892E89328B42
:1074F000B6843A8ABE8AEF80204C55C12685EF10AB
:1075000030368D4763E5A7007D556FA01FD383DB21
:107510004400EF00D0772A84EF00B078930774001E
:1075200031443305850263C5A702EF005076EF00B2
:1075300010762A84EF00F076930774003144330507
:10754000850263CDA702EF0090749307450019A848
:10755000EF003075330585021307F0179307C01746
:10756000E357A7FC2D55E3C277FB63000B02D686D9
:107570005286A6854A85EFE0106341BFEF00707226
:10758000330585029307C5FFF1BF832749001385A3
:10759000C90083D52700EFF01FF071F9B5B7695521
:1075A000ADB797F7FF1F239FA78897F7FF1F938714
:1075B0002789904381470C463307F50042074183F2
:1075C0006393B70082805446139847008507C2969C
:1075D0002390E600D5B797F7FF1F938767869C43F4
:1075E00003C58700828017F5FF1F0355A58582809C
:1075F000EFA2BFC3C1671387D7FF6307E5026368C4
:10760000A700F117630EF50001456FA05FC4138753
:10761000E7FF630EE500FD171D8D13351500F5B767
:10762000EF40003D7D15D5BFEF40801AE5BFEF402C
:10763000E018CDBFEFA27FBF4111AA8401442EC63E
:10764000EF00F05FB2456346A400014541016FA021
:107650001FC09C48131514003E9583570500E3870F
:10766000B7FE0504E9BF03485500814693F7F60FBE
:1076700063E5070181473E85828058459397560010
:10768000BA9703D727006316B70003D70700E304B0
:10769000C7FE8506E1BF8346450001479377F70F94
:1076A00063E4D700814711A81C451316570005074E
:1076B000B29703D60700E313B6FE3E858280EFA2A1
:1076C0003FB593170501C18797EAFF1F938A4A7751
:1076D0006355F00883A70A00C0479C47035704007E
:1076E000198D420541816366F500014422856FA032
:1076F0007FB512052A94DDBFDC4713944900014A87
:107700003E94834744006341FA02014A8347540090
:107710006347FA028509C20993D9090183A70A00C0
:107720009847E3EBE9FCD1B71C4413195A00A6852E
:107730003E994A85EFF01FF011ED050AD9B75C4478
:1077400013195A00A6853E994A85EFF0BFEE19E15C
:10775000050A6DBFE30009FC51BFAA8481497DBFC2
:10776000EFA2BFAC1C452A8481E79307C5001CC566
:107770001C44231204001CC09307F00F63E9B700F8
:1077800093F5F50F2285EF10B0136FA05FAC9394C3
:107790000501C167C18063F7F500A6852285EF105A
:1077A000D015E5B7C18193F5F50F2285EF10501183
:1077B000A6852285EF101012C9BF97E7FF1F938798
:1077C0002768884382801C4599C797E7FF1F23A934
:1077D000A766014582807D55828097E7FF1F9387CA
:1077E0002766984383474500484792073E95828025
:1077F000EFA2BFA3617100451C183EC6B707800108
:107800003EC81C183ECA8357440002CE02D002CCA8
:10781000231EF100834784002A8902D22301F1024A
:107820003C083ED402D6EFF05FFB835705002316D9
:10783000F102EF30706B2307A1025C400355640036
:10784000F18313F717008347F10252055181F99B29
:10785000D98FA307F102EFE0702639C5AA8403553A
:107860000500EF80401683D704002AD26800231C4D
:10787000F10083D72400231DF1001C4803D64700E4
:107880008C43EF1010028347B400CA8617460100EC
:10789000130606318117A305F4006C004810EFE0D1
:1078A00090305D616FA0BF9A2155E5BF1C45B1CFF7
:1078B00003C5A700894613576500630BD7028D46A1
:1078C000630ED70285466300D702130740063305CF
:1078D000E50203C7B700418B15CB83C7B700BD8B4B
:1078E0003355F54082801375F5031307803EC5B705
:1078F00009671375F50313070771D1BF372709000F
:107900001375F5031307077CD9B701458280EFA2F1
:10791000DF9103A98500630509048347B900AE849C
:1079200093F7070E91CF03459900930520030D812E
:107930000505B305B50288446105EFF0B0320DA02E
:107940002E85EFF0BFF62A8401CD11238325C900CF
:10795000B307B54063F887002E94B305A440E1FD5A
:107960006FA0FF8E8545C1BFEFA23F8C2A8403D54F
:107970000500011132C636C43AC22EC002CA02CC7A
:1079800002CEEF80400482452ACA22852ECCEFF039
:10799000DFE403570500231EE100EF30F054A24658
:1079A00032469247230FA10036874C08B2862285C3
:1079B0000146EFF05FB305616FA07F89EFA2FF86FC
:1079C00061711C183EC6B70780013EC81C183ECA2C
:1079D0003C0800453ED4AA8402CC02CE02D002D29A
:1079E00002D6EFF09FDF8357050035592316F102C9
:1079F000EF30904F2307A10209C48357440091E759
:107A000021594A855D616FA09F840355640052052A
:107A10005181EFE0B00A2A8965D58347B40093F716
:107A2000070E89C713058401EFF0502583574400E2
:107A3000231EF100834784002301F1025C400355BB
:107A40000900D98313F7070883471102231CA100FB
:107A500093F7F707D98FA300F10283572900231D5D
:107A6000F1005C40F18313F717008347F102F99BA3
:107A7000D98FA307F102EF7010752AD251D1834735
:107A800094006800139757008347B400FD8BD98F8B
:107A9000A305F4001C4803D647008C43EF10606038
:107AA000A687174701001307A70F740005464C105F
:107AB0002685EFF05FA32A8929D58347B400A685E0
:107AC000FD8BA305F400EFF09FE425BFEFA2EFF5D7
:107AD000832485FE2A8441112685EFF03FDD83470C
:107AE00034FF93F7070E9DC32AC62685EFF05FD0BB
:107AF00019C9834734FFB245FD8BA309F4FE81C544
:107B00002285EFF0301641016FA06FF46DDD832701
:107B1000C4FF2685829765F9834734FF93F7070EE4
:107B200081C72285EFF09015032584FEEFF01FE951
:107B3000D9BFEFA28FEC9C4141112A8903C70700EE
:107B400089472E8493566700638CF6020D46638244
:107B5000C6049307F0076302F7022E85EF10A060BA
:107B6000AA848149C16B130C490097E7FF1F9387D3
:107B7000272D9C43984763ECE90241016FA0AFEBCE
:107B800003D745008547E3FAE7FE2E85EF108061B5
:107B9000C1BF03D74500E3F2E7FE2E85EF10A05CDE
:107BA000AA842285EF10805DC204C98C5DBFDC47CA
:107BB0000355A900139A49003E9A93170501C187FE
:107BC000635DF00083570A006395A70263E57403C1
:107BD0008327CA00034D5A001DA0A1672167A98F02
:107BE0001307F7EFE374F7FE63950900EFF05FA06A
:107BF00071FD85099DBF83278A00034D4A00835D7F
:107C0000A90003576900216A138BC7003AC6814A4D
:107C100033CA4D01631E5D0197E7FF1F9387C7229B
:107C20009C43E1DBA2866286814526858297D1B797
:107C3000A1679387F7EF930C4BFF63F04703B245BF
:107C40005A85EFF05F8519CD03278B00104719CABD
:107C500010436380C4023107D5BFEE856685EFF01F
:107C60007F9D71FD93861A0093FAF60F130B0B029A
:107C700055B7835644005C43E3EDF6F622853AC6D9
:107C8000EF10603DA1679387D7042A8A035D440003
:107C9000324763E897008347D90093E707F8A306C4
:107CA000F9001C4766852286E2858297C1670844F1
:107CB000FD17337AFA00529508C02312A40115BFAC
:107CC00097E7FF1F9387C7179843814715C314474A
:107CD000814763FFD500939745004C47BE9519C96E
:107CE00003C7550081476375E600DC451606B29769
:107CF0003E85828003C745008147E37BE6FE16068A
:107D00009C45F5B7EFA2CFD0AA892E8A814497EA85
:107D1000FF1F938AEA1283A70A00984763E4E400EE
:107D20006FA04FD2DC471394440001493E9413BB2B
:107D3000140083474400634BF900014913BB14004E
:107D400083475400634FF9008504F1B70844931743
:107D500059005287DA860146A2853E958299050927
:107D6000C9BF4844931759005287DA860546A28551
:107D70003E9582990509E9B7EFA22FCB814517F50A
:107D8000FFFF1305255F97E7FF1F239D070AEFF00D
:107D90007FF76FA0CFCB97E7FF1F9387670A9C43BE
:107DA00081CFEFA28FC8814517F5FFFF1305855CD2
:107DB000EFF05FF56FA0AFC98280EFA26FC537E427
:107DC00004008327841241112315E100AE89328912
:107DD000368A3A8681460147ED45AA8482972AC6AB
:107DE00021C50356A100D285EF1061258327C41356
:107DF000CE8526858297058915C58327440D2314D2
:107E0000210101462C00268582972A8401C9B7E703
:107E1000040083A7C712ED452800829722854101FF
:107E20006FA04FC24944E5B76554CDBF5C41FD1713
:107E30005CC18280EFA26FBFB7E70400FC5F82974E
:107E400095473305F50281450D816FA04FC0EFA224
:107E5000CFBDB7E70400FC5F829795473305F50275
:107E60000D816FA0CFBEEFA24FBCB7E7040083A780
:107E7000870B0355050082976FA06FBDEFA2EFBA85
:107E8000035505003287AE8617B6FF1F0356A6744A
:107E900097E5FF1F938585FBEFF03FF26FA02FBBA7
:107EA000EFA2AFB8B7E7040083A7C71782976FA008
:107EB0000FBAEFA28FB7B7E7040083A7871397E540
:107EC000FF1F9385A5F8829701456FA04FB8EFA2D9
:107ED000CFB5B7E7040083A7C71F814517B5FF1FBC
:107EE0000355656B82976FA08FB6EFA20FB4B7E70B
:107EF000040083A7871397E5FF1F938525F68297D4
:107F000001456FA0CFB4EFA24FB2B7E7040083A73B
:107F1000C71F814517B5FF1F0355E56D82976FA0F9
:107F20000FB3EFA28FB02E85EF600055EF60900D7C
:107F30006FA0EFB1EFA26FAFEF60D0176FA02FB1BE
:107F40005C49E1175CC95CC583572501A10723196A
:107F5000F50083570501A1072318F5008280F1473A
:107F60003305F50297E7FF1F938747F19C433E9542
:107F700082808D476317F60603D74600854763F274
:107F8000E706EFA28FAA368536842E89EF10A01D52
:107F900039C18357440093140501C18063ED9702F2
:107FA0002285EF10401CFD14231294009307A002B9
:107FB000630EF5009307B0026301F5029307900288
:107FC000631BF5002285EFC0B07E31A00146CA8553
:107FD0002285EF80000F6FA08FA72285EF00105938
:107FE000DDBF828097E6FF1F938686E99C420145AC
:107FF00099CF9843D44217E6FF1F2323E6E8639600
:10800000D70097E6FF1F23AFE6E61385C7FE828001
:10801000EFA2AFA1E9267144330585029145EF70C7
:10802000606201E565556FA08FA297E7FF1F23A54A
:10803000A7E47526330585029145EF70A0607DD1D8
:1080400097E7FF1F23ACA7E2592E97E7FF1F239F57
:10805000A7E0712697E7FF1F239BA7E09747010042
:10806000938747B917E7FF1F2326F7E0970700001C
:10807000938747ED17E7FF1F232CF7DE014565B710
:10808000EFA2AF9AAA8517E5FF1F130525DEEF10B3
:1080900060216FA0CF9BEFA24F99EFF07FFEEF1012
:1080A000E02197E7FF1F9387A7DD9C4381CF1387CC
:1080B000C7FE09CB83D5C7FF17E5FF1F1305C5DC36
:1080C000EFF0403A6FA0AF98EFA22F96EFF09FF13C
:1080D00019C9834785002A8493F7070499E7035554
:1080E000E500EFF05FFB6FA08F968347C500930418
:1080F000450117E9FF1F1309A9D885E38327090064
:108100005CC997E7FF1F23AD97D683274900E1FF9E
:1081100097E7FF1F23A897D6F9B7FD172306F500A9
:108120006105EF60E07E8307840063CB070483472B
:10813000840093E707F82304F400B7E704009C5F8A
:1081400082974205A94741813375F5028347840030
:1081500093F707FCC98F2304F4008347D4003E95AE
:108160001C402318A40089CF984319CB8347C4002F
:108170005040814585073305F5024205418102974C
:10818000832709005CC897E7FF1F23AB97CE83279F
:10819000490089E797E7FF1F23A697CE8347C400CE
:1081A000B9D38355040117E5FF1F1305E5CDEFF0A3
:1081B000602B15BFEFA26F8797E7FF1F938707F22A
:1081C0009C4701448583858B81EFAE84B2853A86D6
:1081D000EF1020142A8409C5EF10200B829408CCDC
:1081E00022856FA0CF86EFA2AF8241112E8932C6C1
:1081F000AA89712C324713060502CA86970500002A
:10820000938525D617E5FF1F130545C6EFF09FFAA6
:108210002A8429CD9304C50065261946AA8526859A
:10822000EF00306885452685EF0010651745010091
:108230001305059A4E95834505002685EF00506885
:108240005C4831468145A1075CC85CC48357240162
:10825000E1172319F40083570401E1172318F400F0
:108260001C4C3E85EF907FFFA30425012285410130
:108270006F905FFDEF927FFB4111AA842EC632C43E
:10828000EF100003004DB2452246834784000CC026
:1082900050C093F7F70393E707042304F40023186F
:1082A00004002685EF00707E83479400A9462317BB
:1082B000A40013D7370005073307D7029D8B850726
:1082C0002306F400A306E40083C70401D848850709
:1082D000230FF7FE17E7FF1F130787BA5843232A18
:1082E0000400930744011DEB17E7FF1F232CF7B889
:1082F00017E7FF1F2326F7B817E4FF1F1304C4B8BE
:108300002285EFF0A00B1C44858B5D8D09E581452E
:108310002285EFF0201541016F907FF31CC317E712
:10832000FF1F2321F7B6C9BFEF923FF0970500006A
:10833000938565C40145EFF0DFBE01456F903FF1C5
:10834000EF92BFEEEFF01FBF6F907FF08347C50045
:10835000A1E7EF929FED2A840355E500EFF05FD28D
:1083600015C98347840093F7F7FB2304F4001C40EE
:1083700091C7DC4381C74C4001458297EFF09FC60F
:1083800017E5FF1F130545B0EFF0400F0355E4005C
:10839000EFF07FD06F90BFEB8280EF921FE997E7FD
:1083A000FF1F9387E7AD97050000938525D217E55A
:1083B000FF1F130565AD23A0070023A20700EFE010
:1083C000507E6F90DFE81C4D91CBDC4381CBEF9268
:1083D000DFE58345070082976F907FE7828097E70C
:1083E000FF1F9387A7AC9C4303C50700828097E7D4
:1083F000FF1F9387A7AB9C4303C51700828097E7B5
:10840000FF1F9387A7AA9C4303C52700828097E795
:10841000FF1F9387A7A99C4303C54700828097E766
:10842000FF1F9387A7A89C4303C53700828097E767
:10843000FF1F9387A7A79C4303C55700828097E738
:10844000FF1F9387A7A69C4303C56700828097E719
:10845000FF1F9387A7A59C4303C57700828097E7FA
:10846000FF1F9387A7A49C4303C58700828097E7DB
:10847000FF1F9387A7A39C4303C59700828097E7BC
:10848000FF1F9387A7A29C4303C5A700828097E79D
:10849000FF1F9387A7A19C4303C5B70011E11D45AA
:1084A000828097E7FF1F938767A09C4303C5C7009F
:1084B000828097E7FF1F9387679F9C4303C5D70080
:1084C000828097E7FF1F9387679E9C4303C5E70061
:1084D000828097E7FF1F9387679D9C4303D5070121
:1084E000828097E7FF1F9387679C9C4303C5270102
:1084F000828097E7FF1F9387679B9C4303D54701C3
:10850000828097E7FF1F9387679A9C4303D5670193
:10851000828097E7FF1F938767999C4303D5870164
:10852000828097E7FF1F938767989C4303C5A70145
:10853000828097E7FF1F938767979C4303C5B70126
:10854000828097E7FF1F938767969C4303C5C70107
:10855000828097E7FF1F938767959C4303C5D701E8
:10856000828097E7FF1F938767949C438857828098
:1085700097E7FF1F938787939C4303D5C7028280A9
:1085800097E7FF1F938787929C4303D5E70219E182
:108590001305800C828097E7FF1F938727919C43E8
:1085A00003C50703828097E7FF1F938727909C43AB
:1085B000C85B828097E7FF1F9387C78E88438280BE
:1085C00097E7FF1F9387478E8843828019E17D5587
:1085D0008280F5DE984265DFFDD917E7FF1F13079C
:1085E000E7AF1847AA877155058B6319072203C5A2
:1085F00007001547E37DA7FC03C737001305F00507
:108600007D171377F70FE364E5FC03C35700E3001E
:1086100003FC83C86700E38C08FA03C77700494569
:1086200079171377F70FE364E5FA03C7A70011483A
:108630001305F7FF1375F50FE36BA8F803CE97004A
:108640000D481305FEFF1375F50FE362A8F803C884
:10865000B7006309080065181378F80F1305600D5B
:10866000E36705F703C5C700794879151375F50F5A
:10867000E36FA8F403C8D7000D457D181378F80FF1
:10868000E36705F503D80701930E40175118420818
:1086900013580801E3ED0EF303C8E7007D181378C3
:1086A000F80FE36605F303C827017D181378F80F68
:1086B000E36F05F103C88700C54E75181378F80FEE
:1086C000E3E70EF103D86701856E938EBEE06D1867
:1086D000420813580801E3EC0EEF03D847016D1868
:1086E000420813580801E3E40EEF03D88701791814
:1086F000420813580801E36C05ED03C8A7017D1873
:108700001378F80FE36505ED03C5B7011D487D1526
:108710001375F50FE36DA8EA03C5D7017148791504
:108720001375F50FE365A8EA03D5E7011308E00F19
:108730007D1542054181E36CA8E803C5070249485D
:1087400079151375F50FE364A8E8C85301C937C854
:1087500034005915130858BFE36BA8E603A8870235
:1087600037C53400130555BF5918E36205E717D51F
:10877000FF1F232BC57203C6050117D5FF1F232733
:10878000F5720545E375C5E403D82501D049337674
:108790000603E31E06E203C61501E30A06E217D646
:1087A000FF1F2321B67083C5270001466387A500FC
:1087B00003C61700F1453306B60283C707039305C6
:1087C000C00272971A071307C70516031A9796086F
:1087D0004697B387B70241553E9732974207418388
:1087E000636EE802EF927FA43685EF60D06FEFD022
:1087F000B0212A84EF80B01D2A94EFC090252A94DE
:10880000EF7040072A94EFF0BF802A94EF20506366
:108810002A94EF50406622956F907FA38280EF925A
:10882000DFA04111A307A100EF80801E9305F10096
:1088300017050000130565B9EFF0CFCC01454101E4
:108840006F90FFA0EF92FF9B17E4FF1F13040489B2
:108850000328840079599368180097E4FF1F23A325
:10886000148913781800631E0800BA84BE89368BF9
:10887000328A2E89AA8AEFE01FD67D15269509E552
:1088800031594A856F907F9BEFE0FFD47D15269587
:10889000A167E357F5FE97E7FF1F938727BB984330
:1088A0003E8C814B11C70145EFC0B03E933B150094
:1088B0004A85DA865686D285EF7070372A8911CDBF
:1088C0001C44F99B17E7FF1F232EF78083270C001A
:1088D000CDDBE3880BFA82976DB7268597E7FF1FFC
:1088E00023A00780EFE0FFCB4146CE8517E5FF1FB1
:1088F00013054588EF00A174EFA070080325040B51
:10890000EFA0700A0545EFA070100545EFF03FF1AC
:108910008DBF97D7FF1F9387677C9C47858BD5C7F3
:10892000EF92BF9017E5FF1F1305058397D7FF1F31
:1089300023A6077A97D7FF1F23A4077A97D7FF1F8D
:1089400023A2077AEFE09033EF40C002EFE0F00A95
:10895000EFE0700F97D7FF1F9387C7769C4381C7BF
:108960000545EF60B03397D7FF1F9387675F9C4340
:1089700089C741657D15EF50A06BEFC0703AEFA03D
:10898000F00097E7FF1F9387678A9C4313971701AF
:1089900063540700EFC0A04597D7FF1F23AC077CA7
:1089A00097D7FF1F23AA077C97D7FF1F23A8077C11
:1089B00097D7FF1F23A6077CEFF09F984923EFF07E
:1089C000AFBBEFC080676F909F88828097D7FF1FF3
:1089D0009387C77088438280EF923F85EF60B07EB7
:1089E000EF7080006F90BF86EF929F822A8493047D
:1089F000140201112E85B289A685214636C63A8910
:108A0000EF0081611DE1B24638082686CE85130548
:108A10009404EF40604321462C084A85EF00C15F73
:108A20001335150005616F90FF810145E5BFEF9299
:108A3000CFFF9305450617D5FF1F13056547EFE0E8
:108A400070226F90DF80EF924FFE41112EC6EFF043
:108A50000FC0B24588C141016F906FFFEF924FFB8D
:108A6000AA842E84EF605078AA8985452285892DB5
:108A700083C7E4011389940899E313890403CE851D
:108A800022853D2D2146930519022285192D97D760
:108A9000FF1F9387A7648C432285EF00E06821467F
:108AA000938584022285F52B6F90CFF9EF926FF5B5
:108AB0003971EFC0E04E9305400645EDEF60D06F91
:108AC000630E051097D7FF1F83C7474013B71700E2
:108AD00097D6FF1F238CE63E014489CFC16417D986
:108AE000FF1F1309A95F9309400EFD14EFF03F9893
:108AF0006348A408EFF0AFB54169B7290900096AD6
:108B0000FD7A2A8B81447D199389F97B130A0A71B6
:108B1000938A8AC7EFF0BF9563D5A4041304400E6F
:108B2000B387840217D7FF1F1307475B0324070B84
:108B30003E948357C4016386270918403307EB40EE
:108B400063EAE900834744008507B3874703D69764
:108B50006369F706014681450945EFF0CFE8AA8B26
:108B600029E1EF20105A8547631FF5048965938535
:108B7000057117D5FF1F1305A533EFE0B00EA1A8AF
:108B8000B30734030327090BBA9703D7C701630858
:108B9000970003C75700A38207002382E70005045C
:108BA000B1B79305C5002285EFF05FEB5E852286A5
:108BB0009735010093850503EFF0CFEB5E85EF005D
:108BC000E06F850481BF97D7FF1F938727519C478C
:108BD0008D83858BC1FF21616F902FE6014685450E
:108BE000094502D002D202D402D6EFF0CFDFAA8428
:108BF0007DD1EFC0203A1389C4002A8481454A857B
:108C0000C1210C4041464A85692983294400638873
:108C100009084E8502D802DA02DC02DEEF00816923
:108C20002ACE141005462C0808184ECCEF406019C7
:108C30001375F50F2DE58355840093E525004A85CE
:108C40006D2911460C104A85A92901469735010066
:108C50009385C5F92685EFF0EFE12685EF000066E4
:108C60005C40B5DB014685450D45EFF0CFD7AA84C2
:108C70003DD148401389C400EF00C1632AC64A852C
:108C8000C5263246636AC5004C404A85192901460B
:108C900081452685EFF00FDE26850D252DBF8355F6
:108CA000840071BFEF926FD897D7FF1F9387074358
:108CB0009C4719CD93E7870017D5FF1F1305451F64
:108CC00017D7FF1F2320F742EFE060786F902FD86F
:108CD000DD9B17D7FF1F2327F740EF2090427DF53C
:108CE00017D5FF1F1305C51CEFE04079C5B7EF92FC
:108CF0004FD14169AA892E8AB28A368BBA8B8144B8
:108D000017DCFF1F130C8C3D930C400E7D19EFF008
:108D10000FF663C4A40001442DA033849403832779
:108D20000C0B3E948357C401638027055A87D6866F
:108D30005286CE8513050403EFF01FCB11C52380A7
:108D40000B0022856F906FCF8347F40191CF5A8734
:108D5000D6865286CE8513059408EFF0FFC809C564
:108D600085472380FB00F1BF850455B78357450035
:108D7000638D0716EF92CFC901112A84ED2619C51C
:108D80008547630AF50405616F90CFCBEFC04021A2
:108D90007DF9835744004947ED9BE396E7FEC145C3
:108DA00022854524AA842285F52E0357440002CE4D
:108DB00091472A896317F700228539293C082ACC74
:108DC0003ECEEFC0201D5C55DDDF74084A86A685C7
:108DD000054582974DBF03574400D147E3F5E7FAB5
:108DE000032A0400C169014997DAFF1F938A0A2FF9
:108DF000130B400EFD19EFF08FE76344A90C228599
:108E0000032A04008D26A1452A8922851D2CAA84C7
:108E10002285D92614402A86AA8978082685CA85FB
:108E2000EFF0FFECAA8425D103C7F401894763154D
:108E3000F7008347C101A1DB5546D2851385640045
:108E4000EF00E11F0145EF60103801C583D7C40171
:108E5000B1EB97D7FF1F938767289C47935519005D
:108E6000858913D73700058B11CB8983858B639751
:108E7000B70001452EC6EFF0FFE2B2454E85EF6028
:108E8000703C0346C1012A84937519002685EF7052
:108E9000703131C92685EF607037268511C00145D4
:108EA000EF60D061EF20F0258547E31EF5EC83C726
:108EB00054001307F00FE388E7EC8507A382F40062
:108EC000D9B5B304690383A70A0BBE9483D7C40141
:108ED000638937015546D28513856400EF00C113BD
:108EE00071D1050909BF5DDC5DBF8280EF924FB291
:108EF000EF60902C11CDC164014417D9FF1F1309F5
:108F0000E91D9309400EFD14EFF06FD6634AA400EB
:108F100017D5FF1F1305C5F9EFE060536F908FB2AF
:108F2000330534038327090B3E958357C5016386B8
:108F3000970023120500EF60702D0504F1B797D755
:108F4000FF1F9387A7199C478D83858B99EBEF9221
:108F5000CFAD17D5FF1F1305A5F5EFE020526F9099
:108F60000FAF8280EF926FAC97050000938545B4F8
:108F700017D5FF1F1305C5F3EFE0A0426F902FAD8B
:108F8000EF92AFAA8841B7E70400BC5B0505420534
:108F90004181829709C585472300F50005056F903B
:108FA0000FAB83C7F5FF2E858507A38FF5FE828063
:108FB00083C7F5FFFD1793F7F70FA38FF5FE99EB26
:108FC000EF92AFA6B7E70400BC571385F5FF829771
:108FD0006F90EFA782801C41035745008D8FBA9593
:108FE0001CC12312B5003E85828093D78500A2055F
:108FF0001441DD8D835745001387E6FF18C18907AB
:109000002312F50013D685004111238FB6FEA38FDE
:10901000C6FE4101828018419307F7FF1CC18357A8
:10902000450085072312F500A30FB7FE8280835702
:1090300045008D8F2312F5001C41BE950CC12E8575
:109040008280AA8703D7470008410D8FAA952392F3
:10905000E7008CC38280184108453305A740828011
:1090600083574500035765001D8F1C410845338514
:10907000A7403305A7408280EF922F9B41112EC657
:109080002A84EFF0FFFDB2456373B50001A083575A
:1090900044000840BE952312B4003E9541016F90F4
:1090A0000F9BEF928F9841112E84B28532C6EFF05C
:1090B000BFFC3246A285EFF0907841016F902F9966
:1090C000EF92AF962E848545EFF01FFB23008500BD
:1090D0006F90EF97EF926F9541112317B10089457B
:1090E000EFF09FF98347E1002300F5008347F1008B
:1090F000A300F50041016F908F95EF920F9393D7E6
:109100008500A2054111DD8D2317B1008945EFF0DF
:10911000BFF68347E1002300F5008347F100A30079
:10912000F50041016F90AF92EF922F901397850158
:1091300093D78501C166938606F0D98F13D7850032
:10914000758FD98FA2053707FF00F98D4111DD8D8D
:109150002EC69145EFF05FF26C001146EFF0306ED5
:1091600041016F90CF8EEF924F8C1C41854503C417
:109170000700EFF0DFEB22856F906F8DEF92EF8AA3
:109180001C414111894503C7070083C71700230706
:10919000E100A307F100EFF09FE90355E100410171
:1091A0006F90EF8AEF926F881C414111894503C788
:1091B000070083C717002307E100A307F100EFF0C2
:1091C0001FE78357E100410113D58700A2075D8D9A
:1091D000420541816F90AF87EF922F850C4141117D
:1091E0002A8411466800EFF0906591452285EFF0E2
:1091F0001FE4B247C166938606F01397870113D523
:109200008701598D13D78700758F598DA2073707AE
:10921000FF00F98F5D8D41016F906F831C45BE95F6
:109220000CC18280AE87944391E6584101EF0CC196
:109230005CC1828003C7570013671700A382E70051
:10924000B687D5B70CC3EDB7AA87084119CD184129
:10925000D44398C36313D500D8C32A870346570065
:109260009376160081E6232007008280944381CA0A
:109270008C4203A847008CC363930601CCC3799A40
:1092800014C3A302C7003687D1BF1C45DC471D8D20
:10929000B777DBB6938777DB09853305F50242059F
:1092A00041818280F147B385F50248452E95828041
:1092B0008347450085072302F5008280EF82FFF691
:1092C0002A8419E06F80BFF883474400E5DFFD176B
:1092D00093F7F70F2302F400F5F71C4403D7270098
:1092E00005072391E700DC4399C3228582974C4808
:1092F00089CD83475400898B99E71C4422859C477C
:109300009C439C478297232A0400004023200400AA
:109310004DBFEF829FF18357250041112EC691E783
:109320000144228541016F809FF203570500814768
:10933000F146E307F7FEB385D702404585072E9433
:109340008345440008C4F5F5B247AA8481E7232A7F
:10935000040009A81C456C0022859C439C4382970D
:1093600048C85DDD85472312F400B247232004007E
:10937000231804002319F4005C485CC483D724003C
:10938000FD172391F40071BFEF823FEA97D7FF1FCB
:10939000938707B48843232605002324050041054D
:1093A000EFE0C00D6F80BFEAEF823FE817D4FF1FE8
:1093B000130404B21C40411189CF9C472300B5001F
:1093C0002AC65CC1EFF05FFC1C40DC4399C3324508
:1093D000829741016F80BFE7034745001DEB584D61
:1093E000AA877D550DCBEF825FE41CC3DC4797D67F
:1093F000FF1F23AFE6ACF156130507012390D700FA
:109400009705000093858501EFD0B07901456F8005
:109410001FE47D5582808280EF823FE10111614629
:1094200081452800EF807FE397D7FF1F938747AAE6
:109430009C4328009305F00FDC473EC6EFF0DFF6B3
:1094400005616F80DFE097D7FF1F938767A89C4374
:10945000D847A1679387C7026312F70A397106DEFE
:1094600022DC26DA80004AD84ED652D456D2328533
:10947000B284EFF05FCFAA892685EFF03FD02318A2
:10948000A4FC2685EFF09FCF2319A4FC2685EFF0DE
:10949000FFCE83D744000A8A231AA4FC858393F75E
:1094A000F70F230EF4FC8607BD0793F7073F330140
:1094B000F1408A8A01498347C4FD6365F902CE857C
:1094C000130584FC232C54FDEFF01FEE5281130191
:1094D00004FCF2506254D2544259B259225A925A60
:1094E000216182802685EFF07FC993171900D697F6
:1094F00005092390A7001379F90F75BF828097D7CC
:10950000FF1F9387E79C9C43D847A1679387A702D7
:109510006310F70A397106DE22DC26DA80004AD8A9
:109520004ED652D456D23285B284EFF0DFC3AA8928
:109530002685EFF0BFC4FD572318A4FC2685231908
:10954000F4FCEFF0BFC383D744000A8A231AA4FCBB
:10955000858393F7F70F230EF4FC8607BD0793F777
:10956000073F3301F1408A8A01498347C4FD63659F
:10957000F902CE85130584FC232C54FDEFF0DFE2C5
:109580005281130104FCF2506254D2544259B25930
:10959000225A925A216182802685EFF03FBE9317AE
:1095A0001900D69705092390A7001379F90F75BF05
:1095B000828097D7FF1F9387A7919C43D847A167C5
:1095C00089076318F708397106DE22DC26DA800085
:1095D0004AD84ED652D456D232853289EFF0BFB82F
:1095E000AA894A85EFF09FB9835749000A8A231850
:1095F000A4FC858393F7F70F230CF4FC8607BD07C3
:1096000093F7073F3301F1408A8A8144834784FD01
:1096100063E5F402CE85130584FC232A54FDEFF0A4
:10962000BFD85281130104FCF2506254D254425903
:10963000B259225A925A216182804A85EFF01FB4B2
:1096400093971400D69785042390A70093F4F40F02
:1096500075BF828097D7FF1F938787879C43D84722
:10966000A1679387E7046312F70A397106DE22DCEB
:1096700026DA80004AD84ED652D456D23285B284E9
:10968000EFF07FAEAA892685EFF05FAF2318A4FC28
:109690002685EFF0BFAE231AA4FC2685EFF01FAE9F
:1096A00083D744000A8A2319A4FC858393F7F70F14
:1096B000230EF4FC8607BD0793F7073F3301F14003
:1096C0008A8A01498347C4FD6365F902CE85130583
:1096D00084FC232C54FDEFF03FCD5281130104FC98
:1096E000F2506254D2544259B259225A925A2161CC
:1096F00082802685EFF09FA893171900D697050959
:109700002390A7001379F90F75BF828097C7FF1FB9
:109710009387077C9C43D847A1679387C70463104E
:10972000F70A397106DE22DC26DA80004AD84ED6E6
:1097300052D456D23285B284EFF0FFA2AA89268590
:10974000EFF0DFA3FD572318A4FC2685231AF4FCB1
:10975000EFF0DFA283D744000A8A2319A4FC858393
:1097600093F7F70F230EF4FC8607BD0793F7073F27
:109770003301F1408A8A01498347C4FD6365F902D8
:10978000CE85130584FC232C54FDEFF0FFC15281DC
:10979000130104FCF2506254D2544259B259225A75
:1097A000925A216182802685EFF05F9D9317190000
:1097B000D69705092390A7001379F90F75BF82800A
:1097C00097C7FF1F9387C7709C43D847A167DD07E2
:1097D000631BF702EF827FA5797132853284EFF047
:1097E0009F982AC62285EFF07F992311A102228536
:1097F000EFF07F97B2452300A1022808EFF0DFBA0F
:1098000045616F80DFA4828097C7FF1F9387476CF5
:109810009C43D847A16793878704631BF702EF82B5
:10982000DFA0797132853284EFF0FF932AC622855A
:10983000EFF0DF942311A1022285EFF0DF92B24511
:109840002300A1022808EFF03FB645616F803FA0DA
:10985000828097C7FF1F9387A7679C43D847A1675C
:109860009387A704631CF700EF823F9C0111280037
:109870008145EFF07FB305616F807F9D828097C740
:10988000FF1F9387E7649C43D847A16793875702DC
:109890006311F702EF827F9901113285EFF0BF8CDF
:1098A0002308A10081452800EFF01FB005616F80FB
:1098B0001F9A828097C7FF1F938787619C43D84771
:1098C000A1679387E702631FF702EF821F960111DA
:1098D00032853284EFF09F8AAA842285EFF01F8AB6
:1098E000854719E52285EFF01F884205B337A000B0
:1098F00028008145231891003ECAEFF0FFAA0561B8
:109900006F80FF94828097C7FF1F9387675C9C439B
:10991000D8479947631FF704EF823F9179713285E9
:109920003284EFF05F842AC62285EFF03F85231052
:10993000A1022285EFF03F832301A1022285EFF0EF
:109940009F82A301A1022285EFF0FF812302A102E1
:109950002285EFF05F812313A1022285EFF0BF8003
:10996000B2452314A1022808EFF01FA445616F80BF
:109970001F8E828097C7FF1F938787559C43D847C8
:10998000A1679387C703631FF704EF821F8A79716A
:1099900032853284EFF02FFD2AC62285EFF00FFECC
:1099A0002310A1022285EFF06FFD2311A102228571
:1099B000EFF06FFB2302A1022285EFF0CFFAA302A2
:1099C000A1022285EFF02FFA2303A1022285EFF0F6
:1099D0008FF9B245A303A1022808EFF0FF9C45616F
:1099E0006F80FF868280EF825F8401112A84EFF00E
:1099F0008FF7AA842285EFF06FF82285EFF00FF839
:109A0000035744008D4763F5E7002285EFF00FF719
:109A10002285EFF0AFF62800A685EFF0FF980561EC
:109A20006F80FF8297C7FF1F9387874A9C43D84761
:109A3000A167FD076319F700EF822FFF3285EFF072
:109A40009FFA6F80DF80828097C7FF1F9387474808
:109A50009C43D847A167E5076311F706EF82EFFC47
:109A6000797132853284EFF00FF02AC62285EFF04B
:109A7000EFF02285EFF08FF02310A1022285EFF0A6
:109A8000EFEF520551812311A10222852302010229
:109A9000EFF06FEDA302A1022285EFF0CFEC2303DC
:109AA000A1022285EFF02FECB245A303A102280802
:109AB000EFF09F8F45616F808FF9828097C7FF1FFE
:109AC000938707419C43D847A1679387E7036319AE
:109AD000F700EF828FF53285EFF0FFF06F802FF700
:109AE000828097C7FF1F9387A73E9C43D847A167F3
:109AF000938747046314F702EF822FF3797132855D
:109B00003284EFF04FE62AC62285EFF02FE7B24508
:109B10002808EFF07F8945616F806FF3828097C7D7
:109B2000FF1F9387E73A9C43D847A1679387870233
:109B30006316F702EF826FEF797132853284EFF0AE
:109B40008FE22AC62285EFF00FE2B2452300A10280
:109B50002808EFF07F8545616F806FEF8280EF828C
:109B6000CFEC0111EFF02FE0AA852800EFF0DF83A2
:109B700005616F80CFED97C7FF1F938767359C43C3
:109B8000D847A167D1076319F700EF820FEA328542
:109B9000EFF0FFFC6F80AFEB828097C7FF1F9387CA
:109BA00027339C43D847A167C5076319F700EF82A5
:109BB000CFE73285EFF0BFFA6F806FE9828097C7F9
:109BC000FF1F9387E7309C43D847A167B907631904
:109BD000F700EF828FE53285EFF07FF86F802FE797
:109BE000828097C7FF1F9387A72E9C43D847A16702
:109BF000AD076319F700EF824FE33285EFF03FF6D0
:109C00006F80EFE4828097C7FF1F9387672C9C4388
:109C1000D84789476310F702EF822FE1011132859F
:109C200032C8EFF04FD4AA852800EFF0EFF70561B6
:109C30006F80EFE1828097C7FF1F938767299C435E
:109C4000D847A1678D076317F702EF820FDE011176
:109C500032853284EFF02FD113066100AA844C00C4
:109C60002285EF20D00C2800A685EFF0EFF30561E8
:109C70006F80EFDD828097C7FF1F9387A7259C43E6
:109C800081CBDC4391C7EF824FDA82976F802FDC64
:109C90008280EF828FD979713C08AE843ED2A16573
:109CA000B7070A002A843ED448103C08DD053ED69A
:109CB00036C432C63AC2EFD0BFAA12474810BA859E
:109CC000EFF00FC032464810B285EFF0AFC0A246A9
:109CD0004810B685EFF0CFBE501001478146A685EB
:109CE0002285EFD07FC845616F806FD6EF82EFD3BA
:109CF00001117C000329C501AE843ECAA165B707E6
:109D000007002A843ECC48087C00C5053ECEEFD033
:109D10003FA58345D9004808EFF08FBA50080147A6
:109D20008146A6852285EFD03FC405616F802FD282
:109D3000EF82AFCF83C7950093F7F707A384F500B1
:109D4000EFF0DFFA6F80AFD0EF822FCE79713C0851
:109D5000AE843ED2A165B70709002A843ED44810DC
:109D60003C08938545043ED632C636C4EFD05F9F8B
:109D7000A2464810B685EFF0AFB432464810B2851F
:109D8000EFF04FB5501001478146A6852285EFD0F0
:109D9000BFBD45616F80AFCBEF822FC983C79500F0
:109DA00041112A8493F7F707A384F50032852EC664
:109DB000EFF0CFBC85672AC4637CF500EF50B0405C
:109DC0002246B24509E9114781462285EFF07FEC32
:109DD00041016F80CFC701478346F501FDB7EF8290
:109DE0002FC301113C003ECAB7070A003ECC3C001D
:109DF0003ECE83C79500AA89328593F7F707A384DF
:109E0000F5002E84EFF08FB785676371F504A165C7
:109E1000AA84938585044808EFD09F942685EF5047
:109E2000903A2A891DE591454808EFF06FA9A6856B
:109E30004808EFF02FAACA854808EFF06FA801473D
:109E400081465008A2854E85EFD01FB205616F8014
:109E50006FBF81454808EFF0AFA603490902C1BFB3
:109E6000EF820FBB79711C103ECAB7070F003ECCC2
:109E7000404D1C10AA84AE894808994532C63689DF
:109E80003ECEEFD0FF8D32464808B285EFF04FA3AB
:109E900063040902A5454808EFF00F9E2546CA85D0
:109EA000EFF0E019500801478146CE852685EFD0B6
:109EB000BFAB45616F800FB98355C4024808EFF00E
:109EC0006FA10355E402814515C185478545630FA0
:109ED000F500C167FD179305F00F6309F5007D15C7
:109EE000EF5020749305150093F5F50F4808EFF037
:109EF0002F9D834504034808EFF08F9C834514038E
:109F00004808EFF0EF9B835524034808EFF08F9C3F
:109F1000835544034808EFF0EF9B69B7EF82EFB039
:109F200083C795008146014693F7F707A384F500A0
:109F3000EFF01FF36F80AFB1EF822FAF79713E84E6
:109F40001C103ECA2E89B7070F00A1653ECCFD0547
:109F50001C10AA84480842C03AC23ECE36C432C65B
:109F6000EFD01F8032464808B285EFF06F95A246C9
:109F70004808B685EFF00F9612474808BA85EFF00B
:109F80006F9502486304080291454808EFF0CF8EB0
:109F90001146A285EFF0A00A500801478146CA8504
:109FA0002685EFD07F9C45616F806FAA8945480860
:109FB000EFF08F8C834704002300F50083471400E3
:109FC000A300F500D1BFEF82AFA483C795000111B4
:109FD0002A8A93F7F707A384F5003285AE8432C648
:109FE000EFF0CF9932462A893285EFF0CF97856717
:109FF000637FF900AA894A85EF50F01C2A8419E989
:10A00000114781464A86A6855285EFF09FC80561B3
:10A010006F804FA39387E9FF93F7F70F0547E36836
:10A02000F7FE8347F50195E78947E382F9FE83460A
:10A03000F401528501474A86A685EFF09FC5A167C6
:10A04000D90748083ECC230A010002CEEFF0BFC278
:10A050007DBF639CE7008947639CF900930710204C
:10A06000231FF500EF50901AD9B70947E391E7FC99
:10A070008D47E39EF9FA2285EF50D03B97C7FF1F2B
:10A08000938747049C4399E797C7FF1F938747ED42
:10A090009C4389C703D50400EF60300C231F0400E4
:10A0A0002285C9B7EF826F9801113C003ECAB707FD
:10A0B0000B003ECC3C003ECE83C795002A893285FA
:10A0C00093F7F707A384F500AE84EFF02F8B931777
:10A0D0000501C187635EF004A1652A849385E502CA
:10A0E0004808EFD0EFE7A2854808EFE0BFFE97C72A
:10A0F000FF1F9387E7E69C439DEF01449375F40FA0
:10A100004808EFE0FFFB9355844093F5F50F4808AE
:10A11000EFE01FFB9355044193F5F50F4808EFE07E
:10A120003FFA014781465008A6854A85EFD0DF8374
:10A1300005616F80CF91416585460546A2857D15F5
:10A14000EF3070675DD95105EFD04027130440060A
:10A150003344850265B7EF824F8D0111B7070600C2
:10A160003EC683C7950021642A8993F7F707A38425
:10A17000F500AE8428009305A4040AC40AC8EFD0F1
:10A180002FDE300001478146A6854A85EFD0CFFDFE
:10A19000EFE02FF813049404480822CC230A0100AE
:10A1A00002CEEFF05FAD05616F806F8AEF824F8660
:10A1B000C1642A89014497C9FF1F938929F2130AB0
:10A1C0008002FD14EFE0AFAB6345A40001456F8052
:10A1D0006F87B307440303A7C90ABA9703D70700D9
:10A1E0006306970083D72700638427010504D9BF3E
:10A1F0000545F1BFEF82CF812A8A2E8999C123A01C
:10A2000005008149814497CAFF1F938AEACC614BBC
:10A21000EFE02FAD63C5A4004E856F80AF8233841D
:10A22000640383A70A003E948357040099E76304FC
:10A230000900232089008504E1BF4146D28513052A
:10A240004400EFE0705D65F9A289F5B7EF725FFC3D
:10A2500039717C083ED4B7070A003ED67C083ED848
:10A2600083C795002A8A328593F7F707A384F50000
:10A270002E8932C6EFE09FF085676373F50632469C
:10A28000AA843285EFE03FEE8547AA8963EAA704F6
:10A29000A165938585042810EFD08FCC2685EF50DB
:10A2A00080722A8429E191452810EFE07FE1A6859C
:10A2B0002810EFE03FE2CE852810EFE07FE0014775
:10A2C00081463010CA855285EFD00FEAA167938787
:10A2D000770448183EDC230A010202DEEFF0BF9942
:10A2E00021616F703FF681452810EFE07FDDA68584
:10A2F0002810EFE03FDE97C7FF1F9387E7149C43CA
:10A3000091C7228563870900EFB0600C8345040282
:10A3100065B7EFB0200BDDBFEF729FEF83C79500ED
:10A320004111AA8993F7F707A384F5003285AE841B
:10A33000328AEFE0BFE48567637BF5022A89EF503C
:10A3400080682A84914621C18347F50105476383CC
:10A35000E70291C70D47636EF702AD462DA0930546
:10A36000050303250A004146EFE0104B1DE14101C2
:10A370006F705FED9305950803250A004146EFE0F5
:10A38000B049814679F94A86A6854E85EFF0DF9B74
:10A39000F9BF83250A0013059408EF60600119C115
:10A3A000C146D5B797C7FF1F9387C7D19C4399E78D
:10A3B00097C7FF1F9387C7BA9C4389C72285EF6061
:10A3C000A05479FD8547A30FF4002285EF80B05D8E
:10A3D0002285EF50A0634E8581464A86A685EFF020
:10A3E000BF96A1679387570448003EC4230201002B
:10A3F00002C6EFF05F88A5BFEF72BFE083C795008C
:10A400004111AA8993F7F707A384F50032852E89B5
:10A41000B28AEFE0BFD685676370F50CAA84EF506F
:10A42000805A2A841DE9416B014A97CBFF1F938B09
:10A43000EBCA130C400E7D1B19A833048A0383A7B3
:10A440000B0B3E948357C401638D6703050AEFE04D
:10A450000F82E344AAFE954639A88357C50163924B
:10A4600097029305050303A50A004146EFE0D03AA1
:10A47000994611E181462686CA854E85EFF0DF8C2C
:10A48000A1A883A50A0013050403EF507072C1460A
:10A490007DF12285231E9400EF80F0502285EF503D
:10A4A000E05697C7FF1F938727FA9C438DCB230065
:10A4B00004022285EFA090614E8581462686CA85DA
:10A4C000EFF09F88A1679387070448003EC42302EA
:10A4D000010002C6EFF02FFA41016F701FD68947C5
:10A4E0002300F402D1BF397106DE22DC4AD8800095
:10A4F00052D456D25AD026DA4ED65ECE2E8A328921
:10A500002A8BEFD0DFF30605710541998A8A330162
:10A51000A140232224FC231404FCEFD05FF28347E4
:10A520009A000605350593F7F7072315A4FCA30445
:10A53000FA004A85232624FCEFE05FC49317050147
:10A54000C1876340F0025681130104FCF25062544B
:10A55000D2544259B259225A925A025BF24B2161AB
:10A560008280AA844A85EFE07FC1AA894A85EFE00C
:10A57000FFC0A1659385C5022A89130544FCEFD06D
:10A580002F9E2685EFD0AF93854501C94A86CE859B
:10A59000EFD06F8DAA8B15ED8945130544FCEFE0D4
:10A5A0003FB2A685130544FCEFE0DFB2CE8513056C
:10A5B00044FCEFE03FB2CA85130544FCEFE09FB1D5
:10A5C00001478146130644FCD2855A85EFD0CFB9A6
:10A5D0009DBF8145130544FCEFE09FAEA6851305A2
:10A5E00044FCEFE03FAFCE85130544FCEFE09FAEA7
:10A5F000CA85130544FCEFE0FFAD8144EFD03FE492
:10A60000E3D0A4FC83A70B0113971400BA9783D55A
:10A61000070089C5130544FCEFE0DFAB8504F9BFF3
:10A62000797106D622D44AD000184ECE52CC56CAE2
:10A6300026D25AC8AE893289AA8AEFD05FE00605D1
:10A64000690541990A8A3301A140232A24FC231C6D
:10A6500004FCEFD0DFDE83C7990006052D0593F7D4
:10A66000F707231DA4FCA384F9004A85232E24FCAC
:10A67000EFE0DFB093170501C187634FF00052810F
:10A68000130104FDB250225492540259F249624A15
:10A69000D24A424B45618280AA844A85EFE01FAED0
:10A6A000A1659385A5022A89130544FDEFD04F8B40
:10A6B0002685EFD0CF80854519C5CA85EFC0BFFD7F
:10A6C0002A8B0DE98945130544FDEFE07F9FA685A0
:10A6D000130544FDEFE01FA0CA85130544FDEFE01C
:10A6E0007F9F01478146130644FDCE855685EFD0F6
:10A6F000AFA771B78145130544FDEFE07F9CA685A8
:10A70000130544FDEFE01F9DCA85130544FDEFE0EE
:10A710007F9C8144EFD0BFD2E3D5A4FC83270B01FB
:10A7200013971400BA9783D5070089C5130544FD14
:10A73000EFE05F9A8504F9BFEF723FAF83474500B2
:10A74000404DD5E7FD574DC0834694000947636DE2
:10A75000D7080346B400854663E8C6088306E400CC
:10A7600063C406085C45F9562390D70097B7FF1FCE
:10A7700083C7C77699E3A304E40097B7FF1F9387C5
:10A78000277E9C4381E78947A306F40097C7FF1FF4
:10A79000938787CB9C4381E789472306F40097057D
:10A7A000000093854505AA8413050401EFC0703F9E
:10A7B000FD57231AF40281471CDC014897B7FF1F9D
:10A7C00023AA877097B7FF1F93870771232E04036F
:10A7D00004C08043EFD0FFD061463306C5028145F7
:10A7E0002285EF709FA781473E856F705FA6FD575A
:10A7F000E5BFEF729FA32A8403554502EF50A01CCA
:10A8000009E5231E04006F709FA48357E401E5DF70
:10A81000930504FF1715010013050577EFB01063CA
:10A82000DDB7EF729FA02E89A16541119385E503E5
:10A830002A8436C432C6BE843AC2EFC07FF21247C1
:10A840002285BA85EFE0DF8732462285B285EFE0C8
:10A850007F88A2462285B685EFE0DF87630D090079
:10A8600091452285EFE05F811146A685EFE0207DCE
:10A8700041016F70DF9D89452285EFE0EFFF83C7BF
:10A8800004002300F50083C71400A300F500CDB732
:10A89000EF72BF9983C79500444D054793F7F707BB
:10A8A000A384F5001C42411183C70700636DF704C0
:10A8B0002E842A8985CC03C7D4006309F70217B711
:10A8C000FF1F1307E769184301CFA386F400EF8049
:10A8D000902B83C7D40089E741657D15EF30407523
:10A8E00083D72403918B99C3EFB0B0624A85A285C8
:10A8F000EFF0CFBFA167C10748003EC423020100AB
:10A9000002C6EFF04FB741016F707F94EF72FF9175
:10A9100003D745008D47AA8441112E8432892E85A4
:10A9200063EDE700EFE09F85AA85230009002685F7
:10A93000EFC07FD641016F709F91EFE03F842AC640
:10A940002285EFE0BF83B24585472A862300F900C0
:10A950002685EFC05FD1F9BF397106DE22DC26DA29
:10A9600080004ED652D456D24AD85AD05ECEAE8946
:10A97000B284AA8AEFD0BFAB060513052502419920
:10A980000A8A3301A140232224FC231404FCEFD0C3
:10A990001FAA83C7990006054D0593F7F7072315EE
:10A9A000A4FCA384F9002685232624FCEFE00FFDF8
:10A9B00093170501C1876340F0025281130104FC23
:10A9C000F2506254D2544259B259225A925A025BFE
:10A9D000F24B21618280AA8B03AB0400EFC03FCE13
:10A9E00035E983D7440001498544F11793B717002F
:10A9F000A301F4FC834734FCA165BDC79385E5043E
:10AA0000130544FCEFC0DFD5A685130544FCEFE039
:10AA10002FEBDE85130544FCEFE0CFEB834734FCDE
:10AA2000114691E30946DA85130544FCEFE06FE730
:10AA3000814463080900416B7D1BEFD05F9F63C8B1
:10AA4000A40201478146130644FCCE855685EFC01B
:10AA5000BFF1A5B7A685130634FCEFF03FEB9334A6
:10AA600015002A89860479B79385C50451BF8327C9
:10AA7000C90013971400BA9783D507006386650150
:10AA8000130544FCEFE00FE5850445BFEF726FF757
:10AA900079711C103EC4B7070F003EC61C103EC89B
:10AAA00083C79500AA8A328593F7F707A384F50038
:10AAB000AE893284EFE08FEC93170501C1876350B4
:10AAC000F0062A8A2285EFE06FEB2A895285032B54
:10AAD0000400EFC0DFBE39E58357440081440544DC
:10AAE000F11793B71700A303F10083457100DA87CC
:10AAF0002287CA8652862800EFF0BFD201478146DE
:10AB00003000CE855685EFC03FE6A1679387D70317
:10AB100048083ECC230A810026CEEFF0CF95456150
:10AB20006F70AFF1A28513067100EFF03FDEAA84CB
:10AB3000094445DD3544E30A55FB4A85EFF00FE74C
:10AB40000D4445D50144EFD09F8E634BA400C16BEB
:10AB50000144FD1BEFD0BF8D634EA400154471B7B7
:10AB6000DC4413171400BA9783D7070063812703C7
:10AB70000504D1BFD84493171400BA9703D7070030
:10AB800063197701239027012685EF80C054014483
:10AB9000A9BF0504C1B7EF72AFE783C795004111A4
:10ABA0002A8A93F7F707A384F50032852E89328429
:10ABB000EFE0CFDC93170501C187635BF004AA893E
:10ABC0002285EFE0AFDB2311A1004E85832A04002C
:10ABD000EFC0FFAE29E18357440085440144F117DB
:10ABE00093B71700A300F100034811000357210099
:10ABF000D6875285CE862686CA85EFF0EFB3A16749
:10AC0000F10748003EC42302910022C6EFF0AF8650
:10AC100041016F702FE3A28513061100EFF01FCFE3
:10AC20002A84894471D18357210011678544BA97DA
:10AC3000C2071167C1831307F7EFE367F7FA97B706
:10AC4000FF1F938727489C4391C785451305210023
:10AC5000EF40300E8355210022858144EFC09F9D37
:10AC600041D5231005002285EF808048B5BFEF72E3
:10AC70004FD983C7950041112A8B93F7F707A38417
:10AC8000F50032852E8A3284EFE04FCF931705010D
:10AC9000C1876359F004AA8A2285EFE02FCE2A8962
:10ACA0005685832B0400EFC09FA121E18357440008
:10ACB00081440544F11793B71700A301F10003483D
:10ACC0003100DE875A854A87D6862286D285EFF004
:10ACD000AFA6A167ED0748003EC42302810026C647
:10ACE000EFE07FF941016F704FD5A2851306310067
:10ACF000EFF0DFC1AA84094479D19167CA97C207EE
:10AD00001167C1831307F7EF0544E36AF7FACA85B1
:10AD1000EFC05F92014445F58149EFD04FF263DB0C
:10AD2000A900984893971900BA9703D7070015E729
:10AD300023902701EFD0AFF01544E382A9F82685D0
:10AD4000EF80003B97B7FF1F9387C7379C430144B1
:10AD5000BDD74A85EF4040769DB785097DBFEF722C
:10AD60002FCB79713E847C083EC82E8AB707140029
:10AD7000A1653ECAE5057C08AA89080836C442894F
:10AD800032C6BA8AC6843ECCEFC09F9DCA850808E9
:10AD9000EFE00FB332460808B285EFE0AFB3A2464A
:10ADA000630E09029D450808EFE00FAD1D46814581
:10ADB000EF70AFCA63870A0691450808EFE0CFAB92
:10ADC0001146A685EFE0A027100801478146D285ED
:10ADD0004E85EFC07FB945616F70CFC6B685080854
:10ADE000EFE04FAF1C400808D8439355C701858951
:10ADF00012075183B205D98DEFE0CFAD1C40080892
:10AE000083C58700EFE0CFAB1C40080883C5A700CF
:10AE1000EFE00FAB1C40080883C59700EFE04FAA96
:10AE200051BF89450808EFE02FA583C70400230020
:10AE3000F50083C71400A300F50079B7EF724FBD8A
:10AE400083C795004111AA8993F7F707A384F500FA
:10AE50003285AE843284EFE06FB293170501C1876B
:10AE60006357F0042A89032A0400EFC05F8519E9BB
:10AE7000835744000548F11793B71700A307F10063
:10AE8000814621A81306F100A285EFF03FA81DC15D
:10AE90001C459DC383D6470001480347F100930733
:10AEA0008500D2884A86A6854E85EFF05FEB41018A
:10AEB0006F704FB90948E9B71D48D9B7EF724FB560
:10AEC00065715C083EC4B7077B013EC65C083EC89E
:10AED00083C795002A8A328593F7F707A384F50084
:10AEE000AE89EFE04FA88357E100C5C3894528002C
:10AEF000EFC01F8781452800EFE08F9CEFC0FF8BDC
:10AF000097B7FF1F938747549C4317B4FF1F034411
:10AF1000E4FCAA843334800099C31364240097B7F7
:10AF2000FF1F9387E7039C4399C31364440097B7BB
:10AF3000FF1F938727199C4399C31364840083D50B
:10AF4000040028000149EFE0EF9883D52400280091
:10AF5000EFE04F9883D544002800EFE0AF97EFD0A3
:10AF60000FC993150501C1812800EFE0AF96A285B6
:10AF70002800EFE02F969C44636CF900014781465E
:10AF80003000CE855285EFC03F9E59616F708FAB08
:10AF9000DC441314490028003E94EFE06F8C834793
:10AFA00044000347540089070607BA978607E36EF3
:10AFB000F5FC835524002800814AEFE0AF918345DA
:10AFC00044002800EFE0CF8F834554002800EFE0D5
:10AFD0002F8F8347440063C9FA00814A8347540096
:10AFE00063CFFA00050941BF1C4413975A0028009B
:10AFF000BA9783D50700850AEFE0CF8DD9BF032B21
:10B00000C40093975A0028003E9B83552B00850A65
:10B01000EFE04F8C83550B002800EFE0AF8B7DBF36
:10B02000EF72AFA05C4993E717005CC9EF80203353
:10B030006F70EFA1EF726F9F2E848145EFF08F9BB1
:10B0400005C183570500FD172310F50009C4835778
:10B0500025002310F400EFF0BFFC01456F702F9F17
:10B0600031456DDC23100400D5BFEF726F9A83C7A2
:10B07000950041112A8A93F7F707A384F5003285DA
:10B080002E893284EFE08F8F93170501C187635EAD
:10B09000F004AA89C1452285EFD0BFFA2A8B4E85DC
:10B0A000832A0400EFC0AFE121E583574400231158
:10B0B00001000544F11793B71700A300F100814484
:10B0C0000348110003572100D6875285CE86228679
:10B0D000CA85EFE07FE6A1679387170248003EC468
:10B0E0002302810026C6EFE01FB941016F708F95E2
:10B0F00013061100A285EFF07F81AA8409E52311D0
:10B100000100094475BF930521005A85EFF09FF2B5
:10B11000835721002A84CDD797B7FF1F938787FADB
:10B120009C4391C7854513052100EF40804083551E
:10B13000210026853144EFC0EFCF59D123100500FF
:10B140002685EF70F07A0144A5BFEF720F8E411192
:10B150002E896C00AA8402C6EFF0CF8909CD03576F
:10B16000050005072310E500EFF09FEB81473E85C2
:10B1700041016F70CF8D3247954775DBCA852685B3
:10B18000EF20D008C147E34405FE324485474146DD
:10B190002310F40083570900A685130544002311EA
:10B1A000F400EFD0D0692285C1B7EF726F8683C7F4
:10B1B00095004111AA8A93F7F707A384F500328519
:10B1C000AE893284EFD09FFB93170501C187635E80
:10B1D000F0042A8AC1452285EFD0BFE6AA845285B1
:10B1E000032B0400EFC0AFCD21E5835744002311AA
:10B1F00001008544F11793B71700A300F100014443
:10B200000348110003572100DA875685D286268627
:10B21000CE85EFE07FD2A1679387070248003EC446
:10B220002302910022C6EFE01FA541016F708F81BC
:10B23000A28513061100EFF06FED2A8409E52311B2
:10B240000100894475BF268593052100EFF0FFEFCB
:10B25000AA845DF5835521002285EFC0AFBD4DF175
:10B260000149EFD0CF9D635DA900184893171900DD
:10B27000BA9703D707001DE7035721002390E70083
:10B28000EFD0EF9B6302250397B7FF1F938787E3F8
:10B290009C4389C703552100EF4000222285EF70AF
:10B2A0003065B9BF050975BF954499BF05C19307BE
:10B2B000F00F630FF500C547630CF5009307F5FF2A
:10B2C00005453315F50042054181828001458280A4
:10B2D00041657D158280B9E1EF623FF503450603C4
:10B2E0003284EFF0BFFC9305803EB305B502C20582
:10B2F000C18191C90357E402854763F6E70013054E
:10B300000401EFC020168357E40241677D1763856F
:10B31000E700FD172317F4026F607FF38280EF626E
:10B320005FEE004283C79500444D0349140093F734
:10B33000F707A384F50083470400220911673369E6
:10B34000F900A167B347F90041112A8BAE8A63EC7B
:10B35000E70C834724001307C00EB91793F7F70FC4
:10B360006371F70E03473400C14763ECE70C834772
:10B3700044001307E00793C707086373F70A83497C
:10B38000840083477400A209B3E9F900856763F973
:10B39000F908034A6400834754004E85220A336A41
:10B3A000FA00EF40406245C123962403834B3400EA
:10B3B000137AFA00239A34032388740323994403ED
:10B3C00093890401631A090023A604022398040246
:10B3D0004E85EFC0A00A1DA0034924004A85EFF066
:10B3E000FFEC2397A402834744004E85A388F40210
:10B3F000E3810BFEE30F09FCEFC06005EF7090796D
:10B4000081460146D6855A85EFE09FA5A1679387BF
:10B4100097033EC423020100480002C6EFE0BF8547
:10B4200041016F609FE18544A2862686D6855A85B4
:10B43000EFE01FA3A167938797033EC42302910007
:10B44000E1BFBD44D5B79144C5B7EF627FDC0111C0
:10B450001C08404D3EC2B7070F003EC41C083EC644
:10B460002A89AE89EFC01F9D585C1C5C634CB70AEB
:10B470006394E50063E8A70A3385A740B3B7A70044
:10B48000B305B7401306803E81469D8DEFD0407BCB
:10B4900093140501C180A1659385C5034800EFC0E1
:10B4A0002FAC81454800EFD0BFC18355040448004C
:10B4B000EFD05FC2835524044800EFD0BFC181455F
:10B4C00099C8C167FD179305F00F6386F4002685C0
:10B4D000EF402015AA854800EFD09FBE03554404D5
:10B4E000814511C9C167FD179305F00F6305F5008C
:10B4F000EF402013AA854800EFD09FBC8345640429
:10B500004800EFD0FFBB834574044800EFD05FBB19
:10B51000500001478146CE854A85EFC0EFC40561E2
:10B520006F605FD2814485BFEF623FD083C79500D3
:10B5300093F7F707A384F500EFF03FF16F603FD179
:10B54000EF621FCD83C795004111404D93F7F70778
:10B55000A384F5002A8A3285B284AE89EFD01FC257
:10B560002A8B2685EFD09FC12A892685EFD0BFBFC1
:10B5700093170B0163CA0702E177CA97C207C18319
:10B58000116763E3E70293070910C207C18313073A
:10B59000B00F637BF70093170901C187AA8A63483C
:10B5A000F000C54763FA570141016F60BFC9EFC0A2
:10B5B0008F83E31B25FFF5B763060B0263040902C3
:10B5C000814463870A02B7077F00231064052311B3
:10B5D00024057CC05685EFF07FCD9304803EB304F4
:10B5E000950239A0B7077F00232004047CC0814462
:10B5F00003552404EFB0101095CCEFC0BF832695FF
:10B6000093D7F44133379500AE97BA9708DC5CDCEA
:10B61000CE855285EFF07FE399E023220404A167F1
:10B620009387B70348003EC42302010002C6EFE03F
:10B630008FE49DBF814701481CDC232E0403C9BF52
:10B64000EF62BFBEEFC0FFE9E1473305F502914568
:10B65000EF30507FE55711C597B7FF1F23AEA78680
:10B6600081473E856F60BFBE854717B7FF1F230721
:10B67000F7868280EF627FBB97B7FF1F938787852E
:10B6800080432DC083570404639EA704835724047A
:10B69000639AB7043689B284EFC0CFF95C5C63C3A8
:10B6A000B7046395B7001C5C63EEA702834764048C
:10B6B00063F3F400A6872303F4048347740463F35D
:10B6C0009700A687A303F4048357440441677D17BA
:10B6D0006385E70085072312F4043C4481C7CA85CB
:10B6E000268582976F60BFB697A7FF1F9387877ED7
:10B6F0009C43014599C303C587008280EF62FFB276
:10B700000111B70707003EC683C79500584D0AC40C
:10B7100093F7F7070AC8A384F5002A89AE8401CB02
:10B720001C4283C707002304F700EF70D045216453
:10B73000930554022800EFC0AF82EFF0FFFAAA850C
:10B740002800EFD0FF97300001478146A6854A8543
:10B75000EFC08FA113044402480822CC230A010041
:10B7600002CEEFE04FD105616F607FAEEF62FFABBD
:10B7700001117C003ECAB70707003ECC7C003ECEDC
:10B7800083C795002E84AA8493F7F707A384F50056
:10B79000A165938555024808EFB09FFCEFF0DFF4F8
:10B7A000AA854808EFD0DF91500801478146A2855D
:10B7B0002685EFC06F9B05616F607FA997A7FF1F6C
:10B7C000938747719C43094599C303C597008280BD
:10B7D00097A7FF1F938707709C43094599C303C52B
:10B7E000D700828097A7FF1F9387C76E9C430145B0
:10B7F00099C303C5A7008280EF629FA10111B7071B
:10B8000008003EC683C79500404D0AC493F7F7076A
:10B810000AC8A384F5002A89AE8429C0144285474A
:10B8200003C7060063EEE706834794000946814993
:10B83000638EC700B307F740A304E400B339F000F8
:10B8400083C716002305F400EF70F0330357240379
:10B85000058B09C763840900EFA0B06B21649305D1
:10B8600084022800EFB0DFEFEFF05FF5AA85280033
:10B87000EFD01F85EFF01FF7AA852800EFD05F8477
:10B88000014781463000A6854A85EFC0EF8D13043D
:10B890007402480822CC230A010002CEEFE0AFBDBB
:10B8A00005616F603F9AEF625F9801117C003ECAAC
:10B8B000B70708003ECC7C003ECE83C795002E849F
:10B8C000AA8493F7F707A384F500A1659385850201
:10B8D0004808EFB0FFE8EFF07FEEAA854808EFD008
:10B8E0002FFEEFF03FF0AA854808EFD06FFD50081B
:10B8F00001478146A2852685EFC00F8705616F60ED
:10B900001F9597A7FF1F9387E75C9C43014599C349
:10B9100003C5B7008280EF625F910111B70707008E
:10B920003EC683C79500404D0AC493F7F7070AC87F
:10B93000A384F5002A89AE8405C41C42054783C749
:10B940000700636AF7040347B400630BF700A3051D
:10B95000F400EF7050238347B400A9C3EFD00FD990
:10B9600021649305B4002800EFB09FDFEFF07FF96A
:10B97000AA852800EFD0CFF4014781463000A68584
:10B980004A85EFB07FFE2904480822CC230A010033
:10B9900002CEEFE04FAE05616F607F8BEFD02FDA04
:10B9A000C1B7EF629F8801117C003ECAB70707004C
:10B9B0003ECC7C003ECE83C795002E84AA8493F7AC
:10B9C000F707A384F500A165AD054808EFB05FD97E
:10B9D000EFF03FF3AA854808EFD08FEE50080147FB
:10B9E0008146A2852685EFB03FF805616F603F86EE
:10B9F00097A7FF1F9387074E9C43094599C303C52B
:10BA0000C7008280EF627F8201117C00AE843ECA53
:10BA1000A165B70707002A843ECCD1057C00480801
:10BA20003ECEEFB0FFD3EFF0BFFCAA854808EFD0C1
:10BA30002FE9500801478146A6852285EFB0DFF245
:10BA400005616F60DF80EF624FFE83C7950093F75B
:10BA5000F707A384F500EFF0FFFA6F604FFFEF6286
:10BA60002FFB83C795000329C501411193F7F70701
:10BA7000A384F5001C4283C90700854763EC3705A2
:10BA800097B7FF1F9387479C9C432E84AA8495C732
:10BA9000EFF01FF689476302F5026300090283474E
:10BAA000C900638C370123063901EF70D00D83572D
:10BAB0002903898B99C3EFA0D0452685A285EFF095
:10BAC0007FF4A167CD0748003EC42302010002C6EF
:10BAD000EFE06F9A41016F60EFF697A7FF1F938722
:10BAE000673F9C431D4599C303C5E7008280EF6211
:10BAF000CFF30111B70707003EC683C79500584D25
:10BB00000AC493F7F7070AC8A384F5002A89AE840C
:10BB100005C71C4283C7070093968701E18663C867
:10BB2000060485466385D7048346E7006386F600EE
:10BB30002307F700EF70300521649305E400280027
:10BB4000EFB01FC2EFF07FF9AA852800EFD04FD7E2
:10BB5000014781463000A6854A85EFB0FFE03504F5
:10BB6000480822CC230A010002CEEFE0CF90056105
:10BB70006F60EFEDEF626FEB01117C003ECAB7071B
:10BB800007003ECC7C003ECE83C795002E84AA845D
:10BB900093F7F707A384F500A165B9054808EFB04E
:10BBA0003FBCEFF09FF3AA854808EFD06FD1500853
:10BBB00001478146A2852685EFB01FDB05616F60D6
:10BBC0000FE9EF62EFE4AA84014417A9FF1F1309EC
:10BBD000A930E149EFC0FF906344A400014519A8D2
:10BBE00033053403832709003E9583572500639569
:10BBF000970011056F600FE50504E9BF032E85006E
:10BC000063040E1017A3FF1F1303C34B032303008A
:10BC1000631503002943639A060E03234E0163153F
:10BC200003001D436393070EEF62AFDDC689428AAE
:10BC30003E89BA8AB684328BAE8B2A84A1E9035539
:10BC40004E0009E501431A856F602FDFA167A98FB8
:10BC5000116763F7E700EFF0DFF68145EFF08FBD86
:10BC60000844B70700E05841F98F18455CC1B70791
:10BC7000001FF98F1CC55C4981C76105EFB010003A
:10BC8000E38209FC2285EF70606E6DBF3285EFA004
:10BC9000E0620D434DD91C44116703D54700A167ED
:10BCA000A98F63F7E700EFF0DFF18145EFF08FB880
:10BCB0000323840093164B01D1828347B3000356BC
:10BCC00063008588FD8BA305F300FD777D8E558E7F
:10BCD000FD76FD16B204F18E83274301C58E231233
:10BCE00073012313D3002304530123052301A30469
:10BCF0004301D9D72285EFB07FBBAA850844B5DDC3
:10BD00006105EFB02076ADBF1D431A858280EF62DA
:10BD10002FD00569AA84AE89328A0144FD5A7D1963
:10BD2000EFC0EFF06345A40001456F60AFD1D84488
:10BD300093171400BA9703D70700631B37032390A8
:10BD4000570163050A002685EF70E0389C448DC3D7
:10BD500083D76700B3F72701639C3701D288014876
:10BD6000814701478146014681452685EFF01FE95D
:10BD700005047DB7EF62CFC979711C103EC4B707C7
:10BD80000F003EC61C103EC883C79500AA8A3285A4
:10BD900093F7F707A384F5002E893284EFD00FBE06
:10BDA00093170501C1876350F006AA892285EFD059
:10BDB000EFBC2A8A4E85032B0400EFB05F9039E573
:10BDC0008357440081440544F11793B71700A30338
:10BDD000F10083457100DA872287D2864E862800DB
:10BDE000EFE03FA4014781463000CA855685EFB099
:10BDF000BFB7A1679387F70348083ECC230A8100A9
:10BE000026CEEFD05FE745616F60CFC3A2851306F2
:10BE10007100EFE0BFAFAA84094445DD5285EFE031
:10BE2000EFB80D445DD50546D2852685EFF03FEE8F
:10BE30002A8445B7EF626FBF83550700034627008A
:10BE400041112A842E8532C62EC4EFE02FB611C5CB
:10BE50003246A2452285EFF09FEB41016F602FBF74
:10BE6000EF622FBA83C795004111AA8A93F7F707AB
:10BE7000A384F5003285AE893284EFD02FB09317BA
:10BE80000501C1876357F008C1452A8A2285EFD092
:10BE90004F9B2A8D2285EFD06FAE2A892285EFD065
:10BEA0008FAC930705F893F7F70F1307E007AA8BFA
:10BEB0006371F7062285EFD00FAB2A8C2285EFD075
:10BEC0008FAAAA8C5285032B0400EFB04FFF29E5FF
:10BED00083574400231101008144F11793B71700E1
:10BEE000A300F10005440347110083562100938706
:10BEF00084005685DA8822885286CE85EFE03FE6B8
:10BF0000A167E90748003EC42302810026C6EFD09E
:10BF10009FD641016F606FB213061100A285EFE05A
:10BF2000FF9EAA8409E52311010009446DBF930512
:10BF300021006A85EFF06FA12A8455F58355210011
:10BF40009356C9001316490185486688E2875E87C3
:10BF5000858A51822685EFF07FCA2A8469B7EF620D
:10BF60004FAA83C7950041112A8B93F7F707A38443
:10BF7000F5003285AE893284EFD04FA093170501CA
:10BF8000C1876352F0082A8A2285EFD02F9FAA8AA0
:10BF90002285EFD0AF9E2A892285EFD0CF9C9307D0
:10BFA00005F893F7F70F1307E0072A8C637DF70472
:10BFB0002285EFD04F9BAA8C2285EFD0CF9A2A8D75
:10BFC0005285832B0400EFB08FEF29E183574400A3
:10BFD00085440144F11793B71700A301F10003470B
:10BFE0003100930784005A85DE882688D6865286DB
:10BFF000CE85EFE0DFD68D4748003EC42302910096
:10C0000022C6EFD05FC741016F602FA3A285130640
:10C010003100EFE0BF8F2A84894471D19356C90063
:10C020001316490185486A88E6876287858A5182A6
:10C03000D685EFF0BFBCAA845DB7EF626F9D2A89F9
:10C0400081440144617A916A17ABFF1F130B8B0780
:10C05000EFC0EFBE63C5A40022856F60AF9E83274B
:10C06000090093991400CE9703D5070033074501C3
:10C07000420741836362570311CD03270B0009C7B1
:10C0800085453E85EF30E04A832709000504CE97B9
:10C090002390070085046DBFEFF0BFB2832709002E
:10C0A0000504CE972390070075D58145EFE09FF8F2
:10C0B000D5B7EF62EF9583C7950041112A8A93F7B0
:10C0C000F707A384F50032852E893284EFD00F8BD9
:10C0D00093170501C1876354F004AA89832A0400D9
:10C0E000EFB0EFDD21E18357440085440144F117AF
:10C0F00093B71700A301F10003483100D68752859A
:10C100000147CE862686CA85EFD01FE3A167F507D3
:10C1100048003EC42302910022C6EFD0DFB54101A2
:10C120006F604F92A28513063100EFE02FFE2A8444
:10C13000894479D197A7FF1F9387C7F89C4381CB88
:10C140000449EFC0CFAFAA852685EF30803E1305A6
:10C150000401EFF09FEE2285EF609079814469BF82
:10C16000EF622F8A83C795004111AA8A93F7F707D8
:10C17000A384F5003285AE89328423110100EFC01B
:10C18000FFFF93170501C187635CF0042A8AC1454C
:10C190002285EFC01FEBAA8B5285032B0400EFB062
:10C1A0000FD231E18357440085440144F11793B71E
:10C1B0001700A300F1000348110003572100DA879C
:10C1C0005685D2862686CE85EFD01FD7A167938766
:10C1D000270248003EC42302910022C6EFD0BFA927
:10C1E00041016F608F85A28513061100EFE00FF209
:10C1F0002A84894469D197A7FF1F9387A7EC9843A6
:10C200003E8901CB0449EFC08FA3AA852685EF3074
:10C21000403213050401EFF05FE2EFC04FA29544F6
:10C2200059D9930521005E85EFE03FF2AA8441F5DC
:10C230001C480357210022852390E700EF60506BD4
:10C2400083270900ADDB03552100EF30E026A5B7B9
:10C25000EF523FFB83C795004111AA8A93F7F70776
:10C26000A384F5003285AE893284EFC03FF1931785
:10C270000501C1876359F0042A8A2285EFC01FF0A7
:10C280002A895285032B0400EFB06FC321E1835745
:10C29000440085440144F11793B71700A301F1004E
:10C2A00003483100DA8756854A87D2862686CE85AE
:10C2B000EFD09FC8A167F90748003EC42302910050
:10C2C00022C6EFD05F9B41016F503FF7A285130656
:10C2D0003100EFE0AFE32A84894479D19167CA97AE
:10C2E000C2071167C1831307F7EF8544E36AF7FAC2
:10C2F00097A7FF1F938707DD9843BE8B01CB0449A7
:10C30000EFC0EF93AA852685EF30A0221305040124
:10C31000EFF0BFD2EFC0AF92954459D11C482285AF
:10C32000814423902701EF60B05C83A70B00ADDB55
:10C330004A85EF306018ADB7EF523FEF2A844105D0
:10C34000B284EFF09FCF01C52285EF60705A81461D
:10C350000146A6852285EF70C00B1C4C89C7DC47BF
:10C3600099C3228582976F509FEE97A7FF1F9387EF
:10C3700067B69C43014599C313850701828097A73F
:10C38000FF1F938727B588438280EF521FEA9317D8
:10C39000C600DD8DC2054111C1812A8432C6EFC0BD
:10C3A0007FD33246228511829375F60FEFC05FD19D
:10C3B00041016F50DFE9EF52BFE579713C083ED291
:10C3C000B7070C003ED43C083ED683C79500AE8428
:10C3D0002A8993F7F707A384F500A16593853504AF
:10C3E0004810EFB0EFB7C165FD15014417AAFF1F54
:10C3F000130ACACE930A400EAE892E8B2EC6EFC00A
:10C400000F874205931704014181C183B24563E35D
:10C41000A702C167FD176385F5004810EFC09FCBE9
:10C42000501001478146A6854A85EFB0EFD345619C
:10C430006F505FE13307540383270A0BBA9703D683
:10C44000C70163083601638835014810EFF0FFF338
:10C45000DA85050465B7B285EDBFEF529FDA7971D1
:10C460007C083EC8B70711003ECA7C083ECC83C793
:10C470009500AA89328593F7F707A384F5002E89E2
:10C48000EFC0DFCF8567637EF502A165AA848905C9
:10C490000808EFB0EFAC2685EF30E05213341500FA
:10C4A0000A04A2850808EFC0BFC1A6850808EFC02E
:10C4B0007FC235C0014781461008CA854E85EFB05E
:10C4C000AFCA45616F507FD7B30754030327CA0A29
:10C4D000BA9703D70700631A970003D62700638A29
:10C4E00065030808EFF07FEADE8505042EC6EFB08D
:10C4F0001FF94205931704014181C183B245E3E569
:10C50000A7FCC167FD17E387F5FA0808EFC09FBCD9
:10C5100055B7B285D9BFC165FD15014417AAFF1FE4
:10C52000130ACABB930A80022E8BAE8BC1B7EF529F
:10C53000DFCF18418347170083460700A207D58F36
:10C54000D207D1832390F5008347270003471700C4
:10C550008D45A207D98F91832310F600EFC03FAD20
:10C560006F50FFCEEF52DFCAC164014417A9FF1F0D
:10C570001309C9B693098002FD14EFB05FF063455B
:10C58000A40001456F501FCC330534038327C90A2B
:10C590003E9583570500E38797FE0504F9BFEF52E8
:10C5A0003FC72A8AAE89B284B68AEF30C04109E516
:10C5B00091473E856F501FC92A894E85EF901050D4
:10C5C0002A84638A0A048D476DD503570500C54741
:10C5D000E31147FF0347F9018546AD47E31BD7FC4D
:10C5E0008347450091CB4146A6855D05EFC0D0222B
:10C5F000814761D1AD4775BF130965012302E5008D
:10C60000CA852685EF10202D15CDA547E3830AFAAC
:10C610002302040079BF11CD83570500E39A47F93F
:10C620004146A6851905EFC0301F814759D199476A
:10C6300049B74E85EFF01FF32A8495473DD913097A
:10C6400055007DBF4146A6852310440123113401C6
:10C6500013051900EFC0B01E2285EF60B03C814782
:10C6600089BFEF529FBC79717C003ECCB7070A00AE
:10C670003ECE7C003ED083C79500B2842E8493F7D3
:10C68000F707A384F5001306A1002A892C0026854C
:10C69000EFF0FFE9A16528088D05EFB06F8C9040A1
:10C6A0008355A100035581008546EFF05FEFAA8412
:10C6B000AA852808EFC0DFA00356A100835581009A
:10C6C0002808EFF09FCC300801478146A2854A85B3
:10C6D000EFB08FA9854748103ED42302910202D6BD
:10C6E000EFD06FD945616F509FB6EF521FB479718B
:10C6F0007C003ECCB7070A003ECE7C003ED083C70C
:10C700009500B2842E8493F7F707A384F5001306EF
:10C71000A1002A892C002685EFF07FE1A165280879
:10C720008D05EFB0EF8390408355A1000355810044
:10C730008146EFF0DFE6AA84AA852808EFC05F985B
:10C740000356A100835581002808EFF01FC430086C
:10C7500001478146A2854A85EFB00FA14810230208
:10C76000910202D402D6EFD00FD145616F503FAE97
:10C77000EF52BFABEFF0BFE26F507FAD9797FF1F57
:10C780009387877588438280EF523FAA835725009D
:10C790004111AE842A842307B10017F5FFFF13056A
:10C7A000A5696C002316F100EFB0CFD581C42285B6
:10C7B000EF60B02DFD572310F400130620028145D1
:10C7C00013055400EF507FA941016F505FA8EF524D
:10C7D0003FA479717C003ECCB7070A003ECE7C00B6
:10C7E0003ED083C79500AA89AE8493F7F7073285B8
:10C7F000A384F5001306A1002C00EFF05FD30355CE
:10C8000081001144EF30201C15C10355A1000144E3
:10C81000EF90D02A01CD035705008357810045448E
:10C820006316F7008545EFF03FF601442169930553
:10C8300039002808EFA0DFF2A2852808EFC05F8842
:10C840000356A100835581002808EFF01FB430087B
:10C8500001478146A6854E85EFB00F9148104AD416
:10C860002302810202D6EFD00FC145616F509F9D18
:10C87000EF521F9A9797FF1F9387C7652A848843B3
:10C880002E8915C1035745038357C401631DF70063
:10C8900023260502231805024105EFA0303E63045C
:10C8A0000900EF60302F814497A9FF1F9389098306
:10C8B000130A8002EFB0BFBC63CCA4029797FF1F9E
:10C8C0009387076A9C4389C70355C401EF104076DC
:10C8D000630509002285EF6050031306400E814571
:10C8E0002285EF509F97FD57231EF4006F509F95B0
:10C8F0003385440383A7C90A3E9503570500835730
:10C90000C4016315F700CA85EFF01FE885045DB721
:10C91000EF521F9083C795004111AA8993F7F7073B
:10C92000A384F5003285AE84EFC05F8585676370B0
:10C93000F5042A89EF302009014411C983D7040086
:10C940003144638627018545EFF09FF201444E850F
:10C95000A2864A86A685EFD02FBFA16793871704CA
:10C9600048003EC42302810002C6EFD0CFB041018F
:10C970006F505F8DEF52DF899797FF1F9387875521
:10C9800080431DCC0145EFA0E05681470148C164BA
:10C990001CDC232E0403232004041799FF1F130912
:10C9A000E97301449309400EFD14EFB05FAC634B93
:10C9B000A40081451705000013054598EFB08FB41A
:10C9C0006F505F88330534038327090B3E958357E7
:10C9D000C501638597008545EFF09FE90504F1B730
:10C9E0009357050113D78700A380F500931705011E
:10C9F000C183A1832380E5002381F500A381A500E5
:10CA00008280EF529F822300050083C71500A30098
:10CA1000F50083C725002301F50083C73500A30176
:10CA2000F50083C745002302F50083C75500A30224
:10CA3000F50083C7650093059500A3030500230354
:10CA4000F500230405003285EFF09FF96F503F8019
:10CA5000EF520FFC4111E9541DC995C993F9C5FF67
:10CA60002E842A89AA84338AA900B7EA04006314B1
:10CA70009A020D88854401CCB7E704009C5F829739
:10CA80002AC622866C0033053901EFC0405B26853B
:10CA900041016F502FFB83A78A039104829793175C
:10CAA0000501C183A183A38EF4FE93570501238F53
:10CAB000F4FEA183238EA4FEA38FF4FE4DBF63E09A
:10CAC000D502EF528FF6B28741113686BE8536C643
:10CAD000EFC0E056B246410136856F504FF78146B0
:10CAE00036858280838705001387F5003D05FD8725
:10CAF00093F77708834607007D158606B58FA30058
:10CB0000F5006307B7007D17834717009D83DDB7E6
:10CB10008280EF528FF1B7E7040083A707093287BD
:10CB20002A863A858297133515006F504FF201CD52
:10CB3000814799C9EF526FEF4146EFC0405085479A
:10CB40003E856F50CFF081473E8582801DC5EF52F4
:10CB5000CFED414681452A84EF502FF04146814573
:10CB600013050403EF506FEF0147C167232204044C
:10CB700038C87CC805456F508FED014582808147DC
:10CB800029CDA1CDEF526FEAB2842E89130680051C
:10CB900081452A84EF506FECCA8524C42685EFF0C6
:10CBA0001FF9414681452285EF502FEB3044A28585
:10CBB0002285EFF01FF693040401A2852685EFF08D
:10CBC0007FF2A68513050402EFF0DFF12285EFF076
:10CBD000FFF785473E856F508FE73E858280EF5295
:10CBE0002FE34111E9541DC995C993F9C5FF2E845E
:10CBF0002A89AA84338AA900B7EA0400639444030B
:10CC00000D88814401CCB7E704009C5F82972AC657
:10CC100022866C0033053901EFC060422685410150
:10CC20006F504FE283A78A039104829793170501FF
:10CC3000C183A183A38EF4FE93570501238FF4FED5
:10CC4000A183238EA4FEA38FF4FE4DBF71CDEF52BE
:10CC50002FDCB28401E605456F50CFDE2A842E8991
:10CC60000145FDD93C487848B3E6E700F5D6938600
:10CC7000F7FFB3B7F6007D17032A4404BA9734C808
:10CC80007CC8630F0A04C14913050A03B3894941EB
:10CC90002295637B3601B2862E86A685EFF03FE2B1
:10CCA0007C40BE9464C045BFCE862E86CE85EFF014
:10CCB0001FE1C114D2944E9923220404A287930643
:10CCC000040103C7070003C607038507318FA38F3D
:10CCD000E7FEE398F6FE3044A2852285EFF07FE37D
:10CCE0002699C1493306994063EA9900ADD4A686D6
:10CCF000A68513050403EFF09FDC6DB78147B306EB
:10CD0000F4003307F6000347070083C506008507D4
:10CD10002D8F2380E600E39437FF3044A2852285DF
:10CD2000EFF03FDFC1147DBF0145828019C9EF528A
:10CD3000CFCF130680058145EF502FD205456F50A8
:10CD40000FD10145828081473DC9B5C9EF52EFCD72
:10CD5000FC4141462E84AA846393C70413860501CF
:10CD6000A2878146C14503C7070003C5070385079E
:10CD7000298F3305D600034505008506298FA38F2B
:10CD8000E7FEE392B6FE3044A2852685EFF07FD819
:10CD90002285EFF0BFF985473E856F504FCB138555
:10CDA00007031D8E81452295EF502FCB7C40130742
:10CDB00000F813060402A2972388E70255B73E85C0
:10CDC0008280EF528FC66D712E84B284AA85901036
:10CDD00028003689EFF0BFDA19E9D55705A0504091
:10CDE0000C402800EFF09FE66DD9FD142104E5F812
:10CDF0002C004A85EFF03FF5814765D13E855161B2
:10CE00006F50EFC4EF526FC241112EC432C62C00D6
:10CE10000546EFF01FFB41016F506FC3EF52EFC0AB
:10CE200001112A842EC602C802CA02CC02CEEFC06B
:10CE30006048B2462A86A2850808EFF0BFFC137549
:10CE4000F50F05616F50AFC0EF522FBE7971B287F9
:10CE50002A8421462308B10013051101BE853AC476
:10CE600036C6EFC0C01DB246930591013685EFF07E
:10CE70003FB72285141035460C08EFF0BFF82A841E
:10CE8000224711E521460C103A85EFC0401B228550
:10CE900045616F50CFBBEF524FB97171AE84AA8517
:10CEA0000A853284EFF0BFC801C90A86A6852285AB
:10CEB000EFF03FC6814711E1C5473E854D616F5098
:10CEC0000FB9EF528FB31D712A8AB289BE843546DD
:10CED0008547130511012E8CB68A3A8BC28C468D7C
:10CEE0002308F100EFC0A01510100C085285231F75
:10CEF0000100EFF05FFA2A842DE9A147631BFD06CC
:10CF00009307900591E0E5473546E2851305110149
:10CF100013990A012308F10013590901EFC02012E7
:10CF20001357890093978A00D98F90080C0852856F
:10CF3000231FF100EFF03FF62A8405E9A1E0938773
:10CF4000FA0091831379F9003EC663130900414941
:10CF5000668B8144C14B854DB2476397970C6A86B7
:10CF60008C0033855C01EFC0800D228525616F50F8
:10CF70008FAC93079004C9F8A54779B7834701059B
:10CF80000947C14B2308F10083471105A58FA3086A
:10CF9000F10093872400814463EFFB0201471408EA
:10CFA0003386E6008C08B386E400BA95DA9683C629
:10CFB000060083C505000507AD8E2300D600E3906B
:10CFC000E7FE41476398E70490080C085285EFF0AC
:10CFD0009FEC35D535A8B3069B00BA871008B3057A
:10CFE000F60090083E9603C5060003460600850736
:10CFF0008506298E2380C500E39277FF998F9008DC
:10D000000C085285BE94EFF01FE98947014749D5C6
:10D010002A84A1BF90083E96034606001408BE96D7
:10D020002380C600850779BFB2478504638B9712BA
:10D0300081471808B306F70098083E973386F90031
:10D0400003470700034606008507318F2380E6006B
:10D05000E39177FF90080C085285EFF0DFE34DF97C
:10D060003546E285130511012308B101EFB0307D8B
:10D07000139704014183939784002183D98F10185B
:10D080000C085285231FF100EFF0FFE051F18147BA
:10D0900010183387F9003E96034707000346060041
:10D0A000B306FB008507318F2380E600E39277FF0C
:10D0B00075A01808B306F70098083E973386F90064
:10D0C00003470700034606008507318F2380E600EB
:10D0D000E3E127FFCA876398770990080C08528517
:10D0E000EFF07FDB15F581479800B306F700900855
:10D0F00018103E973E960347070003460600850733
:10D10000318F2380E600E39177FF3546E2851305F2
:10D1100011012308B101EFB090721397040141830C
:10D12000939784002183D98F10180C085285231FF0
:10D13000F100EFF05FD6E31D05EC8147101833874F
:10D14000F9003E960347070003460600B306FB00BE
:10D150008507318F2380E600E3E227FFC109410BF9
:10D16000E5BB8147B5B79408BE9683C6060018088C
:10D170003E972300D7008507B9BF638E062CEF5278
:10D18000CF8759712A84BE89B28B854735461305EE
:10D1900011022E8B468C4289BA8A368A2300F1020C
:10D1A000EFB0F06910180C10228523170102EFF080
:10D1B0009FCE631E0510A1476319FC0693079005D7
:10D1C00063930900E5473546DA8513051102931488
:10D1D0000A012300F102C180EFB0706693178A0044
:10D1E00013D78400D98F90080C1022852317F102E1
:10D1F000EFF07FCA69ED639009049307FA00BD88D8
:10D20000918391E0C144C207C183DE8C814A3EC64E
:10D21000414DB24763EAFA0C6286B3854B01881030
:10D22000EFB0905F4DC53D555DA093079004E39C22
:10D2300009F8A54749BF834701050947C14C2300A9
:10D24000F10283471105B3C7F900A300F1029387E8
:10D250002900814963EFFC02814618103306D7008C
:10D260008C083387D900B69556970347070083C5C6
:10D27000050085062D8F2300E600E390D7FE414789
:10D28000639AE70490080C102285EFF0DFC035D5D3
:10D290003DA8B3863A01BA871010B305F60090088E
:10D2A0003E9603C506000346060085078506298EBF
:10D2B0002380C500E39297FF3387EC4090080C1061
:10D2C0002285BA99EFF03FBD8947014741D5656195
:10D2D0006F407FF690083E96034606001410BE96F7
:10D2E0002380C600850769BFB247850A93990A0162
:10D2F000939D8A0093D909016399570D8547354657
:10D30000DA85130511022300F10293D98900EFB0E9
:10D310001053B3ED3D0190000C1022852317B1038B
:10D32000EFF07FB74DF58147A68963E6970626861D
:10D330000C084A85EFB0B05081471810B306F700CB
:10D34000100898083E973E960347070003460600DC
:10D350008507318F2380E600E3E197FE639DA905F1
:10D3600090080C102285EFF01FB335F1814798101B
:10D37000B306F700900818183E973E96034707003B
:10D38000034606008507318F2380E600E391A7FF5F
:10D390004109C10CBDBD18089000B306F7003E96C8
:10D3A0003387FC0003470700034606008507318FDB
:10D3B0002380E60095BF98084E97034707001C108E
:10D3C000CE972380E700850951BF85473546DA852A
:10D3D000130511022300F10293D98900EFB0304602
:10D3E000B3ED3D0190000C1022852317B103EFF03F
:10D3F0009FAAE31E05EC814718089000B306F700CA
:10D400003E963387FC000347070003460600850766
:10D41000318F2380E600E391A7FF41460C084A853F
:10D42000EFB0F04181471810B306F70010089808D4
:10D430003E973E9603470700034606008507318F57
:10D440002380E600E391A7FF90080C102285EFF0FF
:10D450009FA41DDDADBD7D558280EF421FDD011112
:10D460002A842E8593055100328902C002C202C46B
:10D4700002C693047400EFF0AFD61D46A6851305CF
:10D480009100EFB0D03B10088A854A85EFF0BFA02D
:10D4900019ED93071400180883C607000346070018
:10D4A00085070507B18EA38FD7FEE397F4FE0561CC
:10D4B0006F40FFD9EF42DFD52E848C414111AA89FC
:10D4C000838715003289914463D30700A14497975D
:10D4D000FF1F938767F79C43B1C3B5CE8D472310D9
:10D4E000F10083C725004A852301F10083C7350079
:10D4F000A301F10083C745002302F10083C7550053
:10D50000A302F10083C7650093059100A303010006
:10D510002303F10023040100EFF08FCC0C404A8676
:10D520000A85EFF00FCE0328040083564400A68836
:10D530001D0881470147E51642868A854E85EFF032
:10D540005F982A8909E5A6852285EFB0FFB24A8552
:10D5500041016F403FCF4A860A85EFF08FCA7DBFF9
:10D56000EF421FCB2E848C414111AA89838715007D
:10D570003289914463D30700A1449797FF1F938793
:10D58000A7EC9C43B1C3A5CE8D472310F10083C700
:10D5900025004A852301F10083C73500A301F1006E
:10D5A00083C745002302F10083C75500A302F100A1
:10D5B00083C7650093059100A30301002303F100D5
:10D5C00023040100EFF0CFC10C404A860A85EFF03A
:10D5D0004FC383564400032804008A85858EC20603
:10D5E0001D08C1822312D400A68881470147E51691
:10D5F00042864E85EFF07FB841016F40BFC44A8636
:10D600000A85EFF00FC0C9B7EF423FC2B335B00093
:10D61000011185052A891315F601336515012308C3
:10D62000B1009305110136843AC632C03EC442C2ED
:10D63000EFF00FBBA2471248425593D68700230B49
:10D64000F1009305910193578800A30AD100A30B21
:10D65000F100230C0101EFF0AFB832470246032876
:10D660000400B337E000835644009207914411C28E
:10D67000A1444A85A68842860C08EFF09F842A8937
:10D6800009E5A6852285EFB03F9F4A8505616F4079
:10D690001FBCEF42FFB701113EC68647B335B0004D
:10D6A0008505AA891315F6015D8D2308B100930540
:10D6B000110136843A89B28442C446C2EFF04FB2B7
:10D6C00022489248164593578800A30AF100930513
:10D6D000910193D78800230B0101A30BF100230CC8
:10D6E0001101EFF0EFAF3247104083564400B337DB
:10D6F000E000920703280900914891C0A1480C0856
:10D700004E85EFF09FA7AA8411E5835544004A8512
:10D71000EFB09F96268505616F40DFB2AA9593070B
:10D72000F00F17F700001307A7896317B50013C59B
:10D73000F7FF1375F50F828005058346F5FFB58F5A
:10D74000BA9783C70700D5B703574500144193071D
:10D75000F00F17F600001306A6863697420741839E
:10D76000139506014181631BE500AD8FB29703C598
:10D770000700130515F3133515008280850603C5D0
:10D78000F6FFA98FB29783C70700D9BFEF42FFA961
:10D79000B28736842E86BA86AA853E85BA84EFF093
:10D7A0006FE6634B05002285EFB0D0302A86A6864F
:10D7B000A2852685EFF00FE56F407FA9EF425FA5B8
:10D7C0005D712A8BAE8A17E500001305E57C2C00FD
:10D7D000B284368ABA893E89EFF04FE42A8459E54B
:10D7E00034104146DA852800EFF0CFE12A843DED80
:10D7F0008547A303F100A6C2930771002408BEC4A5
:10D80000A68685470D462C18281002DC02DED6C0FD
:10D81000BEC6EFF00FDB2A8431E983477102A6868A
:10D820000D4693F7F7072300FA00C1473EDE2C1898
:10D830008947281026DCA303F100EFF08FD82A8453
:10D8400015E54146A6854E85EFB0607F8D47A686DB
:10D850000D462C182810A303F100EFF08FD62A8470
:10D8600011E54146A6854A85EFB0607D228561615C
:10D870006F405F9DEF427F9B97D7000093874709DA
:10D88000984383C7470079712A89AE8417E5000061
:10D89000130505710C083AC42306F100EFF00FD808
:10D8A0002A8415E514104146CA850808EFF08FD583
:10D8B0002A8411ED140815462C000810EFF08FD4BF
:10D8C0002A8411E521462C082685EFB04077228571
:10D8D00045616F40DF97EF425F9597D700009387D0
:10D8E00027039C477971AA842E8417E5000013054D
:10D8F000A56B0C083EC6EFF06FD20DE51410414643
:10D90000A6850808EFF00FD011ED140811466C0041
:10D910000810EFF02FCF19E58347F10193F7F703D4
:10D920002300F40045616F409F92EF421F903688BC
:10D93000A14881470147E546EFF0AFD86F403F91DE
:10D94000EF42BF8E3688A14881470147E546EFF098
:10D95000DF826F40DF8FEF425F8D01112A842E85B9
:10D960000C0832C6EFF08FCB19E9324797E600007A
:10D97000938606621008C1452285EFF03FE10561FC
:10D980006F40FF8CEF427F8A4111C1472EC032C4E5
:10D990008A8509463EC23EC6EFF0AFC241016F40E4
:10D9A0001F8BEF429F884111AE8613061009AA858E
:10D9B0000A8502C002C202C402C6EFF0AFC4410130
:10D9C0006F40FF88EF427F86328797E6000093869C
:10D9D000265E2E8693050002EFF05FDB6F403F87E7
:10D9E000EF42BF847971C1472ACC2ED032D42C08A3
:10D9F0000D4628003ECE3ED23ED602C402C602C824
:10DA000002CAEFF00FBC45616F407F84EF42FF8197
:10DA10000111AA842E8417E500001305E5598A85B3
:10DA2000EFF0CFBF05E514084146A6850A85EFF063
:10DA30006FBD09ED8347E1010347F101A207D98FCB
:10DA4000CA07C9836177D98F2310F40005616F403D
:10DA50001F8005C9EF426FFD9787FF1F9387474CD3
:10DA600090439785FF1F9385E54B1785FF1F13058F
:10DA70002547EFB080091785FF1F130565466F40E6
:10DA80000FFD1785FF1F1305A54582809DC5EF4239
:10DA9000CFF99787FF1F9387A748944301112E84DE
:10DAA0000A869785FF1F9385E547EFB0800A0A85B0
:10DAB0000294014505616F408FF97D558280EF42E8
:10DAC000CFF6EFB080149787FF1F23ABA74417F55D
:10DAD000FFFF130525F8EF90D0406F404FF71787F1
:10DAE000FF1F130727469317150008433E95FD5760
:10DAF0002310F5008280EF424FF32A84084019E199
:10DB00006F40EFF41C4158401CC06313E5005CC03B
:10DB10008347550023200500F99BA302F500EFB0D1
:10DB2000EFF9E9BFEF42CFEE9787FF1F9387874357
:10DB300098432A8411CB8347350093F7070289C79E
:10DB4000035505008945029713054401EF90101312
:10DB5000835504000355E400EF20701B485809C5A5
:10DB6000EFB0CFF5232A040213058403EFF0BFF8CA
:10DB70008144B149EFA0FF9A63C5A40283473400F2
:10DB80002320040493F727FCA301F4000048EFA02E
:10DB90005F9A1316150081452285EF400FEC6F4008
:10DBA0006FEAB38734030329040385043E994A8549
:10DBB000EFF07FF42304090075BF8347350093F726
:10DBC000070299E3014582808357E500E39CB7FE95
:10DBD000C167FD176316F600054582800545B9A0AB
:10DBE000EF42AFE493170601C187B2842A8401494A
:10DBF0006359F002835705008DCB01456367F6003A
:10DC0000034584003E953325A6001375F50F39A80A
:10DC10001C4813171900BA9783D70700E38097FCB5
:10DC20000509EFA01F91E345A9FE01456F402FE2D2
:10DC3000EF420FDEAE89AA84EFA07F852A84EFD061
:10DC4000BFAAAA86014713068401970500009385A1
:10DC500045E91785FF1F1305252FEFA0AFD52A89AA
:10DC600021CD8C441304C50022859E0593F505083B
:10DC7000EFB00FC5CC4083877400E18163D1070406
:10DC800093E505082285EFB0AFC30D4693854400A8
:10DC90002285EFB00FC183D504002285EFB0EFC518
:10DCA00083D524002285EFB04FC503D6490083A554
:10DCB00009002285EFB0EFBE4A856F40AFD893F5DB
:10DCC000F507C9B7EF426FD601112A84328532C6F3
:10DCD000EFB06FB4EF903F91835704001787FF1F99
:10DCE0001307C73F3246231BF100930700F8A30D2B
:10DCF000F1001C471843231AA1008983858BB307C1
:10DD0000F740B28548083ECE231C0100230D0100D8
:10DD1000EFF01FF205616F408FD3EF426FCF0041EC
:10DD2000014529CC9304C40026853289AE89EFB021
:10DD30008FB295452A8A2685035B0401EFB02FAF89
:10DD40002685EFB02FC68D45AA8A2685EFB02FAE67
:10DD50002685EFB02FC55C48420A135A0A01D297B4
:10DD60005CC423186401814763983A0146054D81DC
:10DD7000330625419337160013F5F70F6F408FCC0C
:10DD8000EF422FC889692A8BAE8B328AB68A8144CA
:10DD90000144314CFD19EFA0CFF863C9A400EFA0F6
:10DDA0004FFB018D33B5AA006F402FC9338984031F
:10DDB00083270B003E9963170A0083478900850477
:10DDC0003E94D1BF03560A00DE854A8533F6C9006A
:10DDD000EFF0BFF47DD10545C1BFEF420FC5011182
:10DDE0002A847C000355E5003ECAB70707003ECCF5
:10DDF0007C003ECEEF10303D2A8985454808EFB0C3
:10DE0000EFC199454808EFB02FA7AA844A85EF10C3
:10DE1000B03D2380A4009787FF1F9387272C9C4346
:10DE20004166130606F09396870113D78701558F35
:10DE300093D68700F18E558FA207B706FF00F58FA6
:10DE4000D98F11462C00138514003EC4EFB0201F5B
:10DE50005008A382040089452285EFF0BFE609C976
:10DE6000AA8513058403EFB0EFBB3C4085073CC097
:10DE700005616F40CFBDEF424FBBEFA08FED2A840D
:10DE80000504EFA00FEC3305A402F14791453305DB
:10DE9000F502EF10207B01E565556F404FBB97877A
:10DEA000FF1F23A9A70AEFA0CFEA2A840504EFA049
:10DEB0004FE93305A40289450605EF10A07869DD16
:10DEC0009787FF1F23A0A708EFA0AFE82A840504C7
:10DED000EFA02FE73304A4029787FF1F239687063E
:10DEE000EFA02FE72A84EFA0CFE593071400338536
:10DEF000A7029787FF1F239AA70497E7000093873D
:10DF000067CF1787FF1F2325F704014579B7EF4235
:10DF10002FB0AA842E8901449789FF1F9389091C79
:10DF2000130A8006EFA0EFE16345A40001456F40AE
:10DF30006FB13305440383A709024A86A6853E953F
:10DF4000EFF0BFC719E10504F1BF0545CDB7EF42BA
:10DF50004FABAA8A2E8BB28B368C3A8A814401440D
:10DF60008149978CFF1F938C6C17130D8006EFA0CF
:10DF70004FDD63C7A40011E085494E856F40EFABCC
:10DF80003389A40383A70C025E86D6853E994A8511
:10DF9000EFF0BFC219CDEFA0CFDB0544636B4501A5
:10DFA000D2866286DA8513050903EFF07FDD11C1A1
:10DFB000854985046DBFEF42AFA5C16441112A892F
:10DFC00001449789FF1F93896911130A8006FD1484
:10DFD00036C632C42EC2EFA0CFD692452246B246F4
:10DFE0006346A400014541016F40CFA533054403BA
:10DFF00083A709023E9509C683473500C18B9DC79B
:10E0000091C68347350093F707028DC363069900D5
:10E010008357E500639C27010357050001CB63E7A5
:10E02000E50083478500BA97E3CFF5FA05044DB7BD
:10E03000EF420F9EC1642A8901449789FF1F93898B
:10E04000E909130A8006FD14EFA0AFCF6344A400D2
:10E050006F404F9F3305440383A709023E958357C2
:10E06000E500638897006304990063942701EFF04B
:10E070007FAB0504D1BFEF424F9889692A8AAE8AE7
:10E08000328BB68B8144178CFF1F130C2C05930C1D
:10E090008006314DFD19EFA0CFCA63C4A4006F40C4
:10E0A0008F993389940383270C028355CA015A86BA
:10E0B0003E994A85EFF07FB005CD814D05A03384B0
:10E0C000AD038327090303D60B00D68533F6C900B9
:10E0D0003E942285EFF07FC419E5850DEFA06FC453
:10E0E000E3CFADFC31A02285EFF0FFA023040400B4
:10E0F000850455B7EF42EF904169AA8A014A178B10
:10E10000FF1F130BABFD7D19C14B054CEFA06FC377
:10E110006344AA006F406F9293098006B3073A03E5
:10E1200083290B02BE9983D7E900638C270163849E
:10E130002A016398570103A4890311E44E85EFF087
:10E14000DFC9050AE1B78357040163997707930490
:10E15000C4002685EFA03FF085452A8D2685835C87
:10E160000401EFA0DFEC2685EFA0FFFF62056185CB
:10E17000635F05028D452685EFA07FEB89452685E7
:10E18000EFA0FFEA89452685EFA07FEA8545268531
:10E19000EFA03FEB83470500094793F7F707639824
:10E1A000E70099452685EFA0DFE9A30285014848ED
:10E1B000337D2D01231894016A9548C40040B5BFF2
:10E1C000EF42AF8637E404008327041D82979787C8
:10E1D000FF1F83C7A7DD1755FF1F13052547A300A2
:10E1E000F5008327441C82978327841C81461306ED
:10E1F000F00F8145014582976F406F851787FF1F9C
:10E200001307C7CA18439785FF1F83C525DA978769
:10E21000FF1F938727D88346870303469703639797
:10E22000D5009787FF1F2383C7D8828083C58701C6
:10E230000347A7036317B6009787FF1F2388E7D616
:10E24000828003C687016317C7009787FF1F238F4C
:10E25000D7D4828083C68701130750026319D70081
:10E26000930760021787FF1F2302F7D4828083C6BB
:10E270008701130660026315D60093077002DDB7AD
:10E2800083C7870155BF9787FF1F9387A7D0D44BBC
:10E2900009476385E608EF325FF91789FF1F130905
:10E2A000A9CC3E8483470900918B9DCFB7E404003D
:10E2B00083A7041D829783A7441C1785FF1F13059E
:10E2C00025CB829783A7841C81461786FF1F0346B0
:10E2D00026CC81450145829721C183470900ED9BEA
:10E2E0001787FF1F2302F7C88347040093F7F70F30
:10E2F00085C791471787FF1F2328F7CAEFF05FEC08
:10E30000EFF0DFEFB7E70400BC4F414691451785BA
:10E31000FF1F0345A5C882976F307FF38280EF32DD
:10E32000DFF08D4741116304F504C5476306F5022C
:10E3300085476310F5029787FF1F238BA7C6B7E7B2
:10E340000400BC4B930500101785FF1F034505C54E
:10E35000829741016F30BFEF85471787FF1F230961
:10E36000F7C4B7E70400BC4B93050020F1BF9787C3
:10E37000FF1F938727C2D44B1147638DE600B7E791
:10E38000040083A7071D8297B7E70400BC4B9305E1
:10E3900000045DBF05491787FF1F232727C183C7D7
:10E3A000070032C62E8493F7F70FC5D7B7E40400F1
:10E3B00083A7041D7D141374F40F8297E37689FC00
:10E3C000B245994703C61500E3F0C7FCFC440906B3
:10E3D0001785FF1F130505BE8297BC4893050008EB
:10E3E0001785FF1F034585BB829779BFEF32FFE397
:10E3F0001787FF1F130707BA4047184B1C40978623
:10E40000FF1F23AFF6B86316E4001787FF1F232B07
:10E41000F7B8130584FEEF907FF3035564FFEF9088
:10E420003FC6EFA0BFE96F309FE2EF321FE0978752
:10E43000FF1F938727B6D84BDC4799C3EFF01FFB2C
:10E4400085471787FF1F2321F7B69787FF1F9387FD
:10E45000E7A59C43930500021785FF1F034505B4FC
:10E4600083C787031787FF1F2302F7B4B7E70400AA
:10E47000BC4B82976F30BFDD9787FF1F23AEA7B0DD
:10E480008280EF32FFD837E404007C4CA145178529
:10E49000FF1F0345A5B082977C48A1451785FF1F44
:10E4A0000345C5AF9784FF1F9384C4AE8297DC44B5
:10E4B00089E7EFF05FDD6F30FFD803D567FFEF909E
:10E4C0003FBCAA897DD5D84891476310F7027C4CA0
:10E4D00091451785FF1F034565AC82977C489145A0
:10E4E0001785FF1F034585AB829703A9490103D414
:10E4F00009018947B7E904001787FF1F2326F7AAF8
:10E5000083A7091D21044204829783C784011755FC
:10E51000FF1F1305A51361191757FF1FA308F71253
:10E5200083A7491C418082979787FF1F238207A8F2
:10E5300083A7C91C814609469375F40F4A858297C3
:10E5400011E99787FF1F83C7E7B689C79750FF1F59
:10E55000E780C081B7E70400BC4F2146A14517857D
:10E56000FF1F0345A5A38297B9B7EF321FCC93F7DE
:10E57000052001112E8481CBEFF03FEB13450420E1
:10E5800005616F30DFCC93F70510A9CB9784FF1F8F
:10E59000938444A0DC48EFF07FC61787FF1F130762
:10E5A000E790184383C78401034787036316F70086
:10E5B000DC4499C3EFF09FE385471787FF1F2325AE
:10E5C000F79EB7E70400BC4B930500021785FF1FB9
:10E5D0000345C59C8297134504105DB793F7050862
:10E5E000ADC79787FF1F83C7F79CE9171946978523
:10E5F000FF1F9385459C1305D10093F4F70F1789EE
:10E60000FF1F0349299BEFA0902393970401C18327
:10E610001787FF1F1307879A231DF100231CF100A2
:10E620009787FF1F938707973ACE3ACAD8432306A6
:10E63000010009CBDC439315890154080D46E1859F
:10E64000680082971345040825BF93F72500B1CFD2
:10E650009787FF1F93870794D84B89476306F70274
:10E660009787FF1F83C7479013F7270011EF918B00
:10E6700099CFB7E70400BC4F1306000A89451785F8
:10E68000FF1F0345A591829713452400D5BD9787A9
:10E69000FF1F9387A7819C4383C787031787FF1FAB
:10E6A0002306F790EFF0FFDDC5B793F7050291C79A
:10E6B000EFF03FDD13450402E1B593F7850091C704
:10E6C000EFF0BFD61345840065BD93F7150091C7E1
:10E6D000EFF07FBB1345140065B593F7450091C774
:10E6E000EFF07FBA1345440061BD93F7050485C37D
:10E6F0009787FF1F83C7078A81CBEFF07FAC9147D5
:10E700001787FF1F2322F78A1345040495BD93F74B
:10E7100005010145E38607E69787FF1F93878787F3
:10E72000D84B91476310F7049787FF1F9387C783E0
:10E730009C4313D727008583D98F858B91E7B7E753
:10E74000040083A7071D8297B7E70400FC4F91459B
:10E750001785FF1F03458584829785471787FF1F0D
:10E760002324F7841345040121BD9787FF1F2383CA
:10E77000A7948280EF327FAB9787FF1F23A2078287
:10E780009787FF1F23A0078285471774FF1F130475
:10E79000E4711787FF1F2329F7801C4083C7870375
:10E7A0001787FF1F2304F780EF90FFDF39C19757CA
:10E7B000FF1F23A1A7EA1C4017050000130525DB56
:10E7C00083C787031777FF1F2302F77E1757FF1FA3
:10E7D000A30EF7E69777FF1FA38E077AB7E704002B
:10E7E00083A7070882979777FF1F2389A77A6F303F
:10E7F0001FA6B7C7898E938767ED1757FF1F232B77
:10E80000F7E455BF1777FF1F0347C778795555E3DE
:10E810009777FF1F9387077803C717000507977639
:10E82000FF1FA389E67603C717008D463377D7020B
:10E830009776FF1FA380E67683C617001777FF1F22
:10E840001307C766184393F6F60FA9EA83478703B1
:10E850001777FF1F230CF77485471777FF1F230BCC
:10E86000F7729777FF1F938727709C430145998B19
:10E87000A9E3EF329F9B37E404007C48C14517753C
:10E88000FF1F0345A57182973C4885451775FF1FFB
:10E890000345C570829701456F307F9B83C7170082
:10E8A00085466395F600834797035DB78347A703C3
:10E8B00045B782809777FF1F83C7C76DA1CBEF3223
:10E8C000DF9637E404009777FF1F2385076C7C48A9
:10E8D00085451775FF1F0345656C82977C4C9145F4
:10E8E0001775FF1F0345856B82977C489145177507
:10E8F000FF1F0345A56A82973C48C1451775FF1F56
:10E900000345C569829701456F307F9479558280B0
:10E91000EF32BF912A84035565FFEF906FF697772A
:10E92000FF1F93872767D847BE841DEBEFA05F9832
:10E930009C48232004008DEB9777FF1F23A4876654
:10E940009777FF1F23AE8764B7E70400BC4B894568
:10E950001775FF1F03458564829701456F303F8F10
:10E96000630A87001843D1B780C39777FF1F23AB93
:10E970008762D9BF7955DDB7EF323F8B9777FF1F9D
:10E9800093878773884323260500232405005105B8
:10E99000EF80D02E6F30BF8BEF323F891774FF1F8F
:10E9A000130484711C40411189CF9C472302B50098
:10E9B0002AC61CC1EFF05FFC1C409C4B99C332453A
:10E9C000829741016F30BF88EF323F864111444D3D
:10E9D000328532842EC6EFA00FF92AC42285EFA01B
:10E9E000EFF903A84400630C0800B24583574400C4
:10E9F0001840224683D54500AA8626850298410103
:10EA00006F30FF84EF327F82404D1DC408C09705F0
:10EA100000009385E50213054401EF809018977775
:10EA2000FF1F938767699C43014589E79777FF1F1D
:10EA300023A487686F30BF817D55EDBFEF32EFFEB5
:10EA4000011168009305F00F02C602C802CA02CC89
:10EA500002CEEFF07FF405616F306FFF9777FF1FF5
:10EA6000938787659C43D847A1679D076311F70289
:10EA7000EF32AFFB01113285EFA0EFEE230AA100C8
:10EA800081456800EFF05FF105616F304FFC8280D7
:10EA90009777FF1F938747629C43D847A167938767
:10EAA00077036311F702EF324FF801113285EFA0BF
:10EAB0008FEB230AA10081456800EFF0FFED0561AF
:10EAC0006F30EFF882809777FF1F9387E75E9C4354
:10EAD000D8479547631CF702EF322FF501113285B5
:10EAE0003284EFA04FE8230AA1002285EFA00FE9AE
:10EAF00083574400231BA10081453ECC1C40680085
:10EB00003ECEEFF07FE905616F306FF482809307AE
:10EB100085FF89CF8327C5FF91CBDC4B81CBEF32BB
:10EB2000CFF0032585FF82976F306FF28280EF323E
:10EB3000CFEF2A843285EFA00FE3BD4763EBA70038
:10EB400018449377F5000345B70041995D8DA305FF
:10EB5000A7006F30CFEFEF324FED01117C003ECABE
:10EB6000B70707003ECC7C003ECE5C4D8DCF2A849B
:10EB700013858700AE84EF807004A1652A899D0506
:10EB80004808EF80FFBD9305803EB345B9024808B1
:10EB900093F5F50FEFA0CFD2014781465008A68527
:10EBA0002285EF807FDC05616F306FEAEF32EFE79F
:10EBB000EFF07FFA6F30AFE9EF322FE701117C0001
:10EBC000AE843ECAA165B70707002A843ECC480838
:10EBD0007C00938575033ECEEF809FB81C444808A7
:10EBE00083C5B700BD89EFA0AFCD5008014781466E
:10EBF000A6852285EF805FD705616F304FE5EF3244
:10EC0000CFE22A84AE84EFF09FF2A6852285EFF052
:10EC1000BFFA6F30CFE3EF324FE1EFF0FFF96F3023
:10EC20000FE3EF328FE00329C501411163040902AC
:10EC30002A843285B284EFA00FD32AC62685EFA09E
:10EC4000EFD3832749002A8691C7DC4781C7B245A5
:10EC50002285829741016F308FDFEF320FDD444D07
:10EC600081CC2A843285EFA06FD1DC40AA8589C788
:10EC70009C4799C3228582976F306FDDEF324FD961
:10EC8000032AC501411163030A062E89AA8495450A
:10EC900032853284EF80DFAC85452285EFA0CFBD81
:10ECA000AA89CA852285EFA0EFC283274A009DC7A3
:10ECB000DC438DC72285EFA0AFBA83274A001040FE
:10ECC00083564400DC437115A307A100B2961307D5
:10ECD000F1004E86CA852685829701C523800900EA
:10ECE00031A08345F1002285EFA00FB941016F30BB
:10ECF0006FD5EF328FD365711C083EC2B707800114
:10ED00003EC41C0832893EC62A84AE84EFF07FF1EF
:10ED10004A85EFA0AFC68357A10089CFAA855000CE
:10ED20002285EFF0BFF5014781465000A685228578
:10ED3000EF809FC359616F308FD1EF326FCD657116
:10ED40001C088329C5013EC2B70780013EC41C08C8
:10ED50002A84AE8432893EC6EFF03FF06384090214
:10ED60004A85EFA0AFC18357A100AA8581CF50008B
:10ED70002285EFF0BFF0014781465000A68522852D
:10ED8000EF809FBE59616F30EFCBEF320FCA6571D4
:10ED90001C083EC2B70780013EC42A841C08328585
:10EDA0003EC6AE84EFA08FBD8357A10089CFAA8550
:10EDB00050002285EFF09FEC014781465000A68568
:10EDC0002285EF807FBA59616F306FC8EF32EFC58F
:10EDD000444D91E88347450093B71700B307F040CF
:10EDE0003E856F30CFC61845FD577DDB9707000085
:10EDF000938707032A845CCB97050000938565D130
:10EE000013858400EF80E05980C0034744008147A8
:10EE100061FB1777FF1F2323972AD9B7EF324FBF24
:10EE20008329C5014111032985008147638B0908A6
:10EE30000324090191452A8A2285EF807F92854526
:10EE40002285EFA06FA38945AA8A2285EFA0CFA2D1
:10EE5000AA84EF809F9683A749002A8B9DC79C4375
:10EE60008DC72285EFA0CF9F83A74900A306A100ED
:10EE70001040835644009C431307D100B296D685B8
:10EE80001306E1005285829709CD83570B0023803A
:10EE9000F400A183A380F40023800A00A3060100EC
:10EEA00029A88357E10022852380F4008345D100FF
:10EEB000A183A380F400EFA02F9C8347D100B33738
:10EEC000F0000347B900920701453D9BD98FA30588
:10EED000F90041016F300FB7EF322FB541111DE935
:10EEE0009777FF1F9387871D804305C80440130948
:10EEF00084009DC55C4099C79C4B89C726852EC65A
:10EF00008297B2459307803EB385F5024A85EF802C
:10EF1000605521A0404DAA8479F841016F302FB38C
:10EF20004A85EF80A0555C40EDDBDC4BFDD72685A4
:10EF30008297E5B7EF326FAF2A843285EFA0AFA298
:10EF4000AA852285EFF05FF96F306FB0EF32EFAD39
:10EF50002A84AE84EFF01FFEA6852285EFF0BFBFA6
:10EF60006F30EFAE08413355B50005898280EF322E
:10EF7000CFAB1774FF1F130464161C5C0111231719
:10EF800001008D83858BA303F1008327040B2318D5
:10EF900001002319010003D7C7013ECA3C00231416
:10EFA000E1007D572315E1000357C4023ECC02CE99
:10EFB0002316E100EF802FE38357E101231EA10018
:10EFC00093F707E093E71710231FF1009777FF1FD0
:10EFD00083C7671385C305470145638AE7008347F5
:10EFE000840393E727001777FF1F2305F7120561B6
:10EFF0006F30EFA5814717D700001307A71B854681
:10F000001306710085454808EF70E04B6DF18347AA
:10F010008403F59B1777FF1F230EF70E854717779D
:10F02000FF1F2302F70EE1B7EF322F9D977DFF1FE1
:10F03000938DCD0A03A6CD0639712A898147814473
:10F04000930600023357F600058B01C7850493F43D
:10F05000F40F8507E398D7FE83A70D0B2317010252
:10F060002318010203D7C7013EDA3C102314E10242
:10F070007D572315E10203D7CD023EDC231901029F
:10F080002316E10202DEEF800FD68357E103231E31
:10F09000A102014593F707E093E71710231FF10240
:10F0A0009777FF1F83C72706A9EF9777FF1F83C7AF
:10F0B00077063EC69779FF1F938949020144014DA7
:10F0C0009D4A054B954B177CFF1F130C6C08977CD2
:10F0D000FF1F938C6C0703DAC90563090A00EA85F0
:10F0E000631459036685EFF0FFE71DC1050DA147C5
:10F0F0008909E312FDFE2DE09777FF1F23A807047F
:10F10000014521616F302F936285EFF0BFE579DD16
:10F110003247B3878400E3F0E7FE9C001306140037
:10F1200006043E9413178A0093578A00D98FC207AA
:10F13000C183A30EF4FCA183230FF4FC03A70D07E6
:10F14000B317AB01D98F1777FF1F2321F700630493
:10F150007601328461BF15449777FF1F83C787FA12
:10F16000138717009776FF1F238EE6F89316140077
:10F17000230EF10017D700001307C7038147850648
:10F180007008CA854818EF700034E34705F68347D6
:10F19000C10105451777FF1FA306F7F69777FF1FF5
:10F1A000238327F7B9BFEF32AF860111AA892E84D6
:10F1B000EFD0EF9C2A899774FF1F938424F2639900
:10F1C000090A9C5C414793F707036393E70A1777A3
:10F1D000FF1F034797F3894763ECE70883A7040BF6
:10F1E000231701002318010003D7C7013ECA3C00C2
:10F1F0002314E1007D572315E10003D7C4023ECC60
:10F20000231901002316E10002CEEF80CFBD231E9B
:10F21000A100EFC06FCD8357C101230FA10091461C
:10F2200013D78700A207D98F2312F1009777FF1F0A
:10F2300083D767EE13D78700A207D98F2313F10076
:10F2400017D70000130787F68147500095454808F7
:10F25000EF70602705889317240003C484036D981A
:10F260005D8C9777FF1F238787EA05616F209FFDDD
:10F27000EF70B0781775FF1F130545EAEF80002087
:10F2800083A7040B9775FF1F83D505E803D5C70136
:10F29000EF10E0279777FF1F83C7C7E793F60702B2
:10F2A000014789E61777FF1F035707E69776FF1F89
:10F2B0002394E6E61777FF1F130707E1184309CBEE
:10F2C000C18B99C789451775FF1F0355E5E3029761
:10F2D0009777FF1F23AA07E29777FF1F238507E28F
:10F2E0009777FF1F23A207E69777FF1F23A007E664
:10F2F0009777FF1F23AE07E483D7840393F7270C88
:10F3000093E717001777FF1F2316F7E083572903AA
:10F31000A18B99C3EF70E03F11C49777FF1F23A122
:10F3200007DEA1B78D471777FF1F232BF7DCEF9080
:10F330002FA59305803EB305B5021775FF1F130572
:10F34000E5DDEF80201215B79777FF1F938707D968
:10F35000D85325C791C99777FF1F238607DA977778
:10F36000FF1F23A507DE8280EF223FEC83C7F70251
:10F3700041112EC685071777FF1FA308F7D8977787
:10F38000FF1F239CA7D89D471777FF1F232AF7D677
:10F39000EF900F9E2A84EF90AF9DB24501E5EF906C
:10F3A0002F9DAA85B305B4401775FF1F130505D718
:10F3B000EF80400B41016F209FE982809777FF1F0C
:10F3C0009387C7D1D85331C7EF223FE603C7F7026F
:10F3D00005079776FF1FA38AE6D211CD8C5F0D47F4
:10F3E0000145898185899776FF1F23ABE6D0EFF031
:10F3F0009FDB6F20DFE585479305C0441775FF1F2E
:10F400001305C5D11777FF1F232CF7CEEF8080059A
:10F41000CDB78280EF227FE11777FF1F0347A7CE8A
:10F420008547631EF7009777FF1F938727CB83C716
:10F43000870393C787001777FF1F230DF7CC177536
:10F44000FF1F1305A5CDEF806003EF807FEF994785
:10F450001777FF1F2326F7CA9777FF1FA38707CACF
:10F460009777FF1F238107CAEF90AF8F930740065E
:10F470003305F5029777FF1F23AAA7C86F203FDD4A
:10F480009777FF1F83C707C9C18B99C7EF22FFD9A1
:10F49000EFF0FFAD6F20BFDB695582809777FF1FCC
:10F4A0009387C7C3DC5381CBEF223FD88545EFF06C
:10F4B0009FCF6F20DFD982801777FF1F130707C206
:10F4C00001468146BA852148631E06019DCA2390E4
:10F4D000A60083C7850393E717001777FF1F230B49
:10F4E000F7C205A08357C705631DF502F859854784
:10F4F000B397C70093C7F7FFF98F1777FF1F23292B
:10F50000F7C49C5D9183858B85C79777FF1F83C761
:10F5100087BF99EFEF227FD11D45EFF0FFB06F203D
:10F520001FD381E699E39306C7050506090769BF5E
:10F530008280EF221FCD8605AA84B309B500977A91
:10F54000FF1F938A6AC0054B977BFF1F938B0BC0ED
:10F55000214C639434039777FF1F938727B89C5FF0
:10F560009183858B89CB9777FF1F83C7C7B981E7C5
:10F570002145EFF07FAB6F205FCC03DA0400630B13
:10F580000A041779FF1F130969B50144CA8C835710
:10F59000C905639D4703A2855685EFF0BF9C11E521
:10F5A000A2855E85EFF01F9C05C903A74C07B31722
:10F5B0008B00D98F1777FF1F232CF7B883C78C03D5
:10F5C00093E717001777FF1F2306F7B4050409090F
:10F5D000E31F84FB8904B5BF231E0904C5BF177749
:10F5E000FF1F034747B28547631AF700EF22FFC3A7
:10F5F000EFF05FE2EFF0BF976F207FC58280814719
:10F6000085451306000293861700B397F500E98F2E
:10F6100013F7F60F89E7B687E397C6FE01473A85E9
:10F620008280FD4785457D56B396F5001387170008
:10F63000E98E1377F70F89E6FD17E397C7FE0147B9
:10F640003A85828089E901473A85828001473A8577
:10F6500041016F20DFBFEF225FBD41112AC62E8519
:10F660002EC4EFF0DFF9A2457D158547B397A700BB
:10F67000E39EF5FC32469377360099C3719A1106E2
:10F680009777FF1F938747A594433E871778FF1FFF
:10F690001308C8A389EA832708009107F19B97768E
:10F6A000FF1F23ABF6A2032588001843B307A7006A
:10F6B000B3F7B702B387F540FD15FD8D83274800EA
:10F6C000AA95B306B600E3F3F6F8E371D5F82E97E2
:10F6D0009777FF1F23A0D7A03DDB3A858145EF2018
:10F6E000DFB72A87ADB718419777FF1F9387079E2B
:10F6F00023A4070098C35841D8C39777FF1F23ADB1
:10F70000079C8280EF22DFB0AA8401441779FF1F93
:10F710001309C99C9309400EEF807FD56345A4006F
:10F7200001456F203FB2330534038327090B3E9513
:10F730008357C501E38797FE0504F9BFEF227FAC2D
:10F740009779FF1F938989993E84BA84834706007D
:10F7500003A7090041119D83058B3D8F83C7440199
:10F76000AE8A2A89F99BD98F238AF4001C44B68576
:10F77000231204001CC02285328A36C6EF90DF8F28
:10F78000B246D2853686EF90900BDC4883A50900FF
:10F790000840858B56869D8DEFD03FCC61E918409F
:10F7A0007D558347570003476700A207D98FC207DB
:10F7B000C1872394F4006358F00A83C7440193F788
:10F7C0000703B5CBD0489377160003A609001D8E1A
:10F7D0009777FF1F938747C79C43ADEB814641A0B6
:10F7E00003A70B0093172A00BA9718409443834746
:10F7F00057008345670033F65601A207CD8F63118A
:10F80000F602834737000346470003472700A20755
:10F81000D18F4207D98FBD82B3F76701638AF6049F
:10F82000050AEF80DFC3420593170A014181C183B6
:10F83000E3E8A7FA41BFA16A370B0200014A977BB0
:10F84000FF1F938B6B97FD1A7D1BE1BF83C744019C
:10F8500013070003854693F70703E391E7F8A285B2
:10F860004A85EFD0FFCF41016F203F9D6155E5BF35
:10F870007955D5BFEF22DF999764FF1F9384446EBB
:10F880009C40D9EF9777FF1F9387C7839C43639969
:10F89000070CEF80DFBE930780023305F502894530
:10F8A000EFF05FDA41C99777FF1F23AFA78CEF8096
:10F8B0001FBC9307400E3305F5029145EFF09FD82A
:10F8C00035C99777FF1F23A3A78CEF805FB201CDC7
:10F8D000EF80FFB191450E05EFF0DFD621CD977790
:10F8E000FF1F23A7A78AEF801FCB11CDEF80BFCAD0
:10F8F000D9473305F5028945EFF0DFD405CD977779
:10F90000FF1F23A1A788EF809FB591450A05EFF05F
:10F910007FD30DC19777FF1F23A0A78A014521A898
:10F92000EF803FC2930780063305F5029145EFF063
:10F930007FD101E565556F20FF909767FF1F23AFCB
:10F94000A77A0144130A80061769FF1F1309097972
:10F95000B14AEF801FBF6364A4029C40E38407F2B6
:10F96000EF803FBE9307A0043305F5028945EFF011
:10F970007FCD69D19777FF1F23A4A78419BFEF809C
:10F980005FBB89450605EFF0FFCB4DD5B3094403B6
:10F99000032709024E9708CBEF80BFB83305550304
:10F9A0009145EFF03FCA59D5832709020504137426
:10F9B000F40FCE9788DB71BF9767FF1F938707729D
:10F9C000884705898280C167FD176319F50097672D
:10F9D000FF1F9387A77003A5070B8280EF22FF8488
:10F9E000EFF05FD26F20BF86814709C58347E501ED
:10F9F000B337F0001767FF1F1307476E18470983D7
:10FA0000058B19C393E727003E858280EF22FF8193
:10FA10002A84EFF07FFD8347E401AA85130594084B
:10FA200099E3130504039766FF1F9386266B9442A0
:10FA3000130615021307840213059504EFD0CFC0F7
:10FA40006F20FF80EF22CFFC9764FF1F938404692F
:10FA500098442A892E840983058B9C4019C7631416
:10FA6000F5006380050E014401A2E3FEA7FE1387A3
:10FA7000A702E36AA7FE850763FCA70883A9440BD6
:10FA8000EF80FF961316350081454E85EF20EFFC81
:10FA90009767FF1F23A427659767FF1F23A20764AB
:10FAA00049CC9C4493E747001767FF1F232CF7625C
:10FAB0009767FF1F2380076A630F040C9767FF1F78
:10FAC00023AE276101440549EF807F926341A40A78
:10FAD000EF80FF9493050006B3C5A502B7F7360083
:10FAE000938707E81765FF1F130505674169014400
:10FAF0009309400E7D19B385F502EF70B016EF80C3
:10FB00001F97634FA4080145EF3040700544A9A832
:10FB10006398A7029DE583A9440BEF805F8D1316C0
:10FB2000350081454E85EF204FF39767FF1F23A7D0
:10FB3000275B9767FF1F23A5075A9C44ED9BADB732
:10FB400085C51767FF1F0347E7609307F005E3FCD0
:10FB5000E7F021F8EF60F03C6DD19C4493E7070299
:10FB60001767FF1F2320F75822856F20AFED83A76B
:10FB7000440B131534003E958357050081CB834712
:10FB8000250099C721468145EF202FED05042DBFA3
:10FB900023012501E5BF9767FF1F23A307540DBF6E
:10FBA0003305340383A7040B3E958357C501638453
:10FBB0002701EFF0BFE5050499B7EF220FE7EF80CB
:10FBC0001F86130400063345A4029764FF1F938425
:10FBD000E45083C784073E951375F50F9767FF1FA1
:10FBE000238AA7569307F00563E7A7020545EF3080
:10FBF000E061EF80DF823345A402B7F536009385DC
:10FC000005E8B305B5021765FF1F1305E554EF704E
:10FC100070056F20CFE39C4405458983858B81CB9C
:10FC2000EF904F8888408145EFF0DFE1DDB7EF309E
:10FC3000E05DC5B7EF22CFDD130495082A891306CE
:10FC40009005A28513050503EF90603F130690050C
:10FC500081452285EF206FE04A85EF30C054814412
:10FC6000176AFF1F130A8A47930A8002EF803F81B9
:10FC700063C4A4006F200FDD338454038327CA0AB2
:10FC80003E94035704008357C9016317F702834763
:10FC900044009DC3930964014546CE851305540075
:10FCA000EF90E039454681454E85EF200FDB2285F8
:10FCB00023020400EF30005785044DBFEF22EFD63A
:10FCC0009767FF1F9387C7299C432A8491C70DC557
:10FCD0000355C501EFE00FC29767FF1F9387C776F3
:10FCE0009C4389CBEFB0DFD085476315F5002285B3
:10FCF000EF50C05D6F20AFD541657D15E1BFEF22AC
:10FD0000CFD21764FF1F1304643D4440938714004F
:10FD10001767FF1F2326F73CEF30605E1C44898382
:10FD2000858B9DE75840B7E7B0009387075063F194
:10FD3000E7020145EFF01F9D01CD0545EF809FF6DD
:10FD4000084085450505EFF0FFCF0145EFF01FF7AF
:10FD500026856F20CFCFEF22AFCBA1642A89014443
:10FD60009769FF1F93894945FD14338AA500EF80E9
:10FD70000FEF6344A4006F20EFCC03A70900931793
:10FD80002400BA979843658F42074183634C27014B
:10FD9000635A470123800700A380070023810700DF
:10FDA000A38107000504E1B7EF222FC58359450061
:10FDB000C547411163F537310441C1E5338534014D
:10FDC000834785FF034795FF0348B5FFA207D98FF7
:10FDD0000347A5FFC207220733670701D98F0347EF
:10FDE000C5FF0348D5FF2207336707010348E5FF36
:10FDF0000345F5FF420722083365A800498FB98FF4
:10FE00001767FF1F130707391768FF1F1308883A82
:10FE10003A85832807006384172B1107E31B07FF2C
:10FE20001767FF1F13070739184313182700429558
:10FE30001CC10507A1473367F7029767FF1F23AB74
:10FE4000E73693F735001397470083474601C16BA8
:10FE5000368993F7F7FCD98F32842E8A230AF6006D
:10FE6000814A176CFF1F130C6C27FD1B976CFF1F3B
:10FE7000938C0C0F176DFF1F130D8D34EF802FDF48
:10FE800063C7AA00E154268541016F20CFBA130849
:10FE9000400EB3870A0303280C0BB30DF800638EE2
:10FEA0000D2083D7CD01638A772183A70C00014BF6
:10FEB000639707169767FF1F9387C7209C4363903C
:10FEC000071683C7040003C70D0493F7F707631BE6
:10FED000F71ACA872287CE86268693859D061385C4
:10FEE0001D04EFF0BF85631F051883D7CD010327DD
:10FEF00009002320B4012312F400FD572313F4005A
:10FF00008347170093F6F7078347D40093F707F862
:10FF1000D58FA306F40093F7F707B337F000B307C4
:10FF2000F0402307F400834717009D839396370022
:10FF300083474401DD9BD58F230AF40083473700B4
:10FF400083464700A207D58F83462700C206D58F78
:10FF50001CC88347770003478700A207D98F231562
:10FF6000F4000D476304EA00BD5491DF9387071046
:10FF7000C207C1831307B00FBD54E376F7F0EF80DB
:10FF80000FC98144E31105F09766FF1F83C606235E
:10FF9000938716001767FF1F2302F7221767FF1FBB
:10FFA00013078721231BD40093972600144303577C
:10FFB0008400E175BE96A1671386F7FFB377C7008B
:10FFC00098426D8FD98F9CC21848F18F3E07D98F08
:10FFD0009CC2EF80CFC89767FF1F83C7271E33F5EA
:10FFE000A7029767FF1F238BA71C71BD9307A0046F
:10FFF000B308FB0283270D00BE9803D7080083D700
:020000040001F9
:10000000CD01631DF70083C7040003C7880093F781
:10001000F707630BF70083C7FD019DEB050BEF802E
:100020004FD2E345ABFC71BD9385980113859800D1
:10003000CA872287CE86268646C6EFF02FF0B248C2
:1000400079F98347440193E74700230AF40071BD1F
:1000500083C7040003C7980293F7F707E310F7FC80
:10006000CA872287CE8626869385A8031385A80291
:10007000EFF0CFEC45F58347440193E72700230ACF
:10008000F400C1B783C7FD018DCB83C7040003C74C
:100090009D0993F7F7076312F702CA872287CE8676
:1000A000268693852D0C1385AD09EFF02FE911E518
:1000B0008347440193E7270049BF850AC1B3FD5434
:1000C000D9B3EF220F94797183544500AA8B2E8403
:1000D000B28AEF80CFBB590563499504B7E40400A9
:1000E00003A90407EF80AFBA59054205418102997F
:1000F0002A8905CD2AC623180100EF804FB959057A
:100100002319A1006146814528089769FF1F93893B
:10011000E9FC4ACAEF206F942302810203A48900FC
:10012000058819E4BC544A85829745616F20EF9099
:1001300074003008D6855E85EFF01FC765F568004E
:10014000EF807FF1176AFF1F130A0A3083270A0026
:10015000AA84035B010189CB89476397FA00835521
:1001600001025E85EF50203003552102EF704FC829
:1001700019E503552102EF708FD43334A000931793
:1001800064000344C1022C0868001374F4FB5D8C06
:1001900023068102EF60B056E9576314F5028356D7
:1001A000E1029767FF1F938727019C43139726005F
:1001B0006176BA979843718F98C39767FF1F238F13
:1001C000D7FE831721026345F00085476396FA0046
:1001D000B25793F7070C95E7D247C2040347C10211
:1001E000C180BE9426C62318610113770703C14757
:1001F000631DF70083475102054793F7F7076390A4
:10020000E704B7E70400BC5739BF92570544A18300
:1002100093F7F707E377F4FE15C78347C102130787
:10022000000293F707036397E700EFB06FFC854781
:10023000E319F5FC8347C10293F7070389CFEFB0B9
:10024000AFCA21A8EFB08FD7E30985FCEFB04FFA12
:10025000E31985FAD9B7EFB0EFD8AA85014605456D
:10026000EF707FF82A8451DD8347C102414793F73D
:1002700007036384E70232478347170093F707F8C1
:10028000A300F7003247925783461700A18393F7E4
:10029000F707FD17D58FA300F70003560101B245FC
:1002A000130BC4005A85EF80DFDFE24A1306900586
:1002B0008347C10283C4EA01918BB384C4021385CE
:1002C0001404569595C35444B3879A0083C7070412
:1002D00003C70600137707F82380E60058448346D7
:1002E0000700D58F2300F700B25703A60900814607
:1002F000858B1D8EDA85EFD0EF9B15E9B25783A56C
:100300000900484413869406858B56969D8DEFD040
:10031000CF9411ED83270A0099EFB25705479183D7
:100320008D8B6387E7049DCF09476389E7042285A6
:10033000EF80DFF8F9B5EFB0AFEB85476309F50063
:100340008347C102414793F70703E398E7FC8355CE
:1003500021025A85EF40907C69D183172102E35E28
:10036000F0FAF1B7EFB08FC57D151335150061D1E7
:10037000014681452285EF70FFEF55BFEFB04FE793
:10038000E5B7EF129FEA9764FF1F9384A4D62685F2
:10039000EF809FEB2A8419E16F107FEB1305C400F7
:1003A00005468145EFF0FFD12285EF803FF1C5B7CB
:1003B000EF12BFE74111AE842A8493079503130718
:1003C00015019306F10005466C0026852306010001
:1003D000EFD0CFBE1DEDA68541462285EF80304689
:1003E0008347F1009305140226852308F400EFD01B
:1003F0006FC805E19767FF1F938707059C4389EF47
:100400001306940497C50000938545DB2685EFD03D
:100410008FD441016F10BFE31306940297C500000B
:10042000938545DA2685EFD00FD379D9DDB7EF1262
:100430003FDE9767FF1F938727D88043AE84B2893A
:10044000368AAA8AEF80AF8113162500814522855E
:10045000EF10BFE09767FF1F238207D69767FF1F44
:100460009387C7C703A4070B13F714003E89230F14
:10047000E400CE8525C713059408EFF07FF301C58E
:1004800055556F103FDC8947A30FF4009767FF1F96
:10049000938787FB9C4303278900858093B71700C8
:1004A00086072300F402231E54019767FF1F23A72A
:1004B00047C385889377B7FF99C09367470017674D
:1004C000FF1F2321F7C22285930700061767FF1F2E
:1004D0002302F7C8EFF08FD3014565B71305040376
:1004E000EFF01FED45D569BFEF123FD4FD57231044
:1004F000F500231105002312050023130500130640
:10050000200481452105EF105FD56F105FD4EF12F5
:100510003FD04111AA8401441769FF1F130949CA3A
:100520009309A0042EC6EF80CF81B2456344A40096
:1005300061550DA033053403832709003E95835789
:100540002500639CB7008357050063989700EFF080
:10055000BFF9014541016F10FFCE0504E1B7EF126D
:100560003FCB9767FF1F9387E7B59C434111AA8450
:100570002E84B28903592500C1C39767FF1F83D713
:10058000A7B8639B2707EF700F862A8903D524003D
:1005900093051002B305B40285472302F100935777
:1005A0008900A302F10093578500A303F10083D7CC
:1005B00044002304A100254613D787002305F1003A
:1005C00083D76400A304E1004E8513D78700A305F9
:1005D000E1002306F1001387950093879501A1059B
:1005E000B386B400A6974C00269723032101EFD0D1
:1005F000EF9C41016F101FC5EF60FFFE51BFEF126E
:100600003FC14111AA8401441769FF1F130949BB67
:100610009309A0043AC636C432C22EC0EF707FF2EE
:1006200082451246A24632476344A400615599A010
:10063000B307340303250900AA9703D8070003D59D
:10064000C4016310A80495E91DEE91CA03C6E40134
:10065000930510023306B60225063E9690C2014568
:1006600011CB83C6E40113061002B386C602E50669
:10067000B6971CC341016F10FFBC03D52700E305EB
:10068000B5FC050441BF83C5E40113051002B38521
:10069000A502BE9583C585002300B6007DB7EF1285
:1006A0003FB75C4141112A8403DA2700C167FD1777
:1006B000AE843289630CFA002685EF807F9A8D47DD
:1006C00063EDA7007D5541016F10DFB72E85EF80E8
:1006D0003F999D47E3E2A7FEF5B75C40268583D5A9
:1006E0004700EF809F90835584002685EF80FF8F21
:1006F0008D452685EF803F8EAA89EFF04FE0935716
:1007000005012380F90093578500A380F900238118
:10071000A9005840C167FD178345A7006314FA007C
:1007200093E505082685EF801F8F9767FF1F938746
:1007300067999C430840D9CF8347B400858BD9CBB8
:1007400078003400130671008145EFF05FEB1DC99E
:100750008347B400184093069005F99BA305F40065
:100760008347E701B387D702B306F70083C60604C1
:10077000A303D1009386170493879706BA96BA9776
:1007800036C43EC61764FF1F130444951C440C4036
:1007900026858983858B9D8D834771009E05DD8D20
:1007A00093F5F50FEF803F871C4410402245898365
:1007B000858BCA861D8EA685EFC0DFCFE31505F0B9
:1007C0001C440C40324689838840858B9D8DEFC048
:1007D000DFC8D5BD8347B40013079005F99BA30577
:1007E000F4008347E501B387E7023307F5000347C9
:1007F0000704A303E10013871704938797062A973A
:100800003E953AC42AC6BDBFEF129FA0032A4500F9
:100810009307F00FAA840347AA00AE893284368971
:100820006316F700EFB06FAB2305AA00938AC900E7
:100830000146D6852685EFF09FE62A8A21E51767CF
:10084000FF1F130767C01843DC4039C383C6A700E6
:100850000547638FE60283D547005685EF40102C8D
:1008600005C9DC40839747006354F00201CC1C406B
:1008700089C74A868145014582975C4081C7CA8500
:10088000014582974E85EF807FA352856F109F9B15
:10089000DC4003D54700EF60BFD501E9DC4003D55C
:1008A0004700EF60DFE181471DCD19C41C4089C7B7
:1008B0004A868145014582974E85EF807F9FAA85B4
:1008C0001765FF1F13050583EF80DF9511C45C409A
:1008D00081C7CA85014582971765FF1F1305C5802B
:1008E000EF60F0368547D84085460346A700E30B06
:1008F000D6F8031747006353E000C9F74A86A2857C
:100900004E85EF703F97BDBFEF129F90AA840144C0
:100910001769FF1F1309C98A9309A004130A9508D0
:10092000EF703FC26344A400014535A03305340392
:10093000832709003E958357250099E30504CDB729
:100940000357050083D7C401E31AF7FE5286854595
:10095000EFF0FFC065D56F10FF8EEF127F8BAA847A
:1009600001441769FF1F1309A9859309A004EF70BB
:100970005FBD6344A4006F10FF8C330534038327ED
:1009800009003E958357250081CF83570500639961
:10099000970093059502130610022105EF80206A47
:1009A0000504F1B7EF127F880347E5012A848347E6
:1009B000F5016307B70089E781452E856F103F89F0
:1009C000230FB400054781C9E398E7FE8947A30FC9
:1009D000F4008545DDB7638BE7020947E39FE7FC39
:1009E0002285EFF02FA59757FF1F9387A76D9C4394
:1009F00099E79757FF1F9387A7569C4389C70355CD
:100A0000C401EFF09FF5A30F0400E1B755D6C9BFAD
:100A1000EF121F80EFA0FFEE85476312F508EF800D
:100A2000EFCC1764FF1F130424A21C4081CBEFA05E
:100A30003FFC89476304F5001C4082979757FF1FCE
:100A4000938747689C43B9CF82979757FF1F938737
:100A500027519C4391C382971754FF1F13040468C6
:100A60008327040B83D4C701EF60FFB78327040BF0
:100A7000AA85144003C6E7011C448983858B99C36A
:100A80001366260026854169EF40C03D8144D9495F
:100A90007D19EF705FB063CAA4006F10AFFAEF80EA
:100AA0000FCA41B7EF705F884DB7B3873403032790
:100AB000840ABA9703D527006308250103C64701B6
:100AC00083D50700EF40A03B8504E1B7EF124FF458
:100AD00001449754FF1F938464601309400EFD592D
:100AE000EF70FF98634FA40401449754FF1F938451
:100AF000E45E13098002FD59EF707F98634CA404F3
:100B000001449754FF1F9384645D5949FD59EF7068
:100B10009FA8634AA40497F5FFFF9385450A1755DC
:100B2000FF1F13056563EF60D007970500009385ED
:100B300085851755FF1F1305255BEF6050056F1066
:100B40006FF03307240383A7040B0504BA97239E91
:100B5000370179B73307240383A7C40A0504BA977A
:100B60002390370151BF3307240383A7840A050468
:100B7000BA972391370161BFD44103873500854778
:100B80003356F5026377E600A54899E7238006000F
:100B90008280B387E702EDB73358F502038735004B
:100BA0003375F502B3D7E7021307000363DA0801D0
:100BB00003C6050013077003118A19E213077005B5
:100BC00085064297A38FE6FEC9B718451C41637698
:100BD000F7005C41BA972380B7001C4585071CC508
:100BE0008280EF128FE44111AA872E85B285368666
:100BF00036C6829763480500B246158D3335A0008E
:100C00003305A04041016F108FE4EF126FE00569DA
:100C100041112A8A2320060001448149975AFF1F67
:100C2000938A8A5C056B7D1932C62EC4EF703F85AE
:100C3000AA84EF70DF832695A24532466346A4005E
:100C40004E8541016F100FE003A70A0093171400AF
:100C5000BA9703D707003377670101E71CC2050481
:100C6000E1B703D707009356D700858AE39946FF7B
:100C700033772701E315B7FEBE89D5B7EF12EFDA58
:100C800001112EC6B2843689EFB02FEE2A84615549
:100C900001C8B24589E9232E04002320040201453E
:100CA00005616F10CFDAA1463008CA852685EFF0BE
:100CB0005FF37DF5835781010357A101231EF400E3
:100CC0008357C1012310E4022311F4028357E10189
:100CD000D207D1832312F4028357E101139737011E
:100CE00063560700FD57231FF4005DBF231F040058
:100CF00045BFEF12EFD11754FF1F1304243E832783
:100D0000040B03D7C701C167FD17630EF710975790
:100D1000FF1F9387A7739C4381C70545EF4060770A
:100D2000C1690149930A400EFD19175BFF1F130BA0
:100D3000AB71EF70CFF3634BA90E1757FF1F03473B
:100D400067419307F00563E4E702EF704FED930509
:100D50000006B3C5A502B7F73600938707E8175515
:100D6000FF1F1305653FB385F502EF60A06F814556
:100D70001705000013058520EF60DFF8EFB0EFDE08
:100D800001CD0357C50109CB0357E50111C78347BF
:100D9000050299C3EF60A06BEFB06FDE31C5175746
:100DA000FF1F0347E7479757FF1F938767470DCFFD
:100DB00003C717002304E50003C72700A304E500C9
:100DC00003C737002305E50003C74700A305E50077
:100DD00003C757002306E50003C7670083C77700F2
:100DE000A306E5002307F5001C4493E717001757F7
:100DF000FF1F2329F72E5C4085E7EF708FEF0DC1B1
:100E0000EF702FEF44402A89EF70AFEE33F5A40264
:100E10005C40FD17CA97898F1757FF1F2322F72CB5
:100E20000145EF70DF9F01456F10CFC1B304590337
:100E30008327040BBE9483D7C40163883703138AC6
:100E40000403D2855285EFF0AFD605E183C7F401E4
:100E500099CF938594082E85EFF08FD509C9130695
:100E6000900581455285EF104FBF0509D9B58327FD
:100E70000B00268593B7170086072380F402EFE066
:100E8000FFB8E5B7854763F8A7009307F5FFBE9560
:100E90003305A040E98D2E8582809841C167BA97BD
:100EA00013D707016304A7009CC182804207998F72
:100EB000E5BFEF128FB741112EC63284B684EFB072
:100EC0000FCCE15701C9B24591E99757FF1F23891C
:100ED000073481473E8541016F106FB79D46175615
:100EE000FF1F1306F633A6852285EFF09FCFAA8752
:100EF00075F105479756FF1F2384E632E1BFEF12D5
:100F00002FB1411191E99757FF1F23AB071C0144F3
:100F1000228541016F100FB3B68532858D46700072
:100F2000EFF03FCC2A846DF58347D1000347E10001
:100F30001759FF1F1309891AA2074207D98F0347C0
:100F4000C100D98F1757FF1F232CF718EF706FDAE6
:100F500061D1EF700FDA83244900AA89EF706FD94D
:100F600033F5A40283274900FD17CE97898F1757C1
:100F7000FF1F2327F71669BFEF122FAB1C45AA846A
:100F800091CFD84B01CF83D7470089CBEF601F9219
:100F9000AA8509C588446105EF60C04C9757FF1FBB
:100FA000938747129C43014489EF6F104FAA9C48D6
:100FB00013171400BA9703D5070019C1EFE0CFCF7C
:100FC0000504EF70CFC7E344A4FEC5B7EF12EFA549
:100FD000011185E9EF605FDA01449757FF1F23ABEA
:100FE00007189757FF1F23A907189757FF1F23A715
:100FF00007189757FF1F23A50718228505616F1053
:101000000FA5B6873285C9467000BE85EFF07FBD5B
:101010002A8465F541469305E1001755FF1F130526
:101020006515EF80C0010355C100EF608FD7F1B7A0
:101030008DE19757FF1F23A3070A9757FF1F938739
:10104000E7099C470145ED9B1757FF1F232CF70825
:101050008280EF128F9D4111B68532859546300012
:10106000EFF03FB815EDA2471757FF1F2328F706EB
:101070009757FF1F938787069447B24713F7B6FF2A
:1010800013F6170019C213E74600858393F7F70795
:101090009756FF1F23A8E6041757FF1F230CF70AD4
:1010A00041016F10CF9AEF12AF9603841500DC4117
:1010B0002A89AE8485070387F7FF19C36340800C34
:1010C0008387240091C7635580007D146204618486
:1010D0009C40370700FF0907F98F37070010090701
:1010E0006392E70A6355800079146204618483C7C0
:1010F0000400858B95E39379F40F4E8A93178A0148
:10110000E187634AF008A287635304008147338470
:10111000F9407D14620461848385240081C54A8579
:10112000EFF0BFAA9C40370700FF0907F98F370788
:1011300000100907639AE706930500034A85EFF05C
:10114000DFA883C7040093058005918B99E393057D
:1011500080074A85EFF07FA783C70400858B81CB8A
:101160001374F40F93178401E1876347F004C040C0
:1011700005048305F4FFA1E96F10CF8C7D14620490
:1011800061840DBF370700080907E392E7F6E350D3
:1011900080F67D1499BF930500024A857D1AEFF011
:1011A000DFA2137AFA0F99BF370700080907E39502
:1011B000E7FA9305000371BF930500034A85EFF03A
:1011C000DFA07D1471BF4A85EFF03FA055B7EF1245
:1011D000CF85EF70CFAA2A84EF706FA92295894539
:1011E0000605EFE02FC6E55711C59757FF1F23AD42
:1011F000A7FE81473E856F108F8593070002630627
:10120000F5005D1513355500828005458280EF128B
:101210002F804111AA892A89130419008304F4FF3D
:1012200032C62EC42685EFF05FFDA245324659E155
:101230009307D0026392F408830404000548130462
:1012400029009377F6FEC9E793070003639FF40E26
:10125000830704001307800593F7F7FD6399E706FA
:101260008304140041460904B70600806314080093
:1012700093C6F6FFB3FEC6028147254F654EFD5F5C
:1012800033D3C602138704FD6368EF06BA8463D5BF
:10129000C408630DF5017D55636AF300639467002C
:1012A00063C69E000545B307F602A69705048304AE
:1012B000F4FFC9BF22898DB79307B0020148E392BA
:1012C000F4F8830404002A88130429009DBF01CA8E
:1012D0008947E31BF6F893070003E397F4F88307C5
:1012E00004001307200493F7F7FD639BE7048304CE
:1012F0001400094609048DBF13E704021307F7F928
:10130000636CEE009388F4FB1307700363741E0193
:1013100013077005998CA5BF7D576300E502630430
:101320000800B307F04091C519C19309F4FF23A049
:1013300035013E8541016F00FFF0B687FDF5D5BF51
:101340009304000315F2214605B719FE294629BF6B
:10135000EF021FEC011161540DC53284AE89414684
:1013600081453689EFF0BFEA93140501C180639E81
:1013700009002685EF30102B014401C58145EF207F
:101380005016228505616F00FFEB2285CD46700067
:10139000CA85EFF01F852A846DF52685EF309028E9
:1013A00009E90356C1008345E1012685EF20500B72
:1013B00001C941469305E1001105EF705048D1B7CE
:1013C0005D54C1B7EF02DFE40111E15401CDB284F5
:1013D000AE89414681453689EFF07FE32A846397E1
:1013E00009008144268505616F00DFE52685D14629
:1013F0007000CA85EFF0EFFEAA846DF58357C10037
:10140000EDD3EF700F8E4205931704014181C18324
:1014100063F9A702EFB08FB64204E147418033047D
:10142000F40241460C082A9413054400EF70304141
:101430008357E1002311F4008357C1002310F40007
:1014400055B7E55445B7EF02BFDC7971E15415C5D6
:101450003284AE8941468145B684EFF05FDB1319D3
:10146000050113590901639E09004A85EF40106583
:10147000814401C58145EFB02FB1268545616F00DC
:101480007FDCA6859306300270002285EFF06FF5B1
:10149000AA8465F54A85EF4070622A8411E54A8581
:1014A000EFB04F8C2A8431C58357C100231124012A
:1014B000930964002310F4008347E1009305F100D1
:1014C00041462302F4004E85EF7070371309740112
:1014D00041469305F1014A85EF707036930554003B
:1014E0004E85EFC04FBF930564014A85EFC0AFBE84
:1014F00069B7DD5459B7EF02BFD1797111E5E154F5
:10150000268545616F001FD4B284AE89414681456E
:101510003689EFF0DFCF131A0501135A0A015285FD
:10152000EFE06FCA2A846398090071D98145EFB052
:101530002FB48144F1B72685930610027000CA8546
:10154000EFF02FEAAA844DFD31C8B2479305D100D0
:101550004146858B230FF400B247130504038583AE
:1015600093F7F707A30FF400EF70702D4146930532
:10157000D10113059408EF70902C59B73304690317
:1015800083A70A0B3E948357C4016383370305097D
:10159000EF60FFEDE344A9FEDD549DB7C169014949
:1015A000975AFF1F938A8AB3130B400EFD19CDB7CC
:1015B000231E440159BF49CDEF029FC54111B28995
:1015C000AE8441468145368AEFF07FC4931A050107
:1015D00093DA0A010149175BFF1F130B2BB0EF6071
:1015E0001FE1634AA9000145ADCC81441759FF1F93
:1015F0001309C9AE81A883274B0B131439003E94FD
:1016000083570400638857050509D1BF8327490B19
:10161000139434003E948357040085E7231054014B
:1016200091467000D2854E85EFF0AFDB1DE9B247E1
:1016300013978700E1832183858B58C02301F40031
:101640000DA08504EF60BFDAE3C2A4FC5D5511A8CC
:1016500061558280F1F4214681452285EF00FFBF6C
:10166000014541016F001FBE1971D2C4130AC106A2
:1016700086CEA2CCA6CACAC8CEC6D6C2B6D6BAD85C
:10168000BEDAC2DCC6DE52C463810524FD151C101F
:101690002ACC2ECA02CE3EC89304B0021549A949ED
:1016A00083050600130416009DE1F2465247E24707
:1016B00063FBE620B697238007007245F640664438
:1016C000D6444649B649264A964A0961828093071C
:1016D00050026386F5004808EFF02FCFF5A8835736
:1016E000C10023070100014593F7C70F2316F1003E
:1016F000814501480147014681469308D002130302
:101700000003130E300205048307F4FF99C7638CAE
:10171000970463C3F404638BC70501CA0346C10081
:10172000858A799AD18E2306D10063090800834601
:10173000C100098BF59A558F2306E10019C12307D3
:10174000B100138707FD1377F70FA54663E2E6069E
:101750008146A545294535A0E38717FBE39F67FA36
:101760000546FD564DB70545854571BF05487D5772
:1017700059BFB386A60205048307F4FFBA96E206B2
:10178000E18613F7F70F130607FD1376F60F63E5EF
:10179000C500138707FDF1BF1306F7F91376F60F9F
:1017A000636EC902138797FAE30537FDA306D100DC
:1017B000130790066385E704634BF706130780055C
:1017C0006384E70A6345F702E38107EE13075002DB
:1017D00093055002E381E7F02286D9B51307F7FBA2
:1017E0001377F70FE364E9FC138797FC75BF1307C2
:1017F00030066386E70A13074006E39FE7FC0325EC
:101800000A00A947A307F100930A4A00635805009C
:101810009307D0023305A0402307F1006C00EFF0DE
:10182000AFB56C004808EFF01F88568A75B71307EC
:101830003007638EE7066341F7021307F006638EF5
:10184000E70413070007E399E7F80347C1001367AC
:1018500027002306E10009A813075007638BE7025E
:1018600013078007E39AE7F6938787FA414793B710
:101870001700A307E100139727008347C100ED9BE2
:10188000D98F2306F100930A4A006C0003250A0051
:1018900079B7A947A307F100FDB7A147E5BF8305C5
:1018A0000A004808930A4A00EFF02FB2BDBF832711
:1018B0000A006C0048083EC8EFF0EFFE1C10930AC7
:1018C0004A003EC89DB7BA97FDB30145C5BBEF02BC
:1018D000DF952A88368583464800BA870347580033
:1018E000A206D98E328717B600001306E68F89E567
:1018F00017B6000013060690BE85EFF0FFD66F0006
:101900001F959757FF1F938727919C4381CFEF0225
:10191000DF91D843B2862E861847AA853E85029766
:101920006F00FF9261558280EF023F908357050060
:1019300039712A84231EF100834745009305650011
:1019400041461305F101230FF100EF70406F93053D
:10195000740141461305F102EF70606E8356240056
:1019600017B6000013064691E5450A85EFF0DFCF74
:101970006C08130630020A85EFF0BFF821616F0092
:101980001F8DEF029F8A39712A8493050503414612
:101990001305D101EF70A06A930594084146130521
:1019A000D102EF70C0698347E4010347F401835615
:1019B000C401858B0607D98F17B600001306868CE5
:1019C000E5450A85230EF100EFF01FCA6C081306E7
:1019D00010020A85EFF0FFF221616F005F87EF02CE
:1019E0003F8337040001B70400FF0111814A174902
:1019F000FF1F1309A96E7D149389F4FF17BA000025
:101A0000130ACA8CEF60BF9E63C5AA0005616F0010
:101A10007F838327490B13973A003E97834737000C
:101A200095CF5C43A30107005286B3F68700824737
:101A3000E5454800E58FD58F3EC083462700B3F7C4
:101A40003701858AE206D58F835607003EC0EFF046
:101A5000BFC111468A854800EFF0BFEA850A5DB72D
:101A6000EF02AFFC01468145EFF0BFE96F002FFEAA
:101A700083576500638E071A1D71A2CCA6CACAC817
:101A800086CECEC6D2C4D6C2DAC05EDE801013F7D0
:101A900017003289AA8431CBF99B2313F500EF603C
:101AA0001F9906053D0541990A8BC16A3301A14082
:101AB0008A8B8149014AFD1AEF607F97634CAA0C1B
:101AC0007947930604FB17A600001306267FCA85F4
:101AD0002685EFF0DFDF638F090C13961900DE8592
:101AE000130504FBEFF0FFE15A8183D7640013F77D
:101AF000270021CBF59B2393F400EF605F9406054C
:101B00003D0541998A8A3301A1400A8B8149014AE6
:101B1000EF60FF926345AA0A6547930604FB17A688
:101B200000001306267ACA852685EFF05FDA638700
:101B3000090A13961900DA85130504FBEFF07FDC20
:101B4000568183D7640013F7470005CBED9B2393A1
:101B5000F4006547930604FB17A600001306C6763B
:101B6000CA852685EFF0BFD69C4481C703D74700BE
:101B70003DEB130504FBEFF0BFEE130104FAF64052
:101B80006644D6444649B649264A964A064BF25B15
:101B900025618280DC4413171A00BA9703D7070027
:101BA0006308570193971900DE972390E700850992
:101BB000050A19B7130504FBEFF09FEA35B79C48F7
:101BC00013171A00BA9703D7070019C7939719007C
:101BD000DA972390E7008509050A1DBF130504FB6A
:101BE000EFF01FE8B1BF2314E4FA03D767008326A0
:101BF000C4FA2146520751832315E4FA370700F04F
:101C0000758F9447930584FA130504FB920691821D
:101C1000558F2326E4FA83C7770013F7070183471C
:101C2000F4FABD9BD98FA307F4FAEFF09FCDB1B7BB
:101C30008280EF020FDD1744FF1F1304244A04447F
:101C4000797193F7F4FB1747FF1F232DF74893F79C
:101C50000404A1C78588A1E097A9000093890967BA
:101C6000EF60EFF863DBA4028327440B1399340081
:101C70003E998356090091CE4E86E5454808EFF01F
:101C8000BF9E4808EFF0DFDD214681454A85EF0021
:101C9000CFDC8504F1B7EFF09FD41C4413F7F7F7BE
:101CA0009746FF1F23A0E64493F707086397071E94
:101CB0001C4413F7F7EF9746FF1F23A5E64213F7DF
:101CC00007106318071E18449377F7DF9746FF1F26
:101CD00023AAF6409376072095C6058B630A072052
:101CE00018408983858B3ACA0347840715464C08F8
:101CF0000607D98F17A500001305055A230CF1001C
:101D0000EFF03FC01C4413F7F7BF9746FF1F23AB0C
:101D1000E63C93F707408DC3835744000D464C08BB
:101D2000231AF1008357640017A500001305055717
:101D3000230BF100EFF0FFBC1844FD749387F47F90
:101D4000F98F9746FF1F23AFF6389317470163DFDC
:101D50000700EFA08FE119C98356C5016391061AE8
:101D600017A5000013050554EFF09FCF1C447D77A5
:101D70007D177D8F9746FF1F23A6E6361397370101
:101D8000635A0702858B6388071CEFA04FDF1DC1D4
:101D900018458347E5001D463ACA0357C5004C085D
:101DA00017A5000013058550231CE100230DF10049
:101DB000EFF03FB51844F977FD17F98F9746FF1FED
:101DC00023A2F6329317270163D90700814517052F
:101DD0000000130525CAEF50FFF21844E177FD1704
:101DE000F98F9746FF1F23AFF62E9317070163D392
:101DF0000702EFA0BF982A84814417A900001309A5
:101E0000694BEF600FEE939704014205C183418156
:101E100063EAA71445616F004FC283A70A009314B9
:101E20001900BE9483D7040033F767011DCF1396C2
:101E3000170133F77701B3F637016352060417A68B
:101E400000001306664309E717A600001306864341
:101E5000E5454808EFF05F814808EFF07FC083D781
:101E60000400B3F747012390F4000509EF602FE168
:101E7000AA84EF60CFDF2695E341A9FA15BD368528
:101E800019C7EF40A04361DDEFF01FAAC9BFEFD033
:101E90009FB371D5EFF0FFAED9B785697D7A01495F
:101EA000974AFF1F938A4A34056B896BFD197D1A87
:101EB00075BF858B9DC7EF500FF3231AA1004146D4
:101EC0009745FF1F9385052B13056101EF702017C0
:101ED00049464C0817A500001305853BEFF07FA28B
:101EE000DDB317A500001305A53AEFF07FB7E1BBFE
:101EF00017A500001305453AEFF09FB621B503572B
:101F0000E501C17785073E978357A101FD1413377B
:101F100017003207E58FD98F231DF100231AD10056
:101F200083560502035725022146231BD100231C9B
:101F3000E100035745028566FD16758FFD76F58F26
:101F4000D98F4C0817A500001305C535231DF100D6
:101F5000EFF03F9B21BD17A5000013052535EFF0DD
:101F60003FB089BD5C4813F7E7FF58C8858B89CF20
:101F7000A6864A86C9450A85EFF00FEF835704000D
:101F800099E70A85EFF0DFAD850461049DBD231A52
:101F9000F100835724009305440041462808231B81
:101FA000F100EF70C00951464C080A85EFF07F95AB
:101FB000E1BFEF028FA785473395A7009747FF1F23
:101FC0009387C7119C47411181455D8D9747FF1F3E
:101FD00023AAA7109377057085E393576500858B37
:101FE000A1CBC167938707887D8D05EDEF606FD129
:101FF0009305803EB305B5021745FF1F1305051F66
:102000002EC6EF50A03BB24519C16349B50085C546
:102010001745FF1F1305851DEF50C04441016F0098
:102020000FA3EF600FCE2A84EF60AFCEE360A4FC75
:10203000EF602FCE75BF0145EFF0BFBFC5B7EF0210
:10204000CF9E7971AA8601441749FF1F1309090918
:1020500036C6EF60CFB9B246635CA4028327490B52
:1020600093143400BE9483D704006396D70285C6C8
:1020700017A6000013068625E5454808EFF0CFDED9
:102080004808EFF0FF9D214681452685EF00EF9C33
:1020900045616F00CF9B050465BF19C22320060070
:1020A000814701C59306D00389E53E858280850579
:1020B0000505838705000307050099CF6394E700B2
:1020C000E397D7FE8147D5B79306D0038547E30E44
:1020D000D7FC93371700D1BF9307F002E316F7FE42
:1020E000854761D6050508C2C9B799C123A0050077
:1020F00081470DC11308D0031306F0023307F50022
:102100008306070081CA638706016397C60099C1E9
:10211000050798C13E8582808507CDB731C9EF029A
:102120004F8E41112E8A6C002A89368BB28A97A471
:1021300000009384640DEFF05FFB2A8C0144A689B4
:10214000B14B88406286CA85EF70E01701ED0E043E
:102150004E945C403245DA865686D285829741019C
:102160006F00AF8D0504A104E31D74FD6155C5BF6B
:102170007D55828099E561558280615505616F00CA
:102180006F8CEF02EF882E8A2A8401118145B28478
:1021900052854146BA893689EFF06F87931505015C
:1021A000C1811376F50FA1812285EF507FB12A847A
:1021B00069D552854C08EFF05FF3524A2A8BE30E43
:1021C0000AFA2A8697A500009385450F5285EF707D
:1021D000800FAA8A0DED7D5AEF606FA563C5AA0036
:1021E00099E8014561BF5C4413971A00850ABA97C4
:1021F00023904701D5B74C442EC6EF604FA3B2459C
:10220000131615004E850299E34DA0FC85BF5A8632
:1022100097A500009385050B5285EF70C00A0DE16C
:10222000032A0401EF60AFA1131615008145528502
:10223000EF00AF82DDD40C482EC6EF604FA0C1B7CF
:102240005A8697A50000938525085285EF70A00750
:1022500041E11C44A5CF81ECD443370700E0758FE2
:102260009447D8C33707001F758F98C701BFA14691
:102270003008CE854A85EFE0DF96E31105F018447B
:10228000835781017D762312F7008357A10193962E
:10229000470183576700D182F18FD58FF2467D7653
:1022A0007D16F182858AB206F18FD58F2313F70050
:1022B0008347E1018356C1012305F7008347B70037
:1022C0002314D700FD8BA305F7004DBD7D557DB5CB
:1022D0005A8697A500009385A5F25285EF60B07EDF
:1022E000E31D05E81C4CE38A07E89C43E38707E805
:1022F000CE864A86A6852285829749B5EFF2FEF200
:102300003687B2862E86AA850545EFF0BFE66FF0C8
:102310001EF4EFF29EF13687B2862E86AA8501451D
:10232000EFF05FE56FF0BEF2EFF29EEE411199C162
:1023300023A005009747FF1F938707ED8043814443
:102340001DC82E89AA8931141DC40C4070004E8509
:10235000EFF0BFD419CD81E8A284630C0900B24725
:102360002320F90039A08C4008400146EFF0FFD24D
:1023700065F5404869F8268541016FF0BEEC1841CB
:1023800011CBEFF29EEAAE873E85B2853686029784
:102390006FF0FEEB35558280EFF23EE98357C500C2
:1023A00013D70501C205B387E7021841C181484927
:1023B000BA95BE95EFF0BFFC6FF07EE9584111CBA6
:1023C000EFF2BEE6AE873E85B285368602976FF0A5
:1023D0001EE835558280184509CBEFF21EE5AE8721
:1023E0003E85B28502976FF09EE6355582805C454A
:1023F00099C7EFF29EE32E8582976FF05EE5355523
:102400008280EFF2FEE083290500035AC5002A848A
:102410004849AE848145EFF09FFD2A890DE193D5AF
:102420000401B38545030356C4004848CE95EFF038
:102430009FFA2A8909E548488545EFF05FFB4A8500
:102440006FF05EE0EFF2DEDC2A890441035BC50039
:10245000484979712E848145B28A368AEFF03FF976
:1024600041E193590401B3896903420441802694F0
:10247000A29903440901330480403374440111CC10
:1024800003254901A2865686CE85EFF03FF3AA8444
:1024900031E1330A8A40A299A29A8144630C0A026C
:1024A0005286D685080803244901EF6050398346D7
:1024B00009011C089305F00F338646413385470117
:1024C00036C6EFF09ED9B2461008CE852285EFF0D1
:1024D000FFEEAA84032549018545EFF05FF12685CB
:1024E00045616FF03ED6EFF25ED42E864C41A14698
:1024F0002A84EFF03FF5AA8403450401A145EFE0EB
:102500007F985C403385A74048C026856FF03ED455
:10251000814797A60000938626CC6393C7008280EC
:102520003387F500034707008507398D13574500AA
:102530003697034707001205398D1375F50F1357AA
:1025400045003697034707001205398D1375F50FBF
:10255000E9B7EFF29ECD2A84AA851D461305F00F38
:10256000EFF01FFB834774003385A7403335A0008D
:102570006FF0FECDEFF27ECB4111A1463000EFF0BF
:10258000BFE109ED03578100C167FD1705456317DA
:10259000F7002800EFF0FFFB3335A00041016FF09A
:1025A0001ECBEFF2FEC6AE848C414111A1462A89B2
:1025B00003440501EFF05FDEAA8939E9A1452285D0
:1025C000EFE05F8C9C400357C9002A8AAA97939634
:1025D00007019CC0C182098F639CE602C16513D7C5
:1025E0000701B385B74011E78355E900FD15C20522
:1025F000BE958CC0A1460A864A85EFF0FFD9AA890C
:1026000001E90A85EFF0FFF401C9832749009CC066
:102610004E8541016FF01EC30357C9008357210047
:1026200080403307474163DBE70033FA4703631712
:102630000A004177798C3E9480C0D9BF03450901D7
:10264000A145417AEFE01F84098CAA8A80C0337AC1
:102650004401417B63648A0081495DBFA14630002B
:10266000A2854A85EFF05FD3AA895DF12800EFF0DB
:102670005FEE11E98357A1000357C100337A6A0165
:1026800080C0BA973E9A33045441E9B7EFF2FEB9DD
:102690002A84AA851D461305F00FEFF07FE7A303F8
:1026A000A4006FF0DEBAEFF2DEB52A84034505011F
:1026B0005D71A145EFE00FFD5C402A8B0355E400FE
:1026C0004179B3F727016C003EC6EFE00FFD83555B
:1026D000C400B247A1463008BE95B3856541228546
:1026E0002EC8EFF07FCBAA84634B05002808EFF0DB
:1026F0005FE611C9B2452285EFF0BFD0AA842685D6
:1027000061616FF09EB3C2470357A101417C338BD7
:102710006741B3F72701BA973EC810100C0822850D
:10272000C24BEFF01FE8AA8479F90810EFF07FE2BE
:102730002DE95C403ECA30104C0822855249EFF02A
:102740005FE6AA844DFD0357810283570102631699
:10275000F7002810EFF0FFDF09C55840D247E31C0F
:10276000F7FC63902B058357410285CF83572102E5
:10277000B3FA8B010810BE9A1C442311F102EFF04A
:10278000FFF083490401035A4102B309304193F930
:102790000902631B0A000C102285EFF0DFD4AA8423
:1027A00039FDE31C7BF7B9B74E8963733A0152894F
:1027B000CA861018D6852285EFF01FBEAA8421F1A3
:1027C000630909000C44CA8610182285EFF09FC7E0
:1027D000AA8403450401CA85EFE0CFEA1C443E9574
:1027E00008C4E39E04F0330A2A41CA9A5DB7EFF2A7
:1027F0003EA2411191E5FD54268541016FF09EA452
:10280000C44983D725014CC904C12316F50003C769
:1028100005012A842317E50003C515019316070156
:10282000130700022308A400C182E366A7FCE1D7D6
:10283000B3E4F402E9F08547E3FFD7FAA145EFE0FE
:102840006FE4AA89014A01498357C400931509011D
:102850002285BE95B38535412EC2EFF0BFD119ED6B
:102860000355E4004C00050AEFE02FE39245420ACD
:102870002285135A0A01EFF0FFCF09E905098357B2
:10288000E400420913590901E360F9FC8357E400AD
:1028900063944701D1548DB7639427039245A146B1
:1028A0003000B38535412285EFF01FAF35E12800B8
:1028B000EFF03FCA11C50355E4004C00EFE0EFDD37
:1028C0009247C17A3387374158C04177F98F1CC48A
:1028D0004C401C4463EEF500A14630002285EFF029
:1028E000BFAB1DE52800EFF0DFC6032A44001DC181
:1028F0005C400355E4004179B3F727014C003EC228
:10290000EFE0AFD992452285EFF0DFC6635C0502A8
:10291000AA84DDB512450359A100035BC10033F55C
:10292000AA002A9903450401DA85EFE0AFD54A955C
:1029300008C46314450163130B04330A3A4123228C
:10294000440179B709C58547A308F40075B54C4023
:102950002285EFF01FAB4DFD48408357C400860928
:102960003375A9003E953305354148C033752501BF
:1029700008C42285EFF03FD379D559BF4D5549BFE3
:1029800083471501C9CFEFF2DE872A84034505018D
:1029900041112E8AA145BA893689328BEFE08FCE5C
:1029A0008357C4000605898F7D5563E727075C4080
:1029B00081443EC230004C002285924AEFF07FBE37
:1029C00021ED835B810063994B012800EFF07FB814
:1029D00001E58504C204C18058409247630BF702A9
:1029E000E3FA99FC8356C10061559DC663E6340342
:1029F000C175B3FABA006373D900CA868355A100C2
:102A00005A862285D695EFF03F9919E50355C10006
:102A100021A06155E3884BFD41016FF01E824955AD
:102A20008280EFF29E800147EFF09FF56FF03E82CB
:102A3000EFF2AEFF3284B2862E8683554500084100
:102A4000EFF03FFE635385002A8422856FF03E80BD
:102A5000EFF2AEFA834715013971C954BDC7034B74
:102A600005012EC62A84A1455A853689328AEFE0AF
:102A70006FC10D473307E5028357C400AA8DFD548B
:102A8000998F63E427056304090063000A045C402E
:102A90003ECA30084C082285524DEFF09FB0AA89FB
:102AA00045ED8357810132476397E7002808EFF02F
:102AB0005FAA630605105840D247E31CF7FC814427
:102AC000631B090019A0814499E7268521616FF0F5
:102AD0008EF6E35CA0FE5A85CA85EFE0AFBA014BE3
:102AE00011C5330BB501420B135B0B01014D7D5C2E
:102AF000C17B930C44008357E4006380A70D1C4402
:102B000044403307FB0063EBE40432472311F10236
:102B10000810FD572310E102231221032303F102C1
:102B2000EFF0DFB6630909000C44CA86528622859D
:102B3000EFF05F91AA8903450401CA85EFE08FB4E5
:102B40001C443E9508C4639909000C102285EFF0DF
:102B50009F99AA89CA8435D9CE8485BF03450401CB
:102B6000A145EFE02FB2B387A4002311F1028357F0
:102B7000C400B3F4740123108103BE94898C44C053
:102B8000081023120102EFF07FB00C102285EFF045
:102B90009F95AA840355E400E685EFE00FB05C4002
:102BA000B3F777011CC4E39204F22285EFF0BFAFC4
:102BB000AA84E31C05F0050D3DBFC15439B7835706
:102BC000C101E30209F0E39827F1C177034C040146
:102BD000B377FD00035DA101330C8041137C0C022F
:102BE0003E9DD28ACA8CE28B63F38C01E68BDE8633
:102BF0001010EA852285EFF02FFAAA84E31B05EC7A
